:020000040000FA
:040000006FD00400B9
:101000006F00507B000000000000000090200020D6
:10101000AA220020A9BDF9F56C23002000000000E1
:10102000000000006C230020902000200000000041
:101030000000000090200020000000009020002010
:101040000000000090200020902000209020002030
:101050009020002090200020242F00205E240020DB
:101060000000000090200020902000200424002098
:1010700090200020D22300209020002090200020EB
:101080009020002090200020902000209020002020
:101090009020002001A04111B7170040985F3AC688
:1010A000945F3247E39CE6FE3245410182800111A4
:1010B00013078008F337078093F787083EC20100C3
:1010C0000100B7170040930570052380B70413068D
:1010D00080FA2380C7040100010083C6B70493F699
:1010E000F60DA385D704238007049246F3A6068055
:1010F0000100010093760502D5CEF336078093F602
:10110000860836C4010001002380B7042380C70489
:1011100001000100B70614007D89558D88C70100C4
:1011200001000100010023800704A246F3A6068007
:101130000100010073370780137787083AC6010062
:1011400001002380B7042380C704010001000100CF
:1011500001003727004093061005A303D7802380A2
:101160000704B247F3A70780010001009307800836
:10117000F3B7078093F787083ECE01000100B71749
:101180000040130770052380E704130780FA2380CB
:10119000E7040100010003C7B70413670708A3852C
:1011A000E70423800704F247F3A70780010001004A
:1011B0000561828093760504BDC6F336078093F6F9
:1011C000860836C8010001002380B7042380C704C5
:1011D00001000100B7061400938606047D89558D31
:1011E00088C7010001000100010023800704C246F6
:1011F000F3A6068001000100733707801377870884
:101200003ACA010001002380B7042380C70401000B
:1012100001003727004093062005A303D7802380D1
:101220000704D24781B773370780137787083ACC12
:10123000010001002380B7042380C70401000100DE
:1012400098471367070C98C723800704E24719BF24
:101250000111814601468145114506CE97000000E7
:10126000E780005593078008F3B7078093F7870856
:101270003EC601000100B717004013077005238028
:10128000E704130780FA2380E7040100010003C785
:101290006704136717002383E70423800704B2471A
:1012A000F3A7078001000100F2400561828041112F
:1012B000814601468145114597000000E780404F77
:1012C00013078008F337078093F787083EC40100AF
:1012D0000100B7170040130670052380C70493066A
:1012E00080FA2380D70401000100FD552396B70240
:1012F00023800704A245F3A5058001000100733790
:101300000780137787083AC6010001002380C704CD
:101310002380D7040100010003C767041367170087
:101320002383E70423800704B247F3A70780010063
:10133000010001A0BD473305F50201007D1575FDD3
:101340008280411122C426C206C6AA8401446317C2
:101350009400B24022449244410182800504130566
:10136000803E420497000000E78000FD4180C5B741
:101370009305000273A04580824573901534924016
:101380002242B2424243D2436244F2440255925551
:101390002256B2564257D2576258F25806499649D9
:1013A000264AB64A464BD64B664CF64C065D965DD1
:1013B000265EB65E465FD65F09617300203041113C
:1013C000B7170040985F3AC6945F3247E39CE6FE49
:1013D000324541018280B71700401307000323887C
:1013E000E702854717170000232EF74273002030CD
:1013F000411122C406C637040020976000E0E78050
:10140000A0E11C408297D5BF373700408347470093
:101410009146BD8B6389D70099466394D700834773
:101420005740730020309736000083C6662C9387A0
:10143000160017360000230DF62A0347870097375A
:1014400000009387E71AB6972380E700B7E7040008
:10145000BC4F0946894517150000034565F482977E
:10146000C9B7B787004003C76700098B6309071036
:1014700003C777009306000313770703630DD708AC
:10148000173800000348586217360000130606613B
:101490000547B30606012380E60083C577001737AA
:1014A000000013072760429793F5F50F2300B7005C
:1014B00003C58700973500009385855EC295137537
:1014C000F50F2380A5000347070089451377F7032D
:1014D000630CB70C63E7E50A6306071A8545630CDE
:1014E000B7129737000083C7375C3307F60003470E
:1014F00007001377F70F19CB850793F7F70F0D4701
:101500006363F71A17370000A300F75AB787004044
:1015100009472383E700B787004083C77700E207C6
:10152000E18763DE07049737000083C7F757173753
:1015300000001307A7563E9785462300D7001737AC
:101540000000130727563E97930600032300D70099
:10155000173700001307C7543E97A146850723009D
:10156000D70093F7F70F0D476364F71417370000A0
:10157000A30CF752B787004009472383E7007300A5
:101580002030930610026300D70E930620026305F5
:10159000D70693060002E316D7F403C72702137792
:1015A000C70F13672700D5A803C767001377070481
:1015B00065CB03C7A702173800001308A82F1735FB
:1015C00000001305E526134707082385E70203C734
:1015D000A7021377370F136787002385E702814738
:1015E00013070004B305F5008C41B306F80091071A
:1015F0008CC2E399E7FEF5B503C7A70213470704BA
:101600002385E70203C7A7021377C70F13672700D5
:101610002385E702F9B503C767001377070449C3B9
:1016200003C76702173800001308881C173500002D
:101630001305C513134707082383E70203C767028F
:101640001377370F136787002383E7028147130758
:101650000004B305F5008C41B306F80091078CC275
:10166000E399E7FEBDBD03C7670213470704238361
:10167000E70203C767021377C70F136727002383A7
:10168000E70285B503C767001377070411CB03C7CB
:1016900027021377370F136787002381E70291B57D
:1016A000238006003DBD97370000A38F073EB9BDDC
:1016B00097370000A38A073E75BD230304801547B2
:1016C0002303E48001002302A480828083076480D6
:1016D000E3CE07FE23030480828083076480E3CE89
:1016E00007FE03454480828083076480E3CE07FEC3
:1016F0002302A4808280411126C44AC24EC006C67D
:101700001377F50BAD47AA892E899544630CF70032
:10171000194597000000E78080FA97000000E780F5
:1017200020FB8D444E8597000000E78040F9FD596D
:10173000FD1463983401B240A24412498249410128
:101740008280135509011375F50F97000000E7809B
:10175000E0F92209F1BF011126CC06CEB70408003A
:1017600097000000E780C0F6154597000000E7806D
:1017700000F597000000E78080F697000000E78002
:1017800000F62AC697000000E78080F43245937780
:10179000150089EB136515001375F50FF240E2444F
:1017A00005618280FD14E9F00145CDBF397126DC69
:1017B0004ADA4ED852D656D45AD25ED006DE62CE1F
:1017C00066CCB7E700E07D5783AA070022C603AACC
:1017D000470023A0E71823A2E718B7170040130714
:1017E00070052380E704130780FA2380E70483C78A
:1017F0004704930B75FFB684E20793FBFB0F854606
:10180000AA892E8B328937240040E187015763FA79
:1018100076016308D5008946130700026313D500DB
:101820000157D98F93F7F70FB71C00402382FC04B0
:1018300011472303E4801305F00F97000000E780B1
:1018400000E8094C97000000E78080E863657C159C
:10185000B7050700DA9537870700795563FEE50479
:10186000B3879500636AF704370B0800A94733EB89
:1018700065016395F90881E8814497000000E780DD
:1018800020E5268515A8DA85094597000000E78040
:10189000C0E605090345F9FFFD14050B970000009C
:1018A000E780C0E481C49377FB0FE5F79700000061
:1018B000E780A0EA69F17D55B7170040130770056E
:1018C0002380E704130780FA2380E70403C7470453
:1018D000418B2382E704F250B7E700E023A05711C1
:1018E00023A24711E25432445259C259325AA25AE1
:1018F000125B825B724CE24C21618280A547639B44
:10190000F90685691309F00FB3069900B3742B012A
:10191000B6941349F9FFB3749900856B3379690163
:10192000416B9387F9FFB3F7270199E363FC340117
:1019300093D94900C147E3E637FF3DBF0569C16957
:101940007D19D9B71305800D63886901130500025D
:101950006384790113051008CA8597000000E780A9
:10196000C0D997000000E78040DF31D54E99B3849D
:1019700034416DBFDA852D4597000000E780E0D740
:10198000CA94E30B99EE050997000000E78020D583
:10199000A30FA9FEFDB79387F9FF93F7F70F636DC8
:1019A000FC0C83C71C04130730086315F7063707C0
:1019B00008006361EB06B3079B00B706100063FBEA
:1019C000D704334BEB0089476399F9068980D549E1
:1019D000E38404EADA85094597000000E780E0D156
:1019E00011090327C9FF91472320E480030764807E
:1019F000E34E07FE23033481FD17EDFBFD14110BAD
:101A000081C49377FB0FE9FF97000000E780E0D4E3
:101A100061F155B5B717004003C75704B707080071
:101A20001377070219E3B78707007955E376FBE8D8
:101A300033079B00E3F9E7F841B58547E380F9F008
:101A4000DA852D4597000000E78020CB9389F4FFCD
:101A5000E38404E297000000E78060C893F7390050
:101A600091EB832604800327090093074900E3963E
:101A7000E6E03E89CE84D9BFB5476399F9001305E6
:101A8000900B97000000E78080C3FDB3B1471305BA
:101A9000B00AE388F9FE99476397F904B70508008F
:101AA000B365BB002D4597000000E78000C5814469
:101AB0008D4BA14997000000E78060C263967401D6
:101AC000832704802320F9008504E39534FF8327CE
:101AD000048013172B01635507002312F90069BB1B
:101AE0002322F90051BB9D47639FF90281451305ED
:101AF000B00497000000E78040C0BD4423200900E7
:101B000023220900FD5997000000E78040BD93F7AC
:101B10007400CA9703C70700FD14398D2380A700FE
:101B2000E39334FF91BBA1476397F9069700000048
:101B3000E780A0C28144630D0B008D479304C0036E
:101B40006308FB009304000563048B0193044004C5
:101B50001375C507E30295D2194597000000E78089
:101B600000B697000000E780A0B60545970000008A
:101B7000E780E0B4268597000000E78020B709459C
:101B800097000000E78080B697000000E780E0BC87
:101B9000E31405CE0DB39147639FF900130560066A
:101BA00097000000E780A0B197000000E78040B2F6
:101BB00013059009F9B5E38109CCF1547DB9BD66EF
:101BC0000147173600001306660B938606A6854567
:101BD0008347060093F7F70F91C382800507E3F967
:101BE000E6FE97370000238BB708DDB77D16620647
:101BF000618693178601E18763D4070001458280DF
:101C0000931726003307F500AE9718439C4363E70C
:101C1000E7007D16E37FF7FC7D55828005458280D5
:101C2000FD15E205E18513978501618793F7F50FAF
:101C300063480700FD15139725002A97584365D779
:101C4000138517006205618582803308B5021C4246
:101C500083A80600B335B502C29733B50701AE9825
:101C6000469585486367B5006394A50063E3070163
:101C700081480C43C6950CC388C21CC28280814730
:101C80001397870161876343B7008280139727000A
:101C90002A97232007008507E5B7814701479396D8
:101CA0008701E18663C5B6001335170082809396DD
:101CB0002700AA9694428507558FD5B793D75540EC
:101CC0008A07AA979C4305453315B5007D8D828010
:101CD00017F3FFDFE702A33D2A8497000000E780A7
:101CE00060F405C5931725003E940327C4FF814780
:101CF00011EB7D1516053E954205418517F3FFDF73
:101D00006700233D05838507E5B70145C5BF8147CA
:101D10001397870161876343C70082801397270069
:101D2000B386E50094422A97850714C3D5B77D167C
:101D300062066186014793178601E18763D5070034
:101D400013351700828093172600B306F500AE976F
:101D500094429C437D16B58F5D8FF1BF8A05AA958D
:101D600001476363B500828083A6C5FFF11593D751
:101D70001600D98F9CC11397F601E5B72A83014855
:101D8000014701456343D7008280B387050183A8DB
:101D90000700B30706019C43C697AA976384F8001F
:101DA00033B517010507B3080301620723A0F80044
:101DB00061871108C1BF2A8301478147014563C379
:101DC000D70082803388E50083280800330EE600C0
:101DD000032E0E003388A8403308C84163840801ED
:101DE00033B508018507B308E300E20723A0080123
:101DF000E1871107E9B717F3FFDFE702432B011172
:101E0000B286B2842E86AA850A8597000000E780F4
:101E1000C0FA2A84A6850A8597000000E78020E89A
:101E200033348000060413351500018D056117F366
:101E3000FFDF6700032A17F3FFDFE702C324411126
:101E4000AA89AE8A328BB68402C202C402C6014499
:101E5000131C8401135C8C4163499C02939B140006
:101E6000FD1B0549138CF4FFF15C33048901620406
:101E700061846340740792478E04CE9423AEF4FECF
:101E8000410117F3FFDF6700832313192400B30B0D
:101E90002B01014A93172A00D69783A50B0088438C
:101EA00078003400500097000000E78040DA050A0F
:101EB00093178A01E187F11BE35EFCFC92474E9980
:101EC00005042320F900A2473EC2B24702C63EC421
:101ED00041B7131A8901135A8A41131D240093171D
:101EE0008A01E18763CF970092470A044E941CC091
:101EF000A24705091379F90F3EC2B24702C63EC494
:101F0000ADB7B3079A0313152A0056950841780018
:101F100034005000050AEA97DA978C4397000000D6
:101F2000E780E0D26DBF0000197106C212C416C668
:101F30001AC81ECA22CC26CE2AD02ED232D436D6E9
:101F40003AD83EDA42DC46DECAC0CEC2D2C4D6C6D9
:101F5000DAC8DECAE2CCE6CEEAD0EED2F2D4F6D6C9
:101F6000FAD8FEDA971500009385458B8841E70083
:101F7000050092402242B2424243D2436244F244BC
:101F8000025592552256B2564257D2576258F258CD
:101F900006499649264AB64A464BD64B664CF64CFD
:101FA000065D965D265EB65E465FD65F096173008C
:101FB00020300000972100209381C1041751002098
:101FC0001301418417F5FFFF130505049705002051
:101FD00093854503171600201306C6FD63FAC50056
:101FE0008322050023A0550011059105E3EAC5FEF3
:101FF00017050200130505D197150020938585FB71
:10200000171600201306066563FAC5008322050033
:1020100023A0550011059105E3EAC5FE1715002020
:102020001305456397450020938545116377B500F7
:10203000232005001105E36DB5FEFD42739002BC3F
:102040008D4273904280B722000093828288739001
:102050000230970200209382E2FA93E232007390FA
:1020600052309752000093820297739012346FB0EF
:10207000347973002030397101436EC619A039716B
:1020800041536AC866CA62CC5ECE19A03971015349
:102090005AD056D252D44ED64AD826DA22DC06DEA0
:1020A00033016140828241114AC026C222C406C661
:1020B0008282B24D4101024D924C224CB24B410101
:1020C000024B924A224AB2494101024992442244B7
:1020D000B240410182803D432A876373C3029377F4
:1020E000F700BDEFADE5937606FF3D8ABA960CC3C7
:1020F0004CC30CC74CC74107E36BD7FE11E282808B
:10210000B306C3408A069702000096966780A60031
:102110002307B700A306B7002306B700A305B7003F
:102120002305B700A304B7002304B700A303B70037
:102130002303B700A302B7002302B700A301B7002F
:102140002301B700A300B7002300B700828093F5F6
:10215000F50F93968500D58D93960501D58D61B7C2
:10216000939627009702000096968682E78086FA6B
:102170009680C1171D8F3E96E374C3F8A5B73367E9
:10218000B500FD530D8B79E7B7877F7F9387F7F70E
:1021900010419441B372F6003363F600BE92B3E28D
:1021A00062006397720C6318D6065041D441B37233
:1021B000F6003363F600BE92B3E262006398720ADF
:1021C000631BD60410459445B372F6003363F600E2
:1021D000BE92B3E262006391720A631ED60250455A
:1021E000D445B372F6003363F600BE92B3E26200E8
:1021F000639A72086311D60210499449B372F600CB
:102200003363F600BE92B3E2620063937208510535
:10221000D105E30FD6F61317060193970601631C49
:10222000F7001357060193D706013305F74093755E
:10223000F50F91E982804183C1833305F74093759F
:10224000F50F91E182801377F70F93F7F70F3305BE
:10225000F74082800346050083C605000505850515
:102260006313D60065FA3305D640828011059105C7
:10227000E312D6FE014582802105A105E31CD6FCB0
:10228000014582803105B105E316D6FC0145828007
:102290004105C105E310D6FC01458280B717004017
:1022A00003C777051377E70FA38BE704130700F83D
:1022B000A38DE7043D47238CE70413075003A38C49
:1022C000E70403C7A7051377D70F238DE7048280A0
:1022D000B717004003C7E7020D8941111377C70FF5
:1022E000498F93068008F3B6068093F6860836C6B3
:1022F00001000100930670052380D704930680FA3D
:102300002380D704010001002387E702238007040C
:10231000B247F3A70780010001004101828041110B
:102320002A83014E930E407E130F0019930F40062F
:1023300063E56E129308001913034006B378150382
:10234000854E0D4FA14F337365020D89133515006E
:1023500063EFBE121308F6FF7946729842081358CD
:1023600008013307C70213D61700BE07329761462C
:10237000B3F6C60213068070B386C6023697A1660E
:10238000F58F42075D8FB716004083C7F60293F7BB
:102390000708A303F1000346710083C7F60293F711
:1023A0000708E394C7FE83477100B716004093F710
:1023B000F70F6388071293078008F3B7078093F736
:1023C00087083EC401000100B7170040930670055E
:1023D0002380D704930680FA2380D70401000100EC
:1023E00023AA070383C6170393E60608A388D70228
:1023F00023800704A247F3A70780010001001166AC
:10240000B71700407D16D45BC85F93854703A98E3C
:10241000F18EF5FA93068008F3B6068093F68608E7
:1024200036C601000100930670052380D704930689
:1024300080FA2380D7040100010098C103C7170365
:1024400013670704A388E70223800704B247F3A7B2
:10245000078001000100410182807D133368E3039E
:102460009308E016630E08003368F3039308D01650
:10247000630808009378330093B818009388D8163F
:1024800033081E01131E0801135E0E0155B5639338
:10249000E5030548638608000148630303002A88B2
:1024A00071087298FD15131E0801C205135E0E0116
:1024B000C18179BD13F8150063F4BF007908D5B761
:1024C00013381800E5BF83C7F60293F70708A30384
:1024D000F1000346710083C7F60293F70708E394FF
:1024E000C7FE8347710093F7F70FF1DFE9B531714C
:1024F0004AD966CB06DF22DD26DB4ED752D556D32E
:102500005AD15ECF62CD6AC96EC7AA8C02D8971025
:102510000000E78020B12A8993078008F3B707807D
:1025200093F787083EDA01000100B7170040130750
:1025300070052380E704130780FA2380E704010075
:10254000010003C7F7021377770FA387E70203C7DA
:10255000F70213678700A387E70223800704D25797
:10256000F3A7078001000100054597000000E78000
:1025700060D6130780C13347E902116A93070AE85E
:1025800093065002BD69930BA004814A014B1304CA
:102590008008930470057D1AB347F9023307D70208
:1025A0003EC0FD873ECC938709A69309803E334702
:1025B000F7023AC27D873AC4334739038549B39954
:1025C000990193D93940B306D702B30B7703B3C649
:1025D000F602B3CBFB0236C6FD8636C893D6FB4166
:1025E00036CEB7460F00938606243349D902856656
:1025F000938606FAB3969601B389E90213076055EC
:102600003309D90293060010B389E9023349D9028C
:10261000B3C9F9029316390036CA37190040FD864E
:1026200036D0930D090493D7F9413ED2F336048096
:1026300093F6860836DC01000100930770052380BD
:10264000FD00930680FA2380DD000100010083462F
:10265000390593F6860FA309D9048346390593E615
:102660001600A309D90423800D00E256F3A60680C4
:1026700001000100130C80FA116DF336048093F60B
:10268000860836DE01000100930770052380FD00F7
:1026900023808D010100010083463905216693E600
:1026A0000602A309D90483560905B3E6A601231837
:1026B000D90483560905D18E2318D90423800D002F
:1026C000F256F3A60680010001008346390593F611
:1026D00006026381061A03463905218A6DDE081851
:1026E00097100000E7800098733604801376860800
:1026F000B2C20100010023809D0023808D010100F2
:102700000100B717004003C637051376F60DA389FD
:10271000C70403C6370513660602A389C704835698
:1027200009052166B3E6A6012318D90483560905D5
:10273000D18E2318D90423800D009646F3A6068077
:10274000010001008346390593F60602638B0614E7
:1027500083463905A18AEDFE97000020E780A0930B
:10276000AA8636D497000020E780E092A256E30ABA
:10277000D5FE835609054255B3E6A6012318D904B0
:1027800097100000E780C08F83463905A18AEDDEEF
:10279000035609058346290582473376CA00B306E6
:1027A000DA0293D5F641B296B388F640E24733B8E1
:1027B000C6002E983308F840A247B3B61601330876
:1027C000D84063C70701631DF800924763FA1701F9
:1027D000C247634FF80E63950701B24763EAF80EEC
:1027E000894663E9660FF2469315180013D3F80182
:1027F0005E8613951800B365B30042D646D497B0F1
:102800000100E78060793258050B137BFB0F6347AB
:102810000001631A0838A2586387083813081500A6
:10282000B336A800B69513D6F5013298B336C80072
:10283000AE9613581800FE06B3E606017336048000
:1028400013768608B2C60100010023809D00238014
:102850008D01010001000356C902B296C206C18271
:102860002316D90223800D00B646F3A60680010088
:10287000010021B5F336048093F68608B6C0010046
:10288000010023809D0023808D010100010083460B
:10289000390593E60602A309D90423800D00864674
:1028A0000DB5F336048093F68608B6C40100010026
:1028B00023809D0023808D0101000100834639059E
:1028C00093E60602A309D90423800D00A646BDB5F0
:1028D000E30B0BF0F336048093F68608B6C80100CC
:1028E0000100930680FA23809D002380DD00010013
:1028F00001008346390593F5FC0F93F6860FA30973
:10290000D90483463905CD8EA309D90423800D004F
:10291000C646F3A6068001000100130580FA0346AF
:102920003905930639051D8A631C96297336048080
:1029300013768608B2CC01000100130680FA2380CA
:102940009D002380CD000100010003C60600137620
:10295000F60D2380C60003C6060013660602238018
:10296000C600835609051166D18E2318D9048356F3
:1029700009052166D18E2318D90423800D00E6466F
:10298000F3A6068001000100130680FA834639058C
:1029900093F606026380062683463905130C390533
:1029A000A18AFDDA081897000000E780A06BF336D3
:1029B000048093F68608B6D001000100930680FAE1
:1029C00023809D002380DD000100010083460C0070
:1029D000116693F6F60D2300DC0083460C0093E6A7
:1029E00006022300DC0083560905D18E2318D90482
:1029F000835609052166D18E2318D90423800D0042
:102A00008656F3A6068001000100130680FA83466D
:102A1000390593F60602638A062083463905A18AA2
:102A2000EDFE97F0FF1FE78000672A8C97F0FF1FED
:102A3000E7806066E30C85FF835609051166425501
:102A4000D18E2318D90497000000E7806063834685
:102A5000390513063905A18AFDDAF336048093F6A9
:102A60008608B6D401000100930680FA23809D00F9
:102A70002380DD00010001008346060093F6F60D79
:102A80002300D60023800D00A656F3A60680010081
:102A900001008356090503462905D247B376DA00BB
:102AA0003306CA021305800C9355F6413696330D52
:102AB000F6408257333CD6002E9C3336A601330CA9
:102AC000FC40330CCC403308850392564E86B33518
:102AD000A5033305A503C29597B00100E780C04B5D
:102AE00063468001631E0C16630C0D161306150059
:102AF0003335A6002E959356F5013696B335D6009C
:102B0000AA959396F50105828585D18E6346B0001E
:102B1000639D051A638B061A0356C9021582330595
:102B2000D6003336C500B2956348B00063910524E2
:102B30001306F00F637DA622894663F356159307AB
:102B40008008F3B7078093F78708BED6010001001D
:102B500037170040930770052300F704930780FAA6
:102B60002300F704010001008356C702896781171B
:102B7000D58FC207C1832316F70223000704B65777
:102B8000F3A7078001000100FA506A54DA544A5949
:102B9000BA592A5A9A5A0A5BFA4B6A4CDA4C4A4D8D
:102BA000BA4D296182801308F5FF3335A800FD1561
:102BB0002E951356F5013298B336C800AA9695B9EA
:102BC000F336048093F68608B6CA0100010023801C
:102BD0009D002380AD000100010083463905CD8EA4
:102BE000A309D90423800D00D646F3A60680010070
:102BF000010035B3F336048093F68608B6CE0100A3
:102C0000010023809D002380CD0001000100834648
:102C1000390593E60602A309D90423800D00F64680
:102C2000F3A606800100010095B3F336048093F605
:102C30008608B6D20100010023809D002380CD00CC
:102C4000010001008346390593E60602A309D90471
:102C500023800D009656F3A606800100010045BBB7
:102C60009306F5FF33B5A600FD152E959355F50196
:102C7000AE96B3B5B600AA951396F501858269B5EF
:102C8000F336048093F68608B6D801000100930657
:102C900080FA23809D002380DD000100010083561F
:102CA000C9020566011693F6F60FD18EC206C182DF
:102CB0002316D90223800D00C656F3A60680010014
:102CC0000100850A93FAFA0F95B233E6B60045C2C1
:102CD0000356C9023305D0403338A000B305B040D5
:102CE000B385054115826345B000D1E16371A60843
:102CF000894663F0560593078008F3B7078093F77A
:102D00008708BEDA01000100B717004013077005FD
:102D10002380E704130780FA2380E7040100010001
:102D200003D7C7027D8B2396E70223800704D6577B
:102D300081BDF336048093F68608B6DC01000100FD
:102D4000930680FA23809D002380DD0001000100AE
:102D50008356C9020566011693F6F60FD18EC20698
:102D6000C1822316D90223800D00E656B9B7930716
:102D70008008F3B7078093F78708BEDE01000100E3
:102D800037170040930770052300F704930780FA74
:102D90002300F704010001000356C7029397560071
:102DA000B297C207C1832316F70223000704F65720
:102DB000C1BB914763EEB70217D70100130747095C
:102DC0008A05BA959C41BA978287B717004003A736
:102DD000470B1345F5FF698F23AAE70A03A7070BE3
:102DE000698F23A8E70A03A7070A798D23A0A70AFA
:102DF0008280B717004083A6470B1347F5FFF98E73
:102E000023AAD70A83A6070B558D23A8A70A83A652
:102E1000070A758F23A0E70A8280B717004003A72F
:102E2000470B498F23AAE70A03A7070B1345F5FFB2
:102E300045BFB717004083A6470B1347F5FF758FB3
:102E400023AAE70A03A7070A598D4DB7B717004011
:102E500003A7470B498FEDB7914763EEB70217D72A
:102E60000100130727008A05BA959C41BA9782870B
:102E7000B717004003A7470D1345F5FF698F23AA35
:102E8000E70C03A7070D698F23A8E70C03A7070C1E
:102E9000798D23A0A70C8280B717004083A6470D29
:102EA0001347F5FFF98E23AAD70C83A6070D558D7E
:102EB00023A8A70C83A6070C758F23A0E70C82809C
:102EC000B717004003A7470D498F23AAE70C03A7B4
:102ED000070D1345F5FF45BFB717004083A6470D03
:102EE0001347F5FF758F23AAE70C03A7070C598D2D
:102EF0004DB7B717004003A7470D498FEDB779715C
:102F000022D43714004026D24AD0035924028354D5
:102F1000040206D64209C2044ECE52CC56CA1359F8
:102F20000901C1802DE11379F9F793F4F49F420967
:102F3000C20413590901C18093078008F3B70780C1
:102F400093F787083EC40100010093077005230032
:102F5000F404930780FA2300F40401000100231114
:102F600024032310940223000404A247F3A707803C
:102F700001000100B250225492540259F249624AAF
:102F8000D24A45618280B7F5070081463000B1051D
:102F9000194597000020E7806081A2471397270119
:102FA000E34A07FC1369090893E404409309800885
:102FB000F3B7098093F787083EC001000100930A28
:102FC000700523005405130A80FA2300440501000C
:102FD00001002311240323109402230004048247D8
:102FE000F3A7078001000100294597F0FF1FE78044
:102FF0006034F3B9098093F989084EC201000100D9
:1030000023005405230044050100010083570402F6
:1030100093E707202310F402230004049247B9B772
:10302000B71700408847420541819377050491EB2B
:103030009377F5013755E801130505803345F5020F
:1030400082809377050C130700046397E70093775A
:10305000F50137459C1CCDB72165130505D082804D
:1030600037E700E01C435443A183E206D58F1CC11F
:10307000FD572320F7182322F718828013178500A5
:10308000B7E700E023A0E710618123A2A7108280A8
:10309000B7F700E08847CC47828081473737004048
:1030A000A14663C4C700328582800345B740E38EE2
:1030B000A6FE3385F5000345050085072304A740D8
:1030C000CDB7970700209387E7EE9C431737002082
:1030D0001307C7063E95636EE500173700201307F8
:1030E00067526368A700170700202325A7EC3E85D9
:1030F0008280FD57EDBF8280411122C406C62A841A
:1031000097000000E78000F22947B307E502B240CC
:103110008D83B3D7870222449507B3D7E7023737A9
:103120000040C207C1832316F7004101828041118C
:1031300037150E0006C697000000E78020FCB73761
:103140000040130770F82381E7000D47A381E700D3
:1031500013070004A380E70005472387E700B24078
:103160004101828037370040834727001A0593F7D3
:10317000F703C98F93F7F70F2301F7008280B73762
:10318000004003C7170019C9D98DA380B70003C732
:103190000700136787002380E700828093C5F5FF4F
:1031A000F98DA380B7008280AE872A87B7360040AA
:1031B00021463738004089E7170300006700E3F332
:1031C00083C8B600E30916FF05078348F7FFFD171C
:1031D000C20723041801C183F9BF411122C406C6E6
:1031E0002A8497000000E780E0E32947B307E5025F
:1031F000B2408D83B3D7870222449507B3D7E70245
:1032000037370040C207C1832316F740410182804F
:10321000716541111305052006C697000000E7807F
:1032200000FCB7370040130770F82381E7400D47D3
:10323000A381E74013070004A380E74005472387E5
:10324000E740B24041018280CC41411106C632853F
:1032500003C6150083C5050022064D8E42068D6506
:103260004186138875A2630C0611634BC80413884A
:1032700045A26300060D634AC800938535A2630129
:10328000B6082390060029464DA0138855A2630571
:10329000060D938565A2E316B6FE8D451D4663E6D1
:1032A000E5081146198E63F3C7003E86B7E70400B0
:1032B0002390C600FC4797D501009385E5BC9DA0EF
:1032C000138895A263030611634E060D1388A5A209
:1032D00063000613938505A5E315B6FA99451D46C7
:1032E00063E5E504198E63F3C7003E86B7E7040083
:1032F0002390C600FC47970500209385E5D51DA0C7
:103300009D451D4663E3E5022146198E63F3C70020
:103310003E86B7E70400FC472390C60097050020CF
:103320009385C533BA9582970146B24032854101F3
:103330008280AD451D46E3EAE5FE3146198E63F312
:10334000C7003E86B7E704002390C600FC4797D528
:1033500001009385E5B5F9B7B1451D46E3E7E5FC06
:103360003546198E63F3C7003E86B7E70400239005
:10337000C600FC4797D50100938585B465B78D4598
:103380001D46E3E4E5FA1146198E63F3C7003E8655
:10339000B7E704002390C600FC4797D5010093854A
:1033A00065AF49B78D451D46E3E1E5F81146198E35
:1033B00063F3C7003E86B7E704002390C600FC47CE
:1033C00097D50100938585B1B1BFA5451D46E3EEB4
:1033D000E5F42946198E63F3C7003E86B7E704007B
:1033E0002390C600FC4797D50100938565AB1DBFB0
:1033F000B5451D46E3EBE5F23946198E63F3C70088
:103400003E86B7E704002390C600FC4797D501002D
:10341000938585A601BFB7E7040003A307139706AA
:103420000020938666C24146A54517050020130576
:10343000A5B802832D455DE703C505000947631F55
:10344000E50803A84500411106C603471800328568
:103450000346080022074168518F930828FE63073E
:10346000170563E9E80005186303070323900600C6
:10347000294591A8130648FE630AC7041518E317E7
:1034800007FF15463E87637BF600154701A8130624
:1034900000023E876374F60013070002B7E70400DA
:1034A0002390E600FC471316070111A83E8691C33E
:1034B0000546B7E70400FC472390C6004206CC450A
:1034C000418282970145B240410182801306000883
:1034D0003E87E375F6FC13070008C9B72390060082
:1034E000054582808280416779176304E5044111B4
:1034F00022C406C685472A84639FF500B7E7040007
:1035000022852244B24003A38713970500209385A8
:10351000252F4101028389476399F500B7E704002D
:1035200083A7070B8545829771D9B2402244410198
:1035300082808280797122D452CC2E842A8A97D5B7
:1035400001009385A59B17D501001305A59D06D6FF
:103550003AC626D24AD0B68432894ECE97B0010000
:10356000E780C0EEA68517D501001305A59C97B08E
:103570000100E780A0ED294597B00100E780E0F168
:103580008347840093F70702E1E7834904008947F2
:10359000054532476396F908544083C7160083C631
:1035A0000600A207D58FC166138616FE638CC7027C
:1035B0008D16638FD7068D66938626902945639175
:1035C000D706B7E70400A285225403A34714B250DC
:1035D000F249A6864A86925402595285624A854724
:1035E000456102832D450DEF93070002354563E9E0
:1035F0009702B7E70400FC47484413060002CA8557
:103600008297814997070020938747209C43014573
:1036100081CB9C4391C74E852686CA8582970145FA
:10362000B250225492540259F249624A4561828052
:103630002D457DF79307700F3545E3E397FEB7E718
:103640000400FC4748441306700FCA8582975DBF8B
:103650002145F9B7411122C437E4040083278413BC
:1036600026C2AA84416506C69705002093854519A0
:103670007D1582978327C40A170500001305E5E628
:103680008588829795C0032304132244B240924454
:10369000970600209386C6AD4146C5451705002014
:1036A0001305059C41010283B24022449244014526
:1036B0004101828019C59707002023A9A71401455D
:1036C0008280454582801147636AA70A97D6010028
:1036D000938686810A0536951841411106C63697AC
:1036E000AE87B2850287130700026145639DE7003C
:1036F000B7E70400FC471306000217050020130576
:1037000065F682970145B2404101828005476145D7
:10371000E39BE7FEB7E70400FC47054617050020DA
:10372000130545F6F9BF1307700F6145E39DE7FCEC
:10373000B7E70400FC471306700F170500201305B8
:10374000A5F4C1B7130700086145E39EE7FAB7E7A0
:103750000400FC4713060008170500201305450266
:103760004DB715476145E390E7FAB7E70400FC471A
:103770001546170500201305E50861B70945828045
:10378000411126C2B7E4040083A7C41322C44AC06F
:1037900006C62E8497050020938585062A89829780
:1037A000058905C5970700209387878B83D7A70BCB
:1037B000A28503A3440D2310F4002244B240924496
:1037C0004A850249014641010283B24022449244A3
:1037D000024949454101828097070020238A070258
:1037E0009707002023A80702B717004003A7070C7C
:1037F000B706C0FFFD16758F23A0E70C03A7070DC2
:10380000B7064000558F23A8E70C03A7070C3D9B84
:1038100023A0E70C03A7070D1367070123A8E70CF4
:103820008280B717004003A5470C83A7470C598136
:1038300013451500C18B058999E31365250097078A
:10384000002083C7E7FC6380A7029707002023813D
:10385000A7FC11C9970700209387C7FB03A30700A4
:103860006303030002838280114517F3FFFF6700A3
:1038700043C8411193962500AA852D4506C697F0A9
:10388000FF1FE780A0F2B240014541018280011193
:1038900022CC06CE3714004026CA4AC84EC652C4AF
:1038A00083447405034AB405834984050349940598
:1038B00097F0FFFFE780C09E8347A40593F4F40FC1
:1038C000137AFA0F93E71700230DF40493F9F90F15
:1038D0001379F90FB717004003C7A705058B6DFFD4
:1038E00003D5C705A38D4705238C3705A38C270572
:1038F000A38B9704F2406244D2444249B249224A1F
:103900000561828041119397050122C406C626C233
:10391000C1872E8463DC0700B7E40400FC5482975F
:1039200019C1BC5482972165218D15A893F7150004
:1039300013C515008DE793F725009DC7970000007C
:10394000E78060EEB7E70400BC4F1306000A894524
:1039500017050020034585EC829713452400B240EB
:1039600022449244410182809397250163D8070243
:10397000B7E4040083A7C41E829797000000E78085
:10398000E0EEBC4C37560700130606308965170574
:1039900000200345A5E88297096579B7939715013B
:1039A0000145E3DE07FA17C501001305A56097B0CE
:1039B0000100E78080C1B7E70400BC4F1306006434
:1039C000916517050020034565E582971165A9BF3C
:1039D0002D71232A9110FD74E98C232C811023284A
:1039E0002111232631112A84AE89328993060010D1
:1039F0000A86A6852D45232E111097F0FF1FE7801C
:103A0000E0DA13154401B7E70400FC4751810A05C9
:103A100013962900CA850A958297A6858566014670
:103A2000254597F0FF1FE78060D80A86A685930694
:103A30000010294597F0FF1FE78040D78320C11170
:103A40000324811183244111032901118329C11009
:103A500015618280B7F7070003C70701411106C649
:103A600022C426C24AC0A547631DF7009700000084
:103A7000E78040F6B24022449244024901454101A8
:103A8000828013942500AA843289A286AA850146E1
:103A9000254597F0FF1FE78060D1A2864A86A6855C
:103AA000294597F0FF1FE78060D0E9B71D71A2CCD0
:103AB00037E404005C5C485886CE494697C501004F
:103AC0009385C54A829711E917C501001305454B37
:103AD00097B00100E78060AF01A0B7F600E079572A
:103AE00098CAFD57DCCA0567B7E700E023A0E710D6
:103AF0001306F00290C223A0E71801000100370767
:103B0000002018471306000481459706002023A5CE
:103B1000E6D04157A38AE7403C44080882979707BC
:103B200000209387676C3EC8856713870740231A78
:103B3000E1001D673ACC37070105130707103ACE9D
:103B4000938757D11307B00F2310E1022312F1021C
:103B5000054797F7FFFF9387E7532301E1023ED81C
:103B600017070000130727D197070000938767D234
:103B7000B7F50700BAC23EDC170700001307C7ED10
:103B800097070000938787CE81463000E1051945ED
:103B9000BAC43EDE97F0FF1FE78040C11808814796
:103BA000994630003E960346060085070507A30B9D
:103BB000C700E398D7FEC24791C703574101856705
:103BC0006373F70001A0B7E7040083A7470A08085A
:103BD0008297AA8511C917C501001305A53B97B0A7
:103BE0000100E780A08601A0F6406644256182803E
:103BF000411126C2B7E4040083A7040806C622C404
:103C000017050000130545D0829717040020130400
:103C1000E4C02300A40097000000E7808002970022
:103C20000000E780A0BB03450400224403A38405F1
:103C3000B2409244130600328965410102837971D2
:103C400006D622D413078008F337078093F7870836
:103C50003EC201000100B7170040930570052380A4
:103C6000B704130680FA2380C7040100010083C64D
:103C7000F70293F6A60FA387D70223800704924684
:103C8000F3A60680010001007337078013778708C9
:103C90003AC4010001002380B7042380C704010057
:103CA000010003C7F70213672700A387E7022380F9
:103CB0000704A247F3A7078001000100054597E02C
:103CC000FFFFE780206197000000E78020BA0147EE
:103CD00081468147054685451305407E97E0FFFFF5
:103CE000E780206437E404003C4468005146814585
:103CF0008297B707C0A83EC8B787E803938707D065
:103D00003ECA97E7FF1F9387876B3EC67C586800C3
:103D10008297B250225445618280411197D50100AB
:103D20009385858F17C501001305C51F06C697A08B
:103D30000100E780A07117D501001305A5A697A083
:103D40000100E780A070B2402945410117A301009E
:103D50006700A374411197D501009385258D17C580
:103D600001001305251C06C697A00100E780006E20
:103D700017D501001305C5A197A00100E780006DCC
:103D8000B2402945410117A30100670003714111A9
:103D900022C406C6834705002A849DC797D5010023
:103DA0009385858E17C501001305C51797A00100DF
:103DB000E780C0694C4017D501001305E5AC97A01A
:103DC0000100E780A0683DA058410DEF97D50100A4
:103DD0009385858B17C501001305C51497A00100B5
:103DE000E780C06617D50100130585AB97A00100D9
:103DF000E780C0652244B2402945410117A3010074
:103E00006700A369A1679386D7036313D70297D589
:103E100001009385658717C501001305A51097A0BC
:103E20000100E780A06217D50100130565A87DBFDA
:103E3000ED0797D501009385258517C5010013056A
:103E4000650E631BF70097A00100E780206017D57F
:103E50000100130525A759BF97A00100E780005F67
:103E60004C4017D501001305E5A791BF411197C537
:103E700001009385E57C17C501001305A50A06C658
:103E800097A00100E780805CB2402945410117A35B
:103E9000010067008360797122D426D24AD02E8433
:103EA0002A898145B2844800714606D697E0FFFF13
:103EB000E780A02297F7FF1F9387474CDC4783D703
:103EC0000700231421012313F10097500000E7801D
:103ED00020809547A305F1009307401F3EC6FD577C
:103EE0002305A100230AF10097500000E78080928B
:103EF0002686A285480097500000E7804080B25097
:103F000022549254025945618280971700202390D1
:103F1000077E971700202389076CB7E70400BC478A
:103F2000411106C641468145170500201305451A73
:103F3000829797200000E780605697200000E78076
:103F4000C031014597500000E78020251707002069
:103F50000347071A9307F00A6315F7029307F0F86F
:103F60008945170500201305A51817070020230110
:103F7000F71897070020A38D071697500000E780D9
:103F8000604C97500000E7802059814537050400B8
:103F90009707002023AC07129707002023960712EB
:103FA0009707002023830712970700202394070A0E
:103FB00097070020239207089707002023950710F2
:103FC00097070020239E071097300000E78000C568
:103FD000014597500000E780E04F97C501009385A9
:103FE000A56817C501001305E5F397A00100E78058
:103FF000E04517D501001305259597A00100E7803E
:10400000E044B2402945410117A301006700E3489D
:10401000411122C406C626C293F715002E84638F71
:104020000710814617F6FF1F1306863285451705D0
:1040300000200355250097C00000E780E0B215C9B5
:1040400097C501009385056317C50100130585ED2C
:1040500097A00100E780803F17C5010013054504C4
:1040600097A00100E780803E294597A00100E780E6
:10407000C04297C501009385E55F17C50100130590
:1040800065EA97A00100E780603C17C501001305B1
:10409000650297A00100E780603B294597A00100D9
:1040A000E780A03F17F5FF1F1305452D5C45054729
:1040B0002390E70097300100E780606397C5010017
:1040C0009385455B17C501001305C5E597A0010061
:1040D000E780C03717C50100130505FF97A0010051
:1040E000E780C036294597A00100E780003B930791
:1040F00010F817070020230DF7FE9707002083D73D
:1041000027F317070020A305F7FE17050020130566
:1041100025FEA183914517070020230CF7FC970784
:104120000020A38807FC97500000E780A0311345CA
:104130001400B240224492444101828093F725004A
:10414000E1C317070020035727F845CB9706002047
:104150009386C6F7944297D701009387E7801706A6
:104160000020034686F6814517050020130545F615
:1041700097700000E780A0BEAA8441C197C50100E6
:104180009385055617C501001305C5D997A00100F1
:10419000E780C02BA68517C50100130565F497A01D
:1041A0000100E780A02A294597A00100E780E02EC2
:1041B00097070020239A07F0930710F817070020AD
:1041C0002308F7F29707002083D787E61707002018
:1041D000A300F7F2A18317070020230CF7F0914505
:1041E0008D47170500201305A5F017070020A3022F
:1041F000F7F097500000E780E0241345240015BF36
:1042000093F74500D1C397C501009385654D17C548
:104210000100130525D197A00100E780202317C5D1
:1042200001001305A5ED97A00100E7802022294594
:1042300097A00100E7806026930720F81707002069
:104240002308F7EA9707002083D7C7E01707002065
:10425000A300F7EAA18317070020230CF7E885479E
:1042600017070020A307F7E897400000E780805A6F
:10427000170500201305C5E7914597500000E7801A
:10428000601C1345440075B593F78500A9C797C511
:1042900001009385E54417C501001305A5C897A043
:1042A0000100E780A01A17C50100130565E697A075
:1042B0000100E780A019294597A00100E780E01DD3
:1042C00097070020239207E097700000E78000B96D
:1042D00013458400B9BD93F70501D1C38545170582
:1042E0000020035525D797500100E780206B97C524
:1042F00001009385E53E17C501001305A5C297A0EF
:104300000100E780A01417C501001305A5E197A0DF
:104310000100E780A013294597A00100E780E0177E
:10432000930730F8170700202304F7DC97070020D5
:1043300083D747D217070020A30CF7DA1705002010
:10434000130505DBA1838D45170700202303F7DA4A
:1043500097500000E780000F13450401D9BB93F785
:104360000502D1C797C501009385853717C50100A0
:10437000130545BB97A00100E780400D17C501005C
:10438000130585DC97A00100E780400C294597A024
:104390000100E7808010930740F8170700202309E9
:1043A000F7D49707002083D727C917070020A30158
:1043B000F7D4A18317070020230DF7D285471707ED
:1043C0000020A308F7D297070020239707C697403D
:1043D0000000E780204417050020130565D19145B2
:1043E00097500000E78000061345040299B393F745
:1043F0000504FDC397C501009385852E17C50100EF
:10440000130545B297A00100E780400417C50100DD
:10441000130505D597A00100E7804003294597A023
:104420000100E78080079707002083C767CC130748
:10443000700A6386E7061307800A638CE708130790
:10444000600A6393E704930760F8170700202301CD
:10445000F7CA9707002083D707C717070020A309CB
:10446000F7C8A183170700202305F7C8854717075A
:104470000020A304F7C8B14517050020130545C760
:1044800097500000E78000FC97400000E7808038EC
:104490001345040497070020239707C259B99307CF
:1044A00070F8170700202305F7C49707002083D76B
:1044B00087C117070020A30DF7C2A18317070020AB
:1044C0002309F7C2854717070020A305F7C29945BE
:1044D00065B7930780F8F1B793F705080145E38ABC
:1044E00007C497C501009385A51F17C501001305D3
:1044F00065A397A00100E78060F517C501001305CB
:10450000A5C797A00100E78060F4294597A00100A6
:10451000E780A0F89307A0F817070020230AF7BC4C
:104520009707002083D7C7BB17070020A302F7BC5B
:10453000A18317070020230EF7BA8547170700202D
:10454000A309F7BA97070020239C07B897400000FB
:10455000E780402C17050020130585B99145975039
:104560000000E78020EE13450408E1B6411122C4A3
:1045700097C50100938585122A8417C5010013058C
:10458000659A06C697A00100E78040EC4C4017C52D
:1045900001001305E52C97A00100E78020EB2945D9
:1045A00097A00100E78060EF034704009307F00F36
:1045B000631FF70297C501009385450E17C50100DB
:1045C0001305459697A00100E78040E84C4017C5C9
:1045D00001001305E52997A00100E78020E72244A8
:1045E000B2402945410117A30100670003EBB24027
:1045F000224441018280B1C1411122C417C501008A
:10460000130545922E8497C501009385250406C69F
:1046100097A00100E78080E3A28517C5010013057C
:10462000653097A00100E78060E22244B24029454E
:10463000410117A30100670043E68280411122C4B3
:1046400026C22E84AA8497C501009385E50017C56C
:1046500001001305258D06C697A00100E78000DF45
:1046600017C501001305C52C97A00100E78000DEE7
:10467000294597A00100E78040E297C50100938596
:10468000A5FD970700202397979A17C501001305EA
:104690006589854497070020239C87989707002009
:1046A00023999798971700202393870497A00100D8
:1046B000E780C0D99715002083D5650317C5010091
:1046C0001305852797A00100E78040D8294597A0CA
:1046D0000100E78080DC97170020238797F0972060
:1046E0000000E78080B7228597500000E780E0AAAD
:1046F000054597500000E780E0DD97F7FF1F93879F
:10470000E7C7DC4703D70700C167FD176312F7024D
:104710002244B7E70400B240924403A3870517F58B
:10472000FF1F034525101306000A8545410102833A
:10473000B2402244924441018280011122CC37E4EC
:1047400004005C5C06CE354697C501009385C5061E
:1047500017D501001305C5C0829711E917C50100DF
:104760001305058297A00100E78020E601A097F7D6
:10477000FF1F9387E70B3EC4B7F507008567938754
:104780000780814617F6FF1F1306060AE105194543
:104790003EC697E0FF1FE78060017C44194697F50D
:1047A000FF1F93856508170500201305E58A82978A
:1047B000340017F6FF1F1306260797C501009385DF
:1047C000A55117C501001305A55297600000E780A9
:1047D000002E2A841DCD97C50100938565EF17B57E
:1047E00001001305257497A00100E78020C6A2856B
:1047F00017C50100130545FD97A00100E78000C51E
:10480000294597A00100E78040C9F2406244056154
:10481000828097E00000E780609017C501001305D3
:10482000A5F197500000E780402297A00000E780A4
:10483000A0E497500100E780204917F5FF1F1305FA
:1048400065B097500100E780C03117C5010013051E
:10485000A5EF97500100E780A0492A8497600000E7
:10486000E780808897000100E780002197800100A1
:10487000E78020BA97700000E780C0E097600000F2
:10488000E78080FE97300100E78060E297C5010075
:10489000938505E417B501001305C56819C897A0ED
:1048A0000100E780A0BAA28517C50100130505F431
:1048B000A1B797A00100E78060B917C501001305F3
:1048C00025F597A00100E78060B8294597A0010071
:1048D000E780A0BC97300100E78040BE97F0000061
:1048E000E78000DD55C985453705040097200000A5
:1048F000E780C03297C50100938585DD17B50100BB
:104900001305456297A00100E78040B417C5010078
:10491000130585F197A00100E78040B3294597A0D2
:104920000100E78080B797F7FF1F9387E79483D74D
:10493000070017170020231CF7DA854717170020F8
:104940002304F7CA97200000E780C0AF972000003B
:10495000E780A09017150020035565D997500000F7
:10496000E780A083054597500000E780A0B697C573
:1049700001009385E5D517B501001305A55A97A049
:104980000100E780A0AC17C50100130525EC97A036
:104990000100E780A0ABADB597C50100938545D375
:1049A00017B501001305055897A00100E78000AA7C
:1049B00017C50100130545F997A00100E78000A97C
:1049C000294597A00100E78040AD014569BF41112D
:1049D00022C437E404008327041A06C6829797404E
:1049E0000000E780407F8327040817F5FFFF1305C9
:1049F0006562829797F7FF1F2386A7E217F5FF1FCF
:104A00001305C59797400000E78060132244B24029
:104A1000410117030000670083D2B7E70400FC4799
:104A20001171A2DDCAD986DFA6DBCED72E843289EA
:104A30002E86AA8517F5FF1F1305856B829717F73A
:104A4000FF1F1307E76A83470700930680029387D7
:104A5000E70793F7F70FE3ECF610BA898A0717B761
:104A6000010013076755BA979C43BA9782878D4711
:104A700097C50100938505C817B501001305854A40
:104A8000630FF40097A00100E780409C17C5010068
:104A90001305058597A00100E780409BBDA497A062
:104AA0000100E780A09A17C501001305E58497A0CF
:104AB0000100E780A099294597A00100E780E09DCB
:104AC000930720F8114697F5FF1F938565624A8585
:104AD00017F7FF1F230EF76097F7FF1FA38B0760E1
:104AE00097F0FFFFE780603B2A841DC997C501004E
:104AF000938545C017B501001305C54297A0010075
:104B0000E780C094A28517C501001305A58297A070
:104B10000100E780A093294597A00100E780E09776
:104B200097C50100938505BD17B501001305853FA5
:104B300097A00100E780809117C501001305C5808B
:104B400097A00100E7808090294597A00100E780A9
:104B5000C0944165930730FA054697F5FF1F93858A
:104B600025597D1517F7FF1F2304F75897F0FFFF0E
:104B7000E780A0322A841DC997C50100938585B7B7
:104B800017B501001305053A97A00100E780008CD6
:104B9000A28517B501001305E57997A00100E7800C
:104BA000E08A294597A00100E780208FB7E704003D
:104BB000BC4F0566130606C8A14517F5FF1F034540
:104BC00065C68297FE506E54DE544E59BE5911612F
:104BD000828091476303F40297C50100938585B1F4
:104BE00017B501001305053497A00100E780008682
:104BF00017B501001305857871BDB7E70400FC4FB8
:104C0000914517F5FF1F0345E5C1829797C5010040
:104C1000938545AE17B501001305C53097A0010077
:104C2000E780C08217B501001305057797A0010042
:104C3000E780C081294597A00100E7800086974062
:104C40000000E78020BD914535A485476303F40249
:104C500097C50100938505AA17B501001305852C9A
:104C600097900100E780807E17B501001305457419
:104C700015B597F7FF1F239F273DB7E7040005668B
:104C8000BC4F130606C8C1450DBF8D476303F40230
:104C900097C50100938505A617B501001305852862
:104CA00097900100E780807A17B50100130505721F
:104CB000D5B3930740F8114697F5FF1F93854543F9
:104CC0004A8517F7FF1F2305F74297F7FF1FA382B7
:104CD000074297F0FFFFE780401C2A84E30405EEBB
:104CE00097C50100938505A117B50100130585231C
:104CF00097900100E7808075A28517B50100130524
:104D0000656397900100E7806074294597900100E2
:104D1000E780A07845BD9147E31CF4F6B7E70400AF
:104D2000FC4F9305000217F5FF1F0345A5AF8297BF
:104D300097C501009385059C17B501001305851ED5
:104D400097900100E780807017B501001305856911
:104D5000F1BD894763E3870297C501009385859973
:104D600017B501001305051C97900100E780006E40
:104D700017B501001305456831BB97F4FF1F83C4C5
:104D8000443797F7FF1F83C7B73697C50100938550
:104D90006596A20417B501001305C518DD8C979020
:104DA0000100E780A06AA28517B50100130505661A
:104DB00097900100E7808069C2042945979001001F
:104DC000E780A06DC1849305D4FF93960401C1824E
:104DD0004A8693F5F50F17F5FF1F130595319720B8
:104DE0000000E78060E7E35F90DC930750F817F777
:104DF000FF1F230FF72E83C73900228697F5FF1F69
:104E00009385052F85074A8517F7FF1FA303F72E04
:104E100097F0FFFFE78060082A84E30505DA97C56D
:104E200001009385258D17B501001305A50F9790F7
:104E30000100E780A061A28517C50100130585ADBB
:104E4000C9B5894763E3870297C501009385858AC1
:104E500017B501001305050D97900100E780005F6D
:104E600017B501001305455C35B197400000E78098
:104E7000609AA28517F5FF1F13058527974000004C
:104E8000E780405C81B38D476303F40297C501005E
:104E90009385458617B501001305C5089790010055
:104EA000E780C05A17B501001305C559E5B6B766C6
:104EB00002000146B7750200054597E0FF1FE78035
:104EC000E08E930760F817F7FF1F2303F72297F789
:104ED000FF1FA38007229307000617F7FF1F230B6E
:104EE000F720894717F7FF1FA306F72097F7FF1F43
:104EF0002383072097F7FF1FA38F071EC14717F7CC
:104F0000FF1F230BF71E930720F917F7FF1FA305B9
:104F1000F71E314697F7FF1FA381A71E97F5FF1FC6
:104F20009385051D4A8597F7FF1F2388071C97F077
:104F3000FFFFE78080F62A84E30605C897B50100E5
:104F40009385457B17B501001305C5FD97900100BA
:104F5000E780C04FA28517B501001305255055B352
:104F6000B1476303F40297B501009385A57817B59F
:104F70000100130525FB97900100E780204D17B530
:104F800001001305654F39B6B7E70400FC4F9305E0
:104F9000000417F5FF1F0345E5888297974000003E
:104FA000E7804087B145F9B5914763E3870297B53C
:104FB00001009385257417B501001305A5F6979098
:104FC0000100E780A04817B501001305A54CD9B42E
:104FD00097F4FF1F83C4041297F7FF1F83C777114D
:104FE000A204DD8C8E04B77702006D14BE94228675
:104FF000A68517B501001305254B97900100E780A2
:10500000E044B7E70400FC47228697F5FF1F93852D
:10501000750E2800829793160401C1823000A68580
:10502000094597D0FF1FE78060782A8409C917B522
:1050300001001305254997900100E7800059930767
:1050400070F8194697F5FF1F9385850A4A8517F76B
:10505000FF1F230FF70897F7FF1FA38D870897F00F
:10506000FFFFE78080E32A84E30E05B497B50100D3
:105070009385456817B501001305C5EA97900100AF
:10508000E780C03CA28517B501001305A54495B97A
:105090009947630BF41297B501009385A56517B581
:1050A0000100130525E897900100E780203A17B525
:1050B00001001305A543F9BA914763E3870297B549
:1050C00001009385256317B501001305A5E59790A9
:1050D0000100E780A03717B501001305A5425DBAAE
:1050E00097F4FF1F83C4040197F7FF1F83C777005E
:1050F000A204DD8C8E04B77702006D14BE94228664
:10510000A68517B501001305254197900100E7809A
:10511000E033B7E70400FC47228697F5FF1F93852D
:1051200075FD2800829793160401C1823000A68580
:105130000D4597D0FF1FE78060672A8409C917B51E
:1051400001001305253F97900100E7800048930771
:1051500080F8194697F5FF1F938585F94A8517F75B
:10516000FF1F2307F7F897F7FF1FA38587F897F02E
:10517000FFFFE78080D22A84E30605A497B50100EB
:105180009385455717B501001305C5D997900100C0
:10519000E780C02BA28517B501001305E53A95B647
:1051A00099476303F40297B501009385A55417B599
:1051B0000100130525D797900100E780202917B536
:1051C00001001305E539F9B0B7E70400FC4F93057A
:1051D000000417E5FF1F0345E56482979730000040
:1051E000E7804063994579B18D476303F40297B531
:1051F00001009385255017B501001305A5D297909E
:105200000100E780A02417B501001305E53659B069
:1052100017B501001305453797900100E780E03A84
:105220001305C01297D0FF1FE780A011014597E03A
:10523000FFFFE78020E30D4597100000E780009F07
:10524000294597D0FF1FE780C00F97D0FF1FE78049
:1052500020008DBA99476303F40297B50100938546
:10526000654917B501001305E5CB97900100E7806C
:10527000E01D17B501001305E53129B817F7FF1F29
:10528000034757E797F7FF1F83C7C7E622075D8FDE
:105290009166BA96C2061166C1821306F6EF8D4773
:1052A0006365D60297E7FF1F9387470D9C4B17F660
:1052B000FF1F034616E49386C7002DC203D60700DE
:1052C00069CA8907E39CD7FE89471307A0F81146EE
:1052D00097F5FF1F9385C5E14A8597F6FF1F238940
:1052E000E6E017F7FF1FA306F7E097F0FFFFE78060
:1052F000C0BA2A84E308058C97B501009385853FE1
:1053000017B50100130505C297900100E78000144E
:10531000A28517B5010013052529E5B203D60700BC
:10532000630EE60A8907E39BF6FE8D4779BF914736
:105330006304F40297B501009385C53B17B50100DE
:10534000130545BE97900100E780401017B5010096
:10535000130505276FF00FF4B7E70400FC4F930522
:10536000000817E5FF1F0345E54B8297C9B897B5BD
:1053700001009385253817B501001305A5BA97904C
:105380000100E780A00C17B501001305E5246FF0BC
:105390006FF02390E70017E5FF1F130525FE972008
:1053A0000100E780203797B501009385A53417B534
:1053B0000100130525B797900100E780200917B574
:1053C00001001305652297900100E7802008294518
:1053D00097900100E780600C8147C5BD23900700CE
:1053E00017E5FF1F130585F997200100E78080323C
:1053F00097B501009385053017B50100130585B2F7
:1054000097900100E780800417B501001305451F40
:105410005DBF411122C406C6834705002A849DC78B
:1054200097B501009385C52817B50100130585AF11
:1054300097900100E78080014C4017B501001305EB
:10544000A55397900100E7806000E1A05841B7079D
:10545000CF009387777D631DF70697B5010093858D
:10546000252517B501001305E5AB97900100E780EE
:10547000E0FD1C448356E4008355C40003C60700C6
:1054800017B501001305C55097900100E78000FC97
:10549000294597900100E78040000357E4009707F3
:1054A000002083D7C7246309F7008355C40008444C
:1054B00097E0FFFFE78080CF0356E4008355C400E8
:1054C00008442244B240410117F3FFFF670023550F
:1054D000B707CC009387777D6315F70497B5010074
:1054E0009385051D17B501001305C5A3979001000D
:1054F000E780C0F51C448356E4008355C40003C60E
:10550000070017B501001305A54897900100E78033
:10551000E0F32244B240294541011793010067009E
:10552000C3F7B707CE009387777D6304F70297B57B
:1055300001009385E51717B501001305A59E979007
:105540000100E780A0F04C4017B501001305853934
:10555000CDBDB240224441018280B7E70400FC4740
:1055600041112E8606C622C426C24AC02E842A892C
:10557000AA8517F5FF1F1305A5B7829797B50100F8
:105580009385051917B501001305C599979001007A
:10559000E780C0EB97F5FF1F83C585B517B5010000
:1055A000130505BF97900100E78040EA29459790D1
:1055B0000100E78080EE97F4FF1F938464B383C7F4
:1055C000040041479387070693F7F70F636AF75C78
:1055D00017B70100130787A88A07BA979C43BA97A1
:1055E00082879D476307F40297B5010093854512B2
:1055F00017B501001305059397900100E78000E5BA
:1056000017B50100130545B997900100E78000E444
:10561000ADAC97F7FF1F83C7B7ADDDCB17F7FF1F03
:10562000034737AD97F7FF1F83C7A7AC22075D8FEE
:1056300097F7FF1F83C707ACC2075D8F97F7FF1F60
:1056400083C757ABE207D98F17F7FF1F2320F7A8AF
:1056500083C7640097B501009385850B17B50100DA
:105660001305458C17F7FF1F2301F7A6979001003C
:10567000E780C0DD97F7FF1F938747A58C4317F698
:10568000FF1F034686A417B501001305A5B2979026
:105690000100E780A0DB294597900100E780E0DF6B
:1056A00097F7FF1FA38607A42244B2409244024901
:1056B000930700F817F7FF1F230CF7A29D4517F576
:1056C000FF1F1305E5A2410117430000670083D7C0
:1056D00097600000E780008897F7FF1F238BA7A043
:1056E0009357850017F7FF1FA305F7A093570501F0
:1056F0002A8417F7FF1F230FF79E93578501014553
:1057000017F7FF1FA308F79E97600000E78040850A
:1057100097F7FF1F2381A79E97B50100938545FF4B
:1057200017B501001305058097900100E78000D2AE
:1057300017F6FF1F0346269CA28517B50100130527
:10574000E5A8B1B7CD476303F40297B5010093858F
:1057500025FC17A501001305E57C97900100E78063
:10576000E0CE17B501001305E5A779BD37E40400C5
:105770007C44414697F5FF1F9385959717F5FF1FCA
:1057800013050595829717F5FF1F1305659497106C
:105790000000E78040C497100000E78000AC97F756
:1057A000FF1F83C7079617F7FF1F03477795A207C9
:1057B00003238405D98F17F7FF1F2317F7901306CC
:1057C000000A89452244B2409244024917E5FF1F6E
:1057D00003454505410102838D476303F40297B5F4
:1057E00001009385E5F217A501001305A5739790B5
:1057F0000100E780A0C517B50100130565AE29B506
:1058000017F4FF1F0344E48E97F7FF1F83C7578EDB
:1058100097B501009385C5EF220417A50100130574
:1058200065705D8C97900100E78040C2A28517B536
:1058300001001305A59C97900100E78020C1294530
:1058400097900100E78060C50D4697F5FF1F93858F
:10585000258A228597E0FFFFE7802064AA8421C182
:1058600097B501009385C5EA17A501001305856B5F
:1058700097900100E78080BDA68517B5010013054C
:10588000259997900100E78060BC2244B240924481
:1058900002492945410117930100670003C097E7BA
:1058A000FF1F2399877AB7E70400116603A38705D2
:1058B000130606E8914539B78D476303F40297B59F
:1058C00001009385E5E417A501001305A5659790F0
:1058D0000100E780A0B717B50100130525AF2DB370
:1058E00017F4FF1F0344E48097F7FF1F83C7578017
:1058F00097B501009385C5E1220417A501001305A2
:1059000065625D8C97900100E78040B4A28517B571
:1059100001001305259197900100E78020B32945E8
:1059200097900100E78060B70D4697E5FF1F9385CC
:10593000257C228597E0FFFFE7802056AA841DC1C1
:1059400097B501009385C5DC17A501001305855D9A
:1059500097900100E78080AFA68517B50100130579
:10596000A58D05B797E7FF1F2398876CB7E704005D
:10597000116603A38705130606E89305000299B58F
:10598000894763E3870297B50100938565D817A51A
:1059900001001305255997900100E78020AB17B54A
:1059A0000100130565A58DB197E4FF1F83C46474DE
:1059B00097E7FF1F83C7D77397B50100938545D538
:1059C000A20417A501001305E555DD8C9790010091
:1059D000E780C0A7A68517B50100130565879790D6
:1059E0000100E780A0A6294597900100E780E0AA82
:1059F000228697E5FF1F9385A56F268597E0FFFF19
:105A0000E780A0492A84630E051A97B501009385A3
:105A100025D017A501001305E55097900100E780F8
:105A2000E0A2A28517B501001305C58399BD85477E
:105A300063F98718834519002244B2409244024911
:105A4000B335B00097E7FF1F2380B76217B5010099
:105A5000130585824101179301006700239FA285EA
:105A60002244B24092444A85024941011703000092
:105A70006700032299476303F40297B501009385F9
:105A800025C917A501001305E54997900100E78096
:105A9000E09B17B501001305E5AFBDB617E4FF1F86
:105AA0000344246597E7FF1F83C7976497B50100F8
:105AB000938505C6220417A501001305A5465D8C34
:105AC00097900100E7808098A28517A50100130533
:105AD000257C97900100E780609729459790010009
:105AE000E780A09B194697E5FF1F93856560228597
:105AF00097E0FFFFE780603AAA841DC197B50100D7
:105B0000938505C117A501001305C54197900100B4
:105B1000E780C093A68517A501001305657895B3A6
:105B200097E7FF1F239E875AB7E70400116603A378
:105B30008705130606E89305000869B1854797B500
:105B400001009385E5BC17A501001305A53D630B76
:105B5000F40097900100E780608F17A501001305FE
:105B600065755DB497900100E780408E17A5010030
:105B70001305C57597900100E780408D29459790E2
:105B80000100E78080912244B2409244024997E7A5
:105B9000FF1F239B07524101175300006700032C8E
:105BA00097B501009385C5B617A501001305853784
:105BB00097900100E780808917B501001305C5A102
:105BC000A1B4B24022449244024941018280411171
:105BD00006C622C497E0FFFFE780202C9377F50FDD
:105BE000A1C32A8497B50100938505B417A50100C8
:105BF0001305453397900100E78040859375F40FB6
:105C000017B50100130505D197900100E7800084C6
:105C10002244B24029454101179301006700E38700
:105C2000B240224441018280411122C491462A841B
:105C300017E6FF1F1306065A9D652D4506C697D029
:105C4000FF1FE780A0B6B7F7070003C70701A54706
:105C50006313F70001A09306001001469D652545DA
:105C600097D0FF1FE78080B497E7FF1F23848756F4
:105C70002244B240914617E6FF1F1306A6559D65C4
:105C80002945410117D3FF1F670043B25171CAD1A3
:105C900037E904008327C904A2D52E8686D7A6D368
:105CA0002E84AA8517E5FF1F13058544829797E781
:105CB000FF1F83C7E7431307700A6387E710636C0E
:105CC000F7001307600A6384E704BE502E549E5405
:105CD0000E596D6182801307800A6388E7161307E7
:105CE000900AE394E7FE8D476309F41C97B5010021
:105CF000938585D517A501001305C522978001005E
:105D0000E780C07417B50100130545D125A08D4764
:105D1000630CF40297B50100938505D317A5010024
:105D20001305452097800100E780407217B50100F8
:105D3000130505C897800100E780407129459780C9
:105D40000100E780807551B7854717B5010013053D
:105D5000E5C717E7FF1F2309F73097900100E78099
:105D6000C086B7750200B76602000146054597D0A8
:105D7000FF1FE780A0A3930760F817E7FF1F230921
:105D8000F73697E7FF1FA38607369307002617E726
:105D9000FF1F2321F736E5779387072117E7FF1FBA
:105DA000231CF734B14597E7FF1F2388073497E793
:105DB000FF1FA384A73417E5FF1F13056533973032
:105DC0000000E780206811B7914763E3870297B529
:105DD0000100938565C717A501001305A5149780D9
:105DE0000100E780A06617B50100130525C099B72B
:105DF00097E4FF1F83C4043097E7FF1F83C7772F03
:105E0000A204DD8C8327C9046D14228697E5FF1F49
:105E10009385552E280082978E0493160401B7753A
:105E20000200C1823000A695094597D0FF1FE78088
:105E3000E097930770F817E7FF1F230BF72A9945A0
:105E400097E7FF1FA388A72ABDB7914763E387029F
:105E500097B50100938545BF17A501001305850C73
:105E600097800100E780805E17B50100130585B9B2
:105E7000D1B597E4FF1F83C4E42797E7FF1F83C7CB
:105E80005727A204DD8C8327C9046D14228697E569
:105E9000FF1F93853526280082978E0493160401F0
:105EA000B7750200C1823000A6950D4597D0FF1F3F
:105EB000E780C08F930780F8BDBF17B501001305B9
:105EC00025B797800100E78040701305C01297C086
:105ED000FF1FE7800047014597D0FFFFE78080184C
:105EE0000D4597000000E78060D4294597C0FF1F4B
:105EF000E780204597C0FF1FE7808035F9B3411147
:105F00004AC097F6FF1F83D6867E328917D6FF1FB9
:105F10000356E64822C426C206C62A84AE849700E9
:105F20000000E780805F35C12DC0994763FF97046B
:105F30008347140003470400A207D98F13978700F3
:105F4000A183D98FC2073167C1831307C755639EE9
:105F5000E70297D7FF1F83D78744A301F400A183EB
:105F60002302F40097F7FF1F83D7677891C7A30236
:105F7000F400A1832303F400A68517B501001305DF
:105F8000A5B097800100E780604C97F7FF1F83C79B
:105F9000A765B9CF97D5FF1F83D5654017B5010019
:105FA000130545B097800100E780404A2686A28508
:105FB00017D5FF1F0355A53E97000000E78060C17D
:105FC0006301090497E7FF1F83C7C7219DCB95C8CD
:105FD00097E7FF1F83C747098DE722852244B24018
:105FE0000249A685924441011733000067008345AA
:105FF00017B50100130505AC97800100E780E05C50
:10600000C1B7B24022449244024941018280834791
:1060100055008345450017B501001305A5A5A20746
:10602000DD8D178301006700634217B5010013057A
:1060300065A317830100670043598D4763FBB70AC7
:10604000011126CA06CE22CC0344350097E4FF1F77
:1060500083C4541997B50100938585A6B337800092
:1060600017E7FF1FA300F71809C497B50100938530
:10607000E5A517B501001305E5A597800100E780A8
:10608000E03C97E7FF1F83C7F715638697009700EB
:106090000000E780402697E7FF1F83C7B7148DC72E
:1060A00085472306F100B7E7040083A74717700070
:1060B000854513055030829717B50100130585A259
:1060C00097800100E78060509967938757EE231609
:1060D000F100680085479145A30781002307F1007F
:1060E00097300000E7800036F2406244D2440561F8
:1060F00082808280894763F7B708011122CC06CEDF
:1061000026CA8344250085472A84639DF404914769
:1061100063F5B704034545008347340022055D8DD0
:1061200097D7FF1F239DA72697000000E780C04751
:106130009967938767EE2314F100834734002305A2
:106140009100A305F10083474400954528002306EC
:10615000F10097300000E780E02EF2406244D24424
:1061600005618280FDF89967938767EE2314F1003B
:1061700097D7FF1F83D7A722A305F10023050100AE
:10618000A183E1B782800111996722CCD51717F45A
:10619000FF1F130464452314F1008347040026CA3B
:1061A00097F4FF1F9384A4542305F10083D70400C0
:1061B00028009545A305F100A18306CE2306F10032
:1061C00097300000E780002803D6040083450400D0
:1061D00017B501001305859297800100E78000271D
:1061E000F2406244D244056182809D677971D9177B
:1061F0002316F10097F7FF1F83C7073F06D6230733
:10620000F100A9C3B7E70400FC47414697E5FF1F2B
:10621000938505EC1305F10082976800CD45973012
:106220000000E780202297F5FF1F83C5E53B17B5E7
:1062300001001305A58F97800100E7802021B2504F
:1062400045618280B7E70400BC474146814513059C
:10625000F1008297D9B7B76702045D71938757AA97
:106260003EC085672312F10097F7FF1F9387C7375A
:1062700083C70700A2C4A30301002303F10097F71B
:10628000FF1F9387C74683D7070037E4040086C6FD
:106290002314F10097D7FF1F9387671083D7070058
:1062A000414668002315F1007C4497E5FF1F938564
:1062B00025E28297F1450A8597000000E780E021FA
:1062C000231EA1007C448A850810794682973C44AD
:1062D0001305E103094681458297101093050002DA
:1062E000014597D0FFFFE780403EB64026446161FC
:1062F0008280B7C7A55A01119387C7333EC497E779
:10630000FF1F83C737EE3EC6B7F7070003C7070175
:1063100006CE22CCA5476313F70001A011649305B4
:1063200004F0930600100146254597C0FF1FE78043
:10633000E0473000930504F0A146294597C0FF1FB0
:10634000E780C04697E5FF1F83C5D5E917B5010073
:106350001305858E97800100E780400FF24062446C
:106360000561828001119165A1463000938505F099
:106370002D4506CE97C0FF1FE78040432247B7C791
:10638000A55A9387C7336314F702B24517A50100D6
:106390001305C57DB335B00097E7FF1FA384B7E4AD
:1063A00097800100E780800AF24005618280814584
:1063B00017A501001305C57D97E7FF1FA38407E21A
:1063C00097800100E780800897000000E780A0F236
:1063D000E1BFB7C7A55A79719387F7353EC6B7E7CE
:1063E0000400FC47AA8506D622D4414608088297B5
:1063F000B7F7070003C70701A5476313F70001A01C
:106400001164930504E8930600100146254597C0E2
:10641000FF1FE780A0397000930504E8D1462945A5
:1064200097C0FF1FE780803817B5010013058584EA
:1064300097800100E7806019B25022544561828044
:1064400079719165D1467000938505E82D4506D692
:1064500097C0FF1FE78080353247B7C7A55A93879B
:10646000F73517A501001305A57A6310F702B7E702
:106470000400FC4717E5FF1F130585C541460C08BE
:10648000829717A501001305A57697800100E78084
:10649000C013B25045618280B7F7070003C70701F8
:1064A000A5476313F70001A0916541119306001001
:1064B0000146938505E8254506C697C0FF1FE7807E
:1064C000E02EB24017A5010013058568410117832E
:1064D00001006700830FC16769768146FD170506D5
:1064E0001397060141836364B7003E8582803307BA
:1064F000D50003470700B98F214713F8170085839C
:1065000063050800B18FC207C1837D171377F70FAA
:106510006DF78506F1B741C5A547054763F2B70892
:1065200083471500034705003168A207D98F1397E9
:106530008700A183D98FC207C1831308C8550547B7
:1065400063900707411106C622C426C203442500F2
:10655000914763F087049307540063ECF502A301AD
:10656000C50021822302C5009304340091C6A30212
:10657000D500A1822303D5002A84A68597000000B8
:10658000E780A0F526942300A4002181A300A400A5
:106590000147B240224492443A8541018280054736
:1065A0003A858280B7C7A55A01119387E7343EC464
:1065B0002AC6B7F7070003C7070106CE22CC26CAB2
:1065C000A5476313F70001A091642A84938504EE24
:1065D000930600100146254597C0FF1FE780001D68
:1065E0003000A146938504EE294597C0FF1FE78040
:1065F000E01BA28517A50100130505669780010021
:10660000E780C0E497000000E78020C5F2406244C4
:10661000D2440561828001119165A14630009385C5
:1066200005EE2D4506CE97C0FF1FE78020182247B4
:10663000B7C7A55A9387E7346318F702B24517A581
:1066400001001305E55697D7FF1F239AB7D4C2055B
:10665000C18197800100E78060DF97000000E7803C
:10666000C0BFF24005618280D147D14517A5010026
:106670001305055617D7FF1F2313F7D29780010084
:10668000E780C0DC17D5FF1F035565D197000000D8
:10669000E78080F1F9B721C1411126C206C622C4A4
:1066A000AE848DC52A8497200000E78000BB97E761
:1066B000FF1F83C727B399CB22852244B240A6850A
:1066C00092444101173300006700C3D7B24022440F
:1066D000924441018280828079714AD006D622D4C8
:1066E00026D24ECE93F715002E899DCBAD67371776
:1066F00000409387A7AA1CC3B7E70400BC4F13064A
:106700000019854517D5FF1F034545C982971345D5
:106710001900B250225492540259F24945618280C4
:1067200093F725006388071E2D4697A501009385E2
:106730006558480097800100E780E0C597F6FF1F85
:1067400083C6C6FA139706014183954763F9E70CA0
:10675000014417F5FF1F130565E9130630051308FB
:106760005004930810041303B004130E900593070C
:10677000640063F4F6043A84FD5997F4FF1F83C460
:10678000E4E697F7FF1F83C777E6A204DD8CAD67C9
:106790009387B755638CF41463E3970AA9679387CB
:1067A000A755638FF414A28517F5FF1F130505E4A1
:1067B00097000000E78060EE39A2B307850083C52B
:1067C0000700639AC50483C517006396050583C552
:1067D00027006392150583C53700639EC50283C5F4
:1067E0004700639A650283C757006396C703A2896F
:1067F0000DE897F5FF1F83C565EFB3853541C205E9
:1068000017F5FF1F130585DEC1814E959700000027
:10681000E780A0E8E9A005044204418089BF3A84EA
:10682000FD598547E3EB87F445C8854517F5FF1FFC
:106830001305C5DB97000000E78020E671A8B1676B
:106840009387C7556380F404B5679387D755E39C56
:10685000F4F4A28517F5FF1F130545D99730000002
:10686000E78040BE89476300F4069305E4FFC20554
:10687000C18117F5FF1F130585D797200000E7801A
:10688000C09D91A00546A28517F5FF1F130505D6EB
:1068900097F0FFFFE780E06697F7FF1F83C7C7D435
:1068A0009DE397E7FF1F83C7E79391CF4800978049
:1068B0000100E78040DA93150501C1814800973057
:1068C0000000E78020B8A68517A501001305853CC8
:1068D00097800100E78080B7FD57E39CF9F097F7B8
:1068E000FF1F238507E01345290025B5A28517F56D
:1068F000FF1F1305A5CF97F0FFFFE7808071E1B779
:10690000A28517F5FF1F130565CE97F0FFFFE780FF
:10691000007255BF93F745000145E38C07DE17A5CC
:1069200001001305653897800100E78000CA9730A1
:106930000000E78020C013454900E1BB411122C49B
:1069400037E404005C5C06C6354697A501009385D4
:10695000A5E617B501001305A5A0829711E917A5B3
:1069600001001305E53597800100E78000C601A00E
:106970008327041C82972A84054597B00000E7808E
:10698000407997600100E78060FE97600100E78032
:1069900060D397B00000E780C08A2285B2402244CD
:1069A000410182801567B71700401307575598C3F8
:1069B000D8439D66558FD8C3D843FD76758FD8C30D
:1069C000D8431367F70FD8C335671307C7CC98C3ED
:1069D00082804111054506C622C426C297C0FFFF2A
:1069E000E78020521305800497B0FF1FE780206CDA
:1069F000757585457D1597C0FFFFE780C03B7D75A8
:106A000085451305F53697C0FFFFE780204537140D
:106A100000408327840A8D451305002093E7072053
:106A20002324F40A97C0FFFFE780E038B7E40400AE
:106A300097C0FFFFE780007EC85897800100E7807D
:106A4000C0B817B501001305A59197800100E78034
:106A5000C0B78327840C8545414593E70708232465
:106A6000F40C97C0FFFFE780603F8D4513050008D9
:106A700097C0FFFFE780803E97C0FFFFE780606B15
:106A8000014597C0FFFFE780206E85450545894792
:106A900017F7FF1F230EF7C497C0FFFFE780606E54
:106AA00037070004B7E700E023A0E71097D0FFFF07
:106AB000E780000097D0FFFFE780C0139700000039
:106AC000E78000E897000000E780008A9700000058
:106AD000E780A0B497E0FFFFE780A0EF97000000F9
:106AE000E780601097000000E780600B83A7040830
:106AF00017050000130585BE829797D7FF1F238FC8
:106B0000A788BC4C13060064854582979700000057
:106B1000E78080E997C0FF1FE780808D0145828074
:106B2000B7F7070003C70701A547AE866316F7004E
:106B30009397450191C301A0AA850146254517C336
:106B4000FF1F6700A3C64111B2862E86AA852D4578
:106B500006C697C0FF1FE78060C5B24001454101EE
:106B600082809307000463E8C7021D71A2CC2A84C7
:106B7000080886CE32C697800100E780C081B24601
:106B80001008A285294597C0FF1FE78020C2F64064
:106B90006644256182803955828041110D658D459D
:106BA00006C697C0FFFFE7800021B71700408D663B
:106BB00023A6D70A17F5FF1F1305C5B31387C70A06
:106BC0009387870A1CC15CC5856689675CC958C103
:106BD00014C518C9B7E70400B24003A3871E4101DA
:106BE000028397F7FF1F83C767B299EF411106C66B
:106BF00097100000E7808060B240854717F7FF1FBD
:106C00002306F7B041018280828011C589C517C370
:106C1000FFFF6700A3598280411126C2AE848D45D3
:106C200022C406C62A8497C0FFFFE7802023B71737
:106C3000004099C803A5C70C418D23A6A70CB240FC
:106C4000224492444101828003A5870C418D23A4F4
:106C5000A70CF5B78347050003471500A207D98F96
:106C6000C2076177C18713072720639AE70083452E
:106C700025003705040017030000670023FA82800F
:106C800017F6FF1F1306C6A88147B2861303F00F3D
:106C9000A9483308F6000348080013F7F70F630705
:106CA000A80C630668008507E39517FF2947B3879B
:106CB000E6002380A70097F7FF1F938727A65DA80C
:106CC000411113D765001347170006C693F6350028
:106CD000058B954791CA054699476387C6000946C3
:106CE0009D476383C600A14713F645003336C000B5
:106CF00093F68503050685C2A145638BB604E1457D
:106D0000638AB604930580026388B6049305800302
:106D10006393B600914697F5FF1F2386F5C697F556
:106D2000FF1F2381C5C697F5FF1FA38DD5C4BE8560
:106D300017A501001305450297700100E780007157
:106D4000B240854717F7FF1FA30FF7C241018280AA
:106D50008546D1B78946C1B78D4675BF17A50100D5
:106D600013050502177301006700436E17F7FF1F35
:106D70001307C79ABA972380B700E147E302F5F4F7
:106D800093077002E30CF5FC82802A8723800500BC
:106D9000814717F5FF1F1305A5971308F00F294624
:106DA000B306F50083C606006396E60297F6FF1F5A
:106DB0009386C696B69783C7070005452380F500DE
:106DC0009947636EF7029D4763FDE700E147630D56
:106DD000F7008280638506018507E393C7FC0145C0
:106DE000C5B7238005008280B737004003C737004E
:106DF00083C7050093F70704D98F2380F5008280AD
:106E0000797126D24AD097F4FF1F83C4A4C917F919
:106E1000FF1F130969C806D622D44ECE52CC56CADB
:106E20005AC8B307990083C7070093F7F70FA5C7A0
:106E30009387140093F7F70F0D476361F70C17F76B
:106E4000FF1F2301F7C697F7FF1F938767C5A69714
:106E500083C707001307100293F7F703638FE72830
:106E60006363F70A05476380E720E389076E0947F4
:106E70006389E71413070002E38EE758B7E700E0E1
:106E80003707400023A0E71801000100CA942380BF
:106E9000040023A0E710B787004003C76700058BF5
:106EA000E309077897F6FF1F83C6E6BF0547E3941B
:106EB000E67629472381E70209472383E7022385F2
:106EC000E70297F7FF1FA38107AC97F7FF1FA38C7B
:106ED00007BCB7870040A381070017F7FF1FA30770
:106EE00007AA05472383E700B2502254925402595F
:106EF000F249624AD24A424B4561828097F7FF1FAE
:106F0000238207BA89B7130730026386E70A63E66C
:106F1000E71413074002638AE70813070003E39F9F
:106F2000E7F497F7FF1F938767B7A69703C7070094
:106F3000A1471377F70FE31AF71C17EAFF1F130A8D
:106F4000AA7E83476A0097F6FF1F2385F6A297E77C
:106F5000FF1F83C7D77D91C7FD5797F6FF1F238B70
:106F6000F6A097E5FF1F83C5357C97F7FF1FA38326
:106F7000B7A097E7FF1F83C7277B93F907089306FE
:106F8000000493F707066393D7529307A009638D14
:106F9000F51A63EAB7169307F005638AF54E93076F
:106FA00050096388F52E014479ABFD5717F7FF1F91
:106FB0002301F79CE1B5FD5717F7FF1F230AF79A46
:106FC00075BD17A50100130525ED97700100E78039
:106FD000C05F97F7FF1F938767ACA69703C40700AE
:106FE000814917FAFF1F130AAA8C1374F40F97AA8A
:106FF0000100938AEAEA63C7890429459770010072
:10700000E780A049854717F7FF1FA301F78A17F705
:10701000FF1F230E878817F7FF1F2307F79637E711
:1070200000E0B70640002320D71801000100378692
:1070300000408347A60293F7370F2305F60223206B
:10704000D7102DBDB3073A0183C5070056858509C2
:1070500097700100E780803F79BF854717F7FF1FD2
:107060002306F78421BD17A501001305E5E29770FB
:107070000100E780805597F7FF1F938727A2A69707
:1070800003C40700814917EAFF1F130A2A76137405
:10709000F40F97AA0100938AAAE063C589042945E1
:1070A00097700100E780603F854717E7FF1FA30D3A
:1070B000F77217E7FF1F230A877217F7FF1F2305D1
:1070C000F78C37E700E0B70640002320D71801000F
:1070D0000100378600408347660293F7370F23038A
:1070E000F602B1BFB3073A0183C50700568585098B
:1070F00097700100E78080354DB7854717E7FF1F80
:107100002304F76EA5BB9307400A638DF5349307FC
:10711000200B6388F5369307100AE396F5E883079A
:107120002A00014463D1074297E7FF1F83C7F75F37
:1071300093F63700638E061A0546638EC62209460B
:107140006399C61A1D4775A217E5FF1F0345E55D44
:10715000C94717EAFF1F034A5A5D97E5FF1F83C51A
:10716000E55C17E4FF1F0344745C6319F510CD4719
:107170006316FA1093077008639CF5021307300F2B
:10718000B7170E006308E4001307900DB7B70400AB
:107190006314E40817E7FF1F2324F77EBE8517A5B5
:1071A0000100130565D097700100E780202AE5BB38
:1071B00093078008639DF50033048040B77746004D
:1071C0001374F40F938787CDB3D78702E1B7930782
:1071D0009008639AF5003304804091671374F40FAC
:1071E0009387C766D5B79307A008639BF500330460
:1071F0008040B7173D001374F40F93870790E9B7E9
:107200009307B008639AF5003304804091671374C4
:10721000F40F938797D04DBF93F5F5078D47639B88
:10722000F50033048040B7975B001374F40F938725
:1072300007D859BF8947639BF50033048040B7776F
:107240000B001374F40F9387071BBDBF8547639A28
:10725000F50033048040DD671374F40F938767E310
:10726000A5B789E9330480408D671374F40F9387C1
:1072700077DC99BFF1679387072029BF970000004B
:10728000E78040A0A285528597000000E780809F9C
:1072900019BB9305610017E5FF1F0345054917E476
:1072A000FF1F0344944897000000E78040AE930519
:1072B0007100228597000000E78060AD3C0017E771
:1072C000FF1F2329F77C834761002304F1008347D4
:1072D0007100A304F100894717E7FF1F230CF7682B
:1072E0008357810017E7FF1F2310F7440944A1AC1F
:1072F000154793F64700B336D00093F7870385060A
:1073000085C32146638BC7066146638AC706130699
:1073100080026388C706130680036393C700914702
:1073200017E6FF1F2300D66697E6FF1FA38CF664BF
:1073300097E7FF1F2389E76417E7FF1F0347073F0E
:107340009376070497E7FF1F83C7573E8DEE1377A9
:10735000770C93067008630CD7021377F7078D46F6
:10736000631ED70AB307F040B7955B0093F7F70F9A
:10737000938505D881A81947ADBF854755B789477B
:1073800045B78D4771BF930670086311D702130785
:10739000300FB7150E006389E7021307900DB7B5DC
:1073A00004006383E7021307700845BF9306800C4F
:1073B0006311D702B307F040B775460093F7F70F94
:1073C000938585CDB3D5F50297E7FF1F23AAB75A5A
:1073D000F9B39306900C631AD700B307F040916598
:1073E00093F7F70F9385C566F1BF9306A00C631B57
:1073F000D700B307F040B7153D0093F7F70F93851B
:107400000590C9B79306B00CE319D7F4B307F04061
:10741000916593F7F70F938595D06DB78946631BF8
:10742000D700B307F040B7750B0093F7F70F9385BC
:10743000051B49BF8546631AD700B307F040DD65D9
:1074400093F7F70F938565E3B5BF09EBB307F040FA
:107450008D6593F7F70F938575DCADB7F16593856F
:1074600005209DB783472A00C18B99C7854717E739
:10747000FF1F2304F75005BE97E7FF1F238F074E1A
:107480001DB6854717E7FF1FA30FF74E29BE3C0027
:1074900017E7FF1F2320F760094793070003231412
:1074A000F10097E6FF1F2387E64C2DBD639A07582E
:1074B000A94763ECB74417A70100130727878A057C
:1074C000BA959C41BA97828717E4FF1F0344F425BD
:1074D000094A630C440F636C8A0885476309F40A00
:1074E0009307F00F17E7FF1F0347C74863F6E7004E
:1074F00017E7FF1F2300F74817EAFF1F034A8A47D1
:10750000930700041374FA0F63F447011304000493
:1075100097E7FF1F9387075883AA0700228617E57E
:10752000FF1F13056520D685330A8A40A29A9770FB
:107530000100E78040E697E7FF1F238D474397E769
:10754000FF1F23A9575597E7FF1F83C7B74215476A
:10755000639AE762B7E700E03707400023A0E71827
:1075600001000100B7860040238086028DA58D476B
:10757000630CF40A9947E315F4F697A70100938783
:10758000678117E7FF1F2327F750A947A1BF17E718
:10759000FF1F0347475197E7FF1F9387A73F4946C0
:1075A00097A50100938505886306870097A50100CC
:1075B000938545833E8597700100E780C0DD17E71E
:1075C000FF1F2329A74CC94731BF97E6FF1F83C67A
:1075D000864D054797E7FF1F9387C73B6394E602F5
:1075E0003E851306700297A501009385258197704B
:1075F0000100E78040DA17E7FF1F232DA748930714
:107600007002CDB53E851306300497950100938531
:10761000257997700100E78000D817E7FF1F232B1B
:10762000A746930730047DBD97E5FF1F83C5E50F8F
:1076300017A501001305858897700100E78000E118
:10764000854A17EBFF1F034B0B4697E5FF1F83C5CA
:10765000C50D17A501001305658663185B0B9770B0
:107660000100E780A0DE97E7FF1F83C7070CB5CBBB
:10767000E368F4E6179401001304047F638C670148
:10768000179401001304C47E638647011794010018
:107690001304847F228597700100E780C0FB137577
:1076A000F50F93071500860717E7FF1F2304F72E32
:1076B0008D4717E7FF1FA30FF72C97E7FF1F93874F
:1076C000672D0147BE861376F70F89076365A6020B
:1076D00097E7FF1F23A0D73C97E7FF1F83C7872BA0
:1076E00011B5979701009387277117E7FF1F232391
:1076F000F73A9147C5BB3306E40003460600A38072
:10770000070005072380C7007DBF97700100E78051
:10771000E0D397E7FF1F83C74701E1D7E362F4DCBB
:107720001794010013044471638C570117940100EE
:107730001304047163864701179401001304C47194
:10774000228597700100E78000F11375F50F93070C
:107750001500860717E7FF1F230EF7228D4717E74F
:10776000FF1FA309F72297E7FF1F9387A72201476F
:10777000BE861376F70F8907E37CA6F43306E40090
:1077800003460600A380070005072380C700D5B77E
:1077900097E5FF1F83C565F9179501001305C572AD
:1077A00097700100E78080CA97E7FF1F83C7571EC5
:1077B00093E7470017E7FF1FA30CF71C83472A0036
:1077C00017E7FF1FA304F71C6FF0EFFD17950100EB
:1077D0001305C57097700100E78020DF97E7FF1F52
:1077E0009387C71A83C7070017E7FF1F230EF7F217
:1077F00017E4FF1F0344041833348000A9B317951E
:1078000001001305E56E97700100E78000DC97E743
:10781000FF1F83C7F71793E7070117E7FF1FA309A8
:10782000F71683472A0017E7FF1F2301F7166FF0AB
:107830008FF7179501001305E56C97700100E7803D
:10784000C0D803470A007D8B51EFB787004003C7BC
:1078500067021377C70B136727002383E70203C769
:10786000A7021377C70B136727002385E70203C717
:10787000E7021377C70B136727002387E70203C7C5
:1078800027031377C70B136727002389E702854770
:1078900017E7FF1F230AF7F417E7FF1F2308F70076
:1078A00017E7FF1F2306F70C17E7FF1F2303F70C4B
:1078B00097E7FF1FA38A07F297E7FF1FA38807FE3A
:1078C00097E7FF1FA386070A97E7FF1FA383070A0F
:1078D00097E7FF1FA38A070A97E7FF1FA385071CE7
:1078E0006FF06FEC89476312F70297E7FF1F83C7BA
:1078F000E7E39146638CD70863E0F604638EE70CF8
:107900006369F70A05476380E70EFD5717E7FF1F16
:10791000A302F70637074000B7E700E023A0E71807
:1079200001000100B78600401306F0FC2381C60267
:1079300023A0E7106FF08FD4130720086382E708B5
:107940006362F70213071008E391E7FC37870040F2
:107950008347670293F7C70B93E727002303F702D8
:107960006FF06FE4130730086389E70213074008DC
:10797000E39DE7F8378700408347270393F7C70B5A
:1079800093E727002309F7026FF0EFE13787004004
:107990008347270393F73707F5B7378700408347B7
:1079A000E70293F7C70B93E727002307F7026FF06F
:1079B0008FDF378700408347E70293F73707F5B734
:1079C000378700408347A70293F7C70B93E7270049
:1079D0002305F7026FF02FDD378700408347A702AA
:1079E00093F73707F5B7378700408347670293F768
:1079F0003707ADB7179501001305C5519770010002
:107A0000E780A0BC97E7FF1F238007D2D5B3179567
:107A100001001305255197700100E78000BB97E72F
:107A2000FF1F239307D097E7FF1F9387A7F403C493
:107A30000700894763F3870009441374F40F21B6E4
:107A400013070002E393E7EC6399090A638FF500DB
:107A5000930720026381F50817950100130505506F
:107A600097700100E780809E4DB5179501001305C2
:107A7000254C97700100E78040B50144179B010039
:107A8000130B4B4CA14AB3078A0083C507005A85E4
:107A9000050497700100E780609BE31654FF17957B
:107AA00001001305E5AE97700100E78000B217E40E
:107AB000FF1F0344A4C711E497E7FF1F238907C4EE
:107AC00059B48947E313F4E4854717E7FF1F230000
:107AD000F7C46FF04FCD17E6FF1F034616C597E5B5
:107AE000FF1F83C585C417950100130525469770B0
:107AF0000100E780A0956FF00FCB638FF50493072B
:107B00001002E39BF5F497E5FF1F83C525C2179587
:107B100001001305A54597700100E780209397E7C2
:107B2000FF1F23A947F797E7FF1F938767E5944354
:107B300083D7470017E7FF1F0347E7E417E6FF1F58
:107B40002324D6BE1D4497E6FF1F2391F6BE97E778
:107B5000FF1F238EE7BCC5BA97E5FF1F83C505BD90
:107B6000179501001305054297700100E780008E0C
:107B700097E7FF1F238D07B897E7FF1F239607BAE4
:107B80006FF0CFF62547E387E79C19476391E7023B
:107B9000B786004023808602B7E700E03707400041
:107BA00023A0E71801000100130600FC41B31307EE
:107BB000100A6391E702B786004023808602B7E788
:107BC00000E03707400023A0E7180100010013067A
:107BD00080FCA9BB1307A009E38FE7FC1307400A49
:107BE000E38BE7FC13072002E386E7960547E38370
:107BF000E796B7E700E03707400023A0E718E391D6
:107C0000099601000100B786004023808602130612
:107C100020FC29BB17E7FF1F0347D7D56302F71ED8
:107C200063E7E7029547630EF70E99476308F70489
:107C3000B786004023800602B7E700E03707400020
:107C400023A0E718010001001306A0FCC5B19307AB
:107C5000F005630AF700930750096306F7009307DE
:107C60001002E317F7FCB7E700E03707400023A056
:107C7000E71801000100B786004051BF97E9FF1FD8
:107C800083C949CF93070004CE8A63F43701930A6E
:107C9000000497E7FF1F9387E7DF03AA070013F4A9
:107CA000FA0F2286D28517E5FF1F1305E5A7976017
:107CB0000100E780406EB3878940529417E7FF1FA9
:107CC000230AF7CA97E7FF1F23A687DC638E090202
:107CD000B787004023805703B7E600E0370640002F
:107CE00023A0C6180100010003C727021347070499
:107CF0002381E70203C727021377C70F2381E70217
:107D000023A0C6106FF08F97B7860040238006022D
:107D1000B7E700E03707400023A0E71801000100A3
:107D2000FDB5378700408347370097E6FF1F83C6BE
:107D3000F6C593F70708D58FA301F700B7064000F3
:107D4000B7E700E023A0D718010001001306A0FC4C
:107D50002301C70223A0D7106FF04F9297E7FF1FB0
:107D60009387C7D3A69783C7070093F7F70FC9CBAD
:107D700097E7FF1F83C727D3C1E717E7FF1F034715
:107D800077BF93070002631DF70617E6FF1F130670
:107D9000A699104217EAFF1F034A4A9997E9FF1F65
:107DA00083C9D99817E4FF1F03446498CE8752878C
:107DB000A28697E5FF1F83C58595179501001305DA
:107DC000E51D97600100E780606897E7FF1F238B40
:107DD00047BB97E7FF1FA38737BB97E7FF1F2384A6
:107DE00087BA97E7FF1FA3830792B7E700E037073B
:107DF000400023A0E71801000100B7860040C1BB86
:107E0000B7E700E03707400023A0E71801000100B2
:107E1000B786004015BD29472381E7020947238320
:107E2000E7022385E7022387E7022389E7026FF051
:107E30004F8903C76700118B6308078A83C7570000
:107E4000918BB5CF17E7FF1F0347E7C5854763133E
:107E5000F70697E7FF1FA388E7B297E7FF1F238581
:107E6000079897E7FF1F238307A497E7FF1F238146
:107E700007B097E7FF1F238E07AE97E7FF1FA38585
:107E8000079697E7FF1FA38307A297E7FF1FA3812A
:107E900007AE97E7FF1FA38E07AC97E7FF1FA385E9
:107EA00007AE97E7FF1FA38007C0B78700401147C1
:107EB0006FF04F8317E7FF1FA30AF78479BF854749
:107EC00017E7FF1F2302F79217E7FF1F2300F79E14
:107ED00017E7FF1F230EF7A817E7FF1F230BF7A8CD
:107EE00069BF854717E7FF1F2300F79017E7FF1FBC
:107EF000230EF79A17E7FF1F230CF7A617E7FF1FBC
:107F00002309F7A617E7FF1FA300078E17E7FF1F38
:107F1000A30E079817E7FF1FA30C07A497E7FF1FFF
:107F2000A38907A48280411106C697000000E7805C
:107F300080FBB787004023800700130740FC23869F
:107F4000E7001307C004A386E70017D7FF1F130736
:107F5000A77D2398E70017E7FF1F1307E780239A01
:107F6000E70017E7FF1F1307678C239CE70017E75D
:107F7000FF1F1307E797239EE70029472381E702A6
:107F800009472383E7022385E7022387E702238942
:107F9000E702A3810700930600F8A380D7009306A9
:107FA00090022380D700FD562383D7002381E7006A
:107FB000B706400037E700E02320D71003C71700BB
:107FC00013671700A380E700B24097E7FF1F239FC6
:107FD000079A41018280411106C697000000E780A0
:107FE00080F0B787004023800700130700FC23863A
:107FF000E7003147A386E70017D7FF1F1307C772B3
:108000002398E70017D7FF1F13070776239AE70087
:1080100017E7FF1F13078781239CE7002947238168
:10802000E70209472383E7022385E702A3810700CC
:10803000930600F8A380D700930690022380D70010
:10804000FD562383D7002381E700B706400037E7BA
:1080500000E02320D71003C7170013671700A38081
:10806000E700B24097E7FF1F239207924101828009
:10807000B7170E0017E7FF1F2324F790854717E770
:10808000FF1F2311F790A14717E7FF1F230DF78E5E
:1080900097E7FF1FA389078E97E7FF1F2386078EA9
:1080A00097D7FF1F2385076697D7FF1FA380076613
:1080B000814717D5FF1F1305A565FD5517D6FF1F6F
:1080C0001306C6652947B306F5002380B600B3063C
:1080D000F600238006008507E397E7FE97E7FF1F7A
:1080E000238C079A97E7FF1FA388079A97E7FF1F3C
:1080F0002385079A97E7FF1FA38F078697E7FF1F40
:10810000A38D078697E7FF1F2388078697E7FF1F42
:108110002383078697E7FF1F2382078697E7FF1FC2
:10812000A38C078497E7FF1F2389078497E7FF1F26
:10813000A3850796828017E7FF1F0347C7968547E9
:108140006316F70017030000670023E91703000018
:108150006700A3DD411122C406C617E7FF1F0347CE
:10816000879485472E8613F4F50FAA856317F704C5
:1081700017D5FF1F1305856F97600100E780A021C9
:1081800097D7FF1F23840772B78700402384870295
:10819000B7E600E03706400023A0C6180100010042
:1081A00003C7A7021377C70F2385E702B240224413
:1081B00023A0C61001454101828017D5FF1F13057A
:1081C000A55E97600100E780001D97D7FF1F238DF4
:1081D0000760B787004023828702B7E600E03706D2
:1081E000400023A0C6180100010003C767021377EF
:1081F000C70F2383E7025DBF411106C69700000049
:10820000E78040E7B2404101170300006700E3F256
:10821000411106C697F0FFFFE780C0BE97D7FF1F4A
:1082200083C7975C95C797D5FF1F83C5055C89C930
:1082300017D5FF1F1305855B97F0FFFFE780209D93
:1082400097D7FF1FA382075A97D7FF1F238E077266
:10825000B2404101828041C9D9C597D7FF1F83C76A
:10826000E772D1C3011122CC4AC84EC656C25AC0C9
:1082700006CE26CA52C42E89AA890144930A000454
:10828000371B030063772403B3078940C207C18308
:10829000BE8463F4FA0093040004C204C180130A8C
:1082A0001BD497D7FF1F83C727549DE37D1A631CF8
:1082B0000A00F2406244D2444249B249224A924AF8
:1082C000024B0561828097F0FFFFE780A0B3D1BF2A
:1082D000338589002694A685420497000000E78034
:1082E000A0E7418045B7828097D7FF1F9387477FDC
:1082F00018429C4383D645000345070083C5C70049
:10830000035646006396A50083D5E700638DD5022A
:10831000011106CE2386A7002397D700B705CF000B
:10832000DC4B9385757D05077D162EC22300010069
:108330003AC42316C1002317D10099C30A85829736
:10834000F240056182808280DC4DDC4B81CFB7E753
:108350000400904503A38705914517D5FF1F0345EA
:108360006578028382806D713C083EC6B707E500E0
:10837000232291103EC8AA843C083285232611107E
:108380003ECA23248110232021112E89973000001A
:10839000E78020562A84979501009385A5C3178509
:1083A0000100130525B897600100E780200AA28527
:1083B00017950100130585D297600100E780000939
:1083C000294597600100E780400DB705CB009385F4
:1083D000757D680097100000E780405FA285680007
:1083E00097300000E7804043014781467000CA850E
:1083F000268597200000E780C08205CD2A849795C6
:108400000100938525BD178501001305A5B197606F
:108410000100E780A003A285179501001305C5CCD4
:1084200097600100E7808002294597600100E7809E
:10843000C0068320C1100324811083244110032926
:1084400001105161828097D7FF1F93876769184297
:108450009C43797122D406D60348070083C80701DC
:108460002A8483D64500035546006396080183D8C5
:108470002701638DD8022388070105072399D700B8
:108480003708CC00DC4B1308787D3ACC1307F5FF96
:1084900042CA23080100231EE100231FD10099C70F
:1084A000080832C62EC482973246A245228597001C
:1084B0000000E78080EBB2502254456182806D71EC
:1084C0003C083EC0B707E5003EC23C083EC4232638
:1084D0001110232481102322911023170100231847
:1084E000010023190100231A0100231B010097B783
:1084F000FF1F83D727ED99E3C167FD172316F1000E
:1085000097B7FF1F83D727EC91EB97D7FF1F938770
:10851000275D9C439C43DC4783D7070017B4FF1FAC
:10852000130444EA584C2317F10083574400484B86
:108530002318F10031E1979501009385A5B01785C7
:1085400001001305259E97600100E78020F0179534
:108550000100130565B097600100E78020EF294511
:1085600097600100E78060F38320C110032481102D
:10857000832441105161828097B7FF1F83C7F7E4BE
:1085800089EBB7E70400BC5782975C4C23AA07002D
:10859000E1BFFD1797B6FF1FA389F6E20356070157
:1085A000834704014C470A85230BF10097300000F4
:1085B000E780A02397D7FF1F938787529C430147EB
:1085C000814688430A866C0097100000E78060654A
:1085D000AA8429C1979501009385C5A61785010036
:1085E0001305459497600100E78040E6A68517953E
:1085F0000100130525A797600100E78020E52945C4
:1086000097600100E78060E9584CB7E70400BC5769
:10861000484B9DBF97B7FF1F83C737DBF5D7B7E739
:108620000400BC4F1044854517D5FF1F0345854BFB
:1086300082971DBF5C4EDC4BB9CFB1CD411122C436
:10864000178501001305058E2E84979501009385EB
:10865000A59D06C697600100E78040DFA2851795BB
:1086600001001305E5A297600100E78020DE29459F
:1086700097600100E78060E2B7E704002244B2405F
:1086800003A3870517D5FF1F0345C54513064006FD
:108690009145410102838280411122C417B4FF1F1A
:1086A000130404D01C4C06C689C7DC4399C34C484C
:1086B0008297584CB7E70400BC57484B82975C4CF4
:1086C000B240224423AA07004101828017B7FF1F4E
:1086D000130707CF834707009306F00B850793F72F
:1086E000F70F63E9F60097B6FF1F238BF6CC03451F
:1086F00007008280930700F8FDB783574500638623
:10870000071001114AC817B9FF1F1309A9CB52C49A
:10871000032AC90106CE22CC03274A0126CA4EC627
:1087200056C2F15735E31307D00DFD57636EC704EA
:10873000B7E9040083A709072A84130586004205C8
:108740004181B284AE8A8297232AAA000325C901F7
:108750005C49A9E7979501009385058B1775010082
:108760001305457C97600100E78040CE1795010016
:108770001305459A97600100E78040CD2945976031
:108780000100E78080D1DD57F2406244D244424983
:10879000B249224A924A3E8505618280938744000D
:1087A000B705CF002319F5009385757D3105971026
:1087B0000000E780A0210325C9018345640031053D
:1087C00097300000E78040050325C9012686D6853D
:1087D000310597300000E78040017146A2854A8547
:1087E00097600100E78020BB504419CA83A7890520
:1087F000854517D5FF1F0345E52E8297814769B749
:1088000097000000E780E0CBD5BFFD573E85828012
:10881000411126C297B4FF1F9384C4BAD84C22C416
:1088200037E404003C54484B06C68297DC4C0323D3
:10883000C4052244B240924423AA070017D5FF1F63
:108840000345452A854541010283411126C297D43B
:10885000FF1F9384E4289C4006C622C44AC0D5C3A7
:10886000DC43C5C35CC12300B5002A8497850100A1
:108870009385C574177501001305C56A97600100DB
:10888000E780C0BC294597600100E78000C19C409B
:1088900023A4070023A2070097B7FF1F938747B0C1
:1088A000DC4FDC4B91C7295597000000E78000DFC3
:1088B00097B7FF1F938707B1DC4FDC4B89C7970041
:1088C0000000E78020F537E904008327C9058945C2
:1088D00017D5FF1F0345052182978327C9059145B9
:1088E00017D5FF1F0345052082979C4003A347012E
:1088F0006309030022852244B240924402494101A7
:108900000283B24022449244024941018280011113
:10891000328506CE22CC26CA2E8497300000E7800E
:1089200040FDAA84978501009385856C1775010029
:108930001305455F97600100E78040B1030784009D
:108940000356640083554400A6861785010013056D
:10895000257697600100E78060AF294597600100A8
:10896000E780A0B397B7FF1F83C7E7A3639D970076
:10897000014597000000E78060D281450A85970095
:108980000000E780C0ECF2406244D244056182807E
:108990006D7123248110232611102322911093F747
:1089A00045002E84638707143C083EC0B707E500E6
:1089B0003EC23C083EC423170100231801002319BE
:1089C0000100231A0100231B010097B7FF1F83D763
:1089D000279D99E3C167FD172316F10097B7FF1F85
:1089E00083D7279C91EB97D7FF1F9387670F9C43F3
:1089F0009C43DC4783D7070017B7FF1F1307479A2D
:108A00002317F100544F835747002318F100DC4A25
:108A1000A1E7978501009385E561177501001305AE
:108A2000655097600100E78060A21785010013057B
:108A3000A56297600100E78060A129459760010069
:108A4000E780A0A5134544008320C11003248110B2
:108A5000832441105161828097B7FF1F83C7B79469
:108A60002555D9C3FD1717B6FF1FA30EF69203D6DF
:108A7000060183470701CC460A85230BF100973096
:108A80000000E78080D697D7FF1F938767059C4338
:108A900017B7FF1F1307C790978601009386C65E1E
:108AA00088430A866C0097100000E7808017AA842C
:108AB00051D9978501009385E55717750100130576
:108AC000654697600100E7806098A68517850100DC
:108AD0001305455997600100E78040972945976045
:108AE0000100E780809B268597000000E78000BB9F
:108AF00091BF93F725009DC7B7E70400BC474146E7
:108B0000814528088297255597000000E78000B925
:108B100028089305F00F97000000E78040D3134525
:108B200024001DB793F71500014599DF9700000059
:108B3000E78020991345140001BF5C4D411106C622
:108B400088C317D7FF1F232DF7F8B7E7040083A7C3
:108B50000708170500001305E5E38297B24097D791
:108B6000FF1F2381A7F801454101828001113335A0
:108B7000A000A307A100B7E7040083A7471706CE0C
:108B80001306F1008545130550308297F2400561C8
:108B900082808280411122C406C697D7FF1F83C7F7
:108BA000E7F5014489EF97B7FF1F83C7B763054413
:108BB00099E717D4FF1F034424A31344140022850C
:108BC00097000000E780C0FA178501001305456093
:108BD00009E4178501001305A5602244B240410154
:108BE0001763010067008386797122D4A30F010007
:108BF00037E404008327841726D24AD006D6AA84F5
:108C00002E89130550309305F10132C68297324602
:108C10008347F10193150601C18185CB01452EC61D
:108C200097000000E780C0F483274417B2454A86C6
:108C300026858297054597000000E78060F3B250D3
:108C400022549254025945618280832744174A86F0
:108C500026858297EDB741119397050122C406C678
:108C600026C2C1872E8463D40702B7E40400FC54F3
:108C700017A5FF1F03450578829719C1BC54829739
:108C80002165218DB240224492444101828093F7B4
:108C900015008DC7B7E7040083A7471A17A6FF1F63
:108CA0001306467497D5FF1F938585E417A5FF1F0C
:108CB00003454574829713451400E9B793F72500DF
:108CC00099CFB7E70400BC4F13060064894517A588
:108CD000FF1F0345257282971345240065B793F75C
:108CE00085009DC7B7E7040003A8871A1307401F34
:108CF00097A7FF1F83C70770814613064006994553
:108D000017D5FF1F0355C5DF0298134584009DBF8B
:108D100093F745000145BDD7B7E4040083A70418C5
:108D200017D5FF1F0355C5DD8297BC4C13060064A1
:108D3000914517A5FF1F0345E56B82971345440036
:108D400091B797D7FF1F83D7A7DB6398A70217D7E1
:108D5000FF1F2318B7DA17D7FF1F2315C7DA17D756
:108D6000FF1F2312D7DA2E86178501001305854CC5
:108D7000BE85175301006700636D17850100130559
:108D8000E54C17630100670043840357450097D7FC
:108D9000FF1F83D7E7D6631AF704C1674111F9179C
:108DA00022C417D7FF1F232DF7D437E4040097D729
:108DB000FF1F23A907D497D7FF1FA38107D47C4C9B
:108DC00006C6894517A5FF1F0345C56282977C4CDF
:108DD000914517A5FF1F0345E56182972244B240E4
:108DE000410117030000670023DB1785010013050D
:108DF000E545175301006700437D7D15954763E204
:108E0000A71C178701001307673A0A053A951C410A
:108E1000011122CC06CEBA972E84828717850100D5
:108E20001305454397500100E780207AA1A203C7AC
:108E3000250099476311F7022E8597000000E7800F
:108E400000F583456400178501001305A54197507F
:108E50000100E780A05F97B7FF1F238507381785BC
:108E600001001305E5417DBF03C725009547631940
:108E7000F702C16717D7FF1F035787C8F91703D534
:108E8000A5006309F702B7E7040083A7C717829715
:108E9000178501001305C53F97500100E780E07278
:108EA000854717B7FF1F230FF732178501001305FA
:108EB000A5408DBF97D7FF1F2394A7C483D7E50094
:108EC00097D6FF1F239FF6C283D7050197D6FF1FB2
:108ED000239AF6C283D7250197D6FF1F2395F6C2A2
:108EE00097D7FF1FA38C07C0631BE502B7E70400F9
:108EF000BC4F096613060690A14517A5FF1F034541
:108F0000654F82970356E4008355A400178501003E
:108F10001305453997500100E780405351B7930737
:108F2000700F2316F100B7E7040083A7870D17A67B
:108F3000FF1F0346264C6C0082974DF9854717D7D3
:108F4000FF1FA30DF7BA5DB717850100130585371D
:108F5000D1BD83C5250091476392F50217850100B5
:108F60001305C53797500100E78020669700000081
:108F7000E78080C2F2406244056182809947639233
:108F8000F502228597000000E78060E083456400D9
:108F9000178501001305052D97500100E780004B50
:108FA000D1BF9547639AF50083471400E1F3178515
:108FB00001001305E534BDB5178501001305C5345F
:108FC000E1BF82806D71232481102326111023229A
:108FD0009110328401CD8947630AF5028320C110C4
:108FE0000324811083244110516182801785010080
:108FF00013054532AE8497500100E780005DA285DD
:10900000268597C0FFFFE7808055C9BFB7E70400FA
:10901000FC4728008297178501001305653097509B
:109020000100E780805A8347810039C41307000B91
:109030006380E7021387A7051377F70F8D4663ED6B
:10904000E602A285280097D0FFFFE78060C479B7C9
:109050008547E3F587F883459100177501001305EF
:10906000A521B335B00097B7FF1F238FB7FE9750E8
:109070000100E780A03D9DB703479100A207D98F6B
:1090800035671307D7556385E7086368F7022D67CF
:109090001307B7556387E70631671307C755638A18
:1090A000E70429671307A7556394E702A285280000
:1090B00097D0FFFFE780A0F715B739679306E765FC
:1090C000638DD70663E9F6001307E7556380E7066B
:1090D000A28528003DB73D679306F7556386D706FE
:1090E0001307F766E396E7FE97D0FFFFE7802010AF
:1090F000F5B50146A285280097D0FFFFE78060E024
:10910000F1BDA285280097D0FFFFE78080F0F9B578
:109110008947E3F587EC9305E4FFC205C181130598
:10912000A10097A0FFFFE78060084DBDA285280041
:1091300097D0FFFFE780A0F055B5A285280097D013
:10914000FFFFE78060FB59BD97D0FFFFE780E0039A
:1091500071B5411122C417A4FF1F1304E42AAA8683
:1091600017860100130606062285C14506C69750DC
:109170000100E780C0460357440097A7FF1F93876D
:10918000A7292393E700035764002394E700B24024
:10919000224441018280411106C697000000E78009
:1091A00080FBB7E7040083A7871417A6FF1F1306E9
:1091B000A625D54501458297B2404D4697A5FF1F8C
:1091C0009385852513057030410117030000670062
:1091D000E3A161712324811A37E404008327040882
:1091E0002326111A2322911A2320211B232E311901
:1091F00017050000130565A6829717A9FF1F13091D
:10920000691F994785442300A900231CF100978515
:109210000100938525FF930740061775010013058C
:1092200065D0231CF1082308910097C9FF1F93897B
:10923000094C97500100E780602183D5090017850C
:109240000100130525FB97500100E78020202945E8
:1092500097500100E780602403D5090085699700D5
:109260000000E78040EF8327441710088545130569
:10927000503082978327441717A6FF1F1306C6197D
:10928000CD451305703082978327441717A6FF1F1B
:1092900013068616B5451305603082978327441759
:1092A0003008894513051031829783274417300908
:1092B000894513052031829783274415938509C872
:1092C0000D45829783274415938509C811458297D8
:1092D000A3059100230691002308910002CD230CE1
:1092E0000100832784163009914513057040829749
:1092F000832784161306B100854513050040829725
:1093000083278416700085451305104082978327B4
:1093100084163008854513052040829783278416DC
:1093200010088545130550408297832704157D5505
:109330008297832744137D5582977D5597A0FFFF21
:10934000E78080318327440C829797A0FFFFE78056
:10935000C00C8327841417A6FF1F1306E60AD54501
:109360000145829789471306700F81452809230616
:10937000F1009790FFFFE78040D68D471306000865
:1093800081452808230CF1089790FFFFE780E0D47F
:109390009147230CF10097770100938727AA984300
:1093A00083C747003AC8230AF10097D0FFFFE78040
:1093B000C0EA70008545054597A0FFFFE780E030D3
:1093C00030099305700F094597A0FFFFE780E02F54
:1093D0003008930500080D4597A0FFFFE780E02EB9
:1093E00010089545114597A0FFFFE780002EC16743
:1093F00017C7FF1F1307C770F9171CC323220700E5
:1094000017A5FF1F1305C5FE97A0FFFFE780C02A21
:109410008327C41D17C5FF1F1305056D82973C48A0
:1094200003450900854582978320C11A0324811AC8
:109430008324411A0329011A8329C1195D6182809D
:10944000C16717C8FF1F0358A86BF9176301F80815
:109450003DCDB5CD011126CAB7E4040083A784121F
:1094600022CC2E862315B10006CE2A8401478146E0
:10947000ED45428582972AC611ED17850100130537
:1094800065D997500100E7804014F2406244D2440D
:1094900005618280FC440356A100A28582972C00BE
:1094A00017C5FF1F0355C56597A0FFFFE780802DF7
:1094B00069DD17850100130525D797500100E78066
:1094C000C01083A7C412ED45280082977DBF82801B
:1094D000411106C61DC9854717A7FF1FA303F7F251
:1094E000354697A5FF1F938525F11305603097A793
:1094F000FF1F238907F097F0FFFFE780206FB2403E
:10950000410117F3FFFF6700236997A7FF1FA38A95
:1095100007EEF9B7C16717C5FF1F0355655EF91759
:109520006307F500B7E7040003A3C717028382802F
:10953000854717C7FF1F2303F75C014517F3FFFF9C
:10954000670003631793FFFFE70283B42A8408458B
:109550002E89B28919C900C1971500009385A58687
:10956000610597300100E780800181447D5A9710A2
:109570000000E780E03963C7A4048144971000002D
:10958000E780003A63C8A40497C7FF1F9387C757B3
:109590009C43DC47B307F94091872302F4006383BF
:1095A00009048327C900B307F4409587A302F40098
:1095B0001C4C89C79C4799C3228582971793FFFF4C
:1095C000670043B05C44139714008504BA97239056
:1095D000470171BF1C48139714008504BA97239064
:1095E000070069BF832789000547B307F4409587C3
:1095F000A302F40083570400638EE7028DC309477A
:109600006384E7040D47E395E7FA978701009387A2
:10961000E7231CCC978701009387472411A89787DD
:109620000100938727EA1CCC97870100938787EA7C
:109630005CC8BDBF978701009387C7D51CCC9787AF
:109640000100938727D6EDB7978701009387C7243A
:109650001CCC9787010093872725D9BF95E51793E1
:10966000FFFFE70283A400461844834794007583F4
:109670009D8B6317F70097100000E78060B448C423
:109680001793FFFF6700A3A482801793FFFFE702F1
:1096900023A013893500C16442094111AA890144FC
:1096A000F11413590901054A2EC697100000E780EE
:1096B0002026B2456348A400014541011793FFFFEE
:1096C000670043A083A7090013171400BA9783D734
:1096D00007006388B7006394970063742A01050448
:1096E000E1B70545D9BF1793FFFFE7028399AA8920
:1096F0002E89328BB6843A8ABE8A97A00000E78012
:1097000020FB71C9268597200000E78020098D473E
:1097100063E7A7007D551793FFFF6700039A83DB7C
:10972000440097100000E780A0242A8497100000CE
:10973000E78040259307740031443305850263CDEB
:10974000A70297100000E780A02297100000E78092
:1097500020222A8497100000E780C022930774001B
:1097600031443305850263C3A70497100000E780E6
:1097700020209307450029A897100000E78080204B
:10978000330585021307F0179307C017E35FA7FAA5
:109790002D55E3C277F963040B02D6865286A6855F
:1097A0004A8597200100E78020BAB5B797100000DE
:1097B000E780401D330585029307C5FFD1BF83278E
:1097C00049001385C90083D5270097000000E78072
:1097D00000EC61F581B769553DBF97C7FF1F23971F
:1097E000A73297C7FF1F93872732904381470C46C4
:1097F0003307F500420741836393B70082805446E4
:10980000139847008507C2962390E600D5B797C7FF
:10981000FF1F9387672F9C4303C58700828017C56E
:10982000FF1F0355A52E82801793FFFFE702E387F2
:10983000C1671387D7FF630BE502636AA700F117BF
:109840006300F50201451793FFFF67004388138704
:10985000E7FF6302E502FD171D8D13351500E5B71F
:1098600097500000E780C0267D15C5BF97500000C7
:10987000E78040FBD5BF97500000E78060F9EDB767
:109880001793FFFFE70263824111AA8401442EC6A9
:1098900097100000E780C008B2456348A400014566
:1098A00041011793FFFF670083829C481315140042
:1098B0003E9583570500E385B7FE0504C9BF0348FD
:1098C0005500814693F7F60F63E5070181473E8512
:1098D0008280584593975600BA9703D7270063169E
:1098E000B70003D70700E304C7FE8506E1BF834640
:1098F000450001479377F70F63E4D700814711A82C
:109900001C45131657000507B29703D60700E3134B
:10991000B6FE3E8582801783FFFFE70263779317C9
:109920000501C18797CAFF1F938A0A1E635BF0086F
:1099300083A70A00C0479C4703570400198D4205BE
:1099400041816368F500014422851783FFFF6700AA
:10995000637712052A94CDBFDC4713944900014A6E
:109960003E94834744006341FA02014A834754000E
:109970006349FA028509C20993D9090183A70A003C
:109980009847E3EBE9FCC1B71C4413195A00A685BC
:109990003E994A8597000000E780C0EE05E1050A80
:1099A000C9B75C4413195A00A6853E994A859700A9
:1099B0000000E78020ED19E1050A4DBFE30C09FA2C
:1099C00061B7AA8481495DBF1783FFFFE702E36D9A
:1099D0001C452A8481E79307C5001CC51C4423123B
:1099E00004001CC09307F00F63EDB70093F5F50F6B
:1099F000228597200000E78020E21783FFFF6700A1
:109A0000036D93940501C167C18063F9F500A685D4
:109A1000228597200000E78040E5C5B7C18193F516
:109A2000F50F228597200000E78000DFA6852285BC
:109A300097200000E78040E0C9B797C7FF1F9387D2
:109A4000A70C884382801C4599C797C7FF1F23AD89
:109A5000A70A014582807D55828097C7FF1F9387A3
:109A6000A70A984383474500484792073E9582805E
:109A70001783FFFFE7026363617100451C183EC650
:109A8000B70780013EC81C183ECA8357440002CE67
:109A900002D002CC231EF100834784002A8902D21F
:109AA0002301F1023C083ED402D697000000E78073
:109AB00000FB835705002316F10297500000E78052
:109AC00060C42307A1025C4003556400F18313F7CF
:109AD00017008347F10252055181F99BD98FA307E3
:109AE000F10297100100E780807539CDAA840355F3
:109AF000050097A00000E78080BC83D704002AD22D
:109B00006800231CF10083D72400231DF1001C48AA
:109B100003D647008C4397200000E78000CD8347A1
:109B2000B400CA8617860100130646808117A30574
:109B3000F4006C00481097200100E780E0805D6130
:109B40001783FFFF6700A3582155D5BF1C45B1CF30
:109B500003C5A700894613576500630BD7028D46DE
:109B6000630ED70285466300D7021307400633050C
:109B7000E50203C7B700418B15CB83C7B700BD8B88
:109B80003355F54082801375F5031307803EC5B742
:109B900009671375F50313070771D1BF372709004C
:109BA0001375F5031307077CD9B701458280178326
:109BB000FFFFE702834F03A98500630C0904834775
:109BC000B900AE8493F7070E85C30345990093054A
:109BD00020030D810505B305B50288446105973062
:109BE0000100E780E0A935A02E8597000000E780FE
:109BF00020F62A8419CD97000000E780605C832559
:109C0000C900B307B54063FA87002E94B305A4409A
:109C1000E9F51783FFFF6700834B85457DBF1783F9
:109C2000FFFFE70283482A8403D50500011132C6ED
:109C300036C43AC22EC002CA02CC02CE97A000009F
:109C4000E780E0A782452ACA22852ECC9700000033
:109C5000E780E0E003570500231EE1009750000075
:109C6000E78040AAA24632469247230FA1003687DA
:109C70004C08B2862285014697000000E780E0A6E6
:109C800005611783FFFF670083441783FFFFE70227
:109C9000C34161711C183EC6B70780013EC81C183D
:109CA0003ECA3C0800453ED4AA8402CC02CE02D073
:109CB00002D202D697000000E78060DA83570500E1
:109CC00035592316F10297500000E780A0A323071F
:109CD000A10209C48357440081EB21594A855D6183
:109CE0001783FFFF6700A33E0355640052055181AF
:109CF00097100100E780A0542A8965D18347B400FA
:109D000093F7070E99C71305840197300100E78088
:109D1000609983574400231EF10083478400230188
:109D2000F1025C4003550900D98313F70708834704
:109D30001102231CA10093F7F707D98FA300F102AA
:109D400083572900231DF1005C40F18313F71700AE
:109D50008347F102F99BD98FA307F10297A0000076
:109D6000E780E0952AD235D983479400680013979D
:109D700057008347B400FD8BD98FA305F4001C481E
:109D800003D647008C4397200000E78000A6A687F3
:109D90001777010013078759740005464C10268574
:109DA00097000000E78060942A890DD98347B400AA
:109DB000A685FD8BA305F40097000000E78060DF17
:109DC00031BF1783FFFFE702432E832485FE2A84D9
:109DD0004111268597000000E78080D7834734FF34
:109DE00093F7070E8DCB2AC6268597000000E780E3
:109DF00060C809CD834734FFB245FD8BA309F4FE4B
:109E000091C5228597300100E78080874101178343
:109E1000FFFF6700C32B7DD98327C4FF2685829768
:109E200075F5834734FF93F7070E91C72285973066
:109E30000100E7802087032584FE97000000E7806B
:109E400000E5E9B71783FFFFE70223239C41411197
:109E50002A8903C7070089472E84935667006380C9
:109E6000F6040D466388C6049307F0076304F702FF
:109E70002E8597200000E780C0A7AA848149C16B86
:109E8000130C490097C7FF1F938707C89C43984747
:109E900063E4E90441011783FFFF6700C32103D78F
:109EA00045008547E3F8E7FE2E8597200000E78010
:109EB000A0A9E1B703D74500E3FEE7FC2E85972074
:109EC0000000E78000A3AA84228597200000E78095
:109ED00060A4C204C98C5DB7DC470355A900139A7E
:109EE00049003E9A93170501C187635DF0008357CF
:109EF0000A006397A70263E774038327CA00034D30
:109F00005A002DA0A1672167A98F1307F7EFE3740B
:109F1000F7FE6397090097000000E780209161FD3C
:109F200085098DB783278A00034D4A00835DA90008
:109F300003576900216A138BC7003AC6814A33CAA6
:109F40004D01631E5D0197C7FF1F938767BC9C434C
:109F5000E1DBA2866286814526858297D1B7A1671B
:109F60009387F7EF930C4BFF63F24703B2455A8593
:109F700097F0FFFFE780A0710DC103278B0010470A
:109F800009CE10436382C4023107D5BFEE856685D2
:109F900097000000E780008F71F993861A0093FA0A
:109FA000F60F130B0B0271BF835644005C43E3E9C9
:109FB000F6F622853AC697100000E780807DA167FB
:109FC0009387D7042A8A035D4400324763E89700E9
:109FD0008347D90093E707F8A306F9001C47668575
:109FE0002286E2858297C1670844FD17337AFA001A
:109FF000529508C02312A40125B797C7FF1F938766
:10A00000A7B09843814715C31447814763FFD50024
:10A01000939745004C47BE9519C903C75500814722
:10A020006375E600DC451606B2973E85828003C75D
:10A0300045008147E37BE6FE16069C45F5B717838E
:10A04000FFFFE702E304AA892E8A814497CAFF1F13
:10A05000938A8AAB83A70A00984763E6E4001783D4
:10A06000FFFF67002306DC471394440001493E9438
:10A0700013BB140083474400634BF900014913BB31
:10A08000140083475400634FF9008504E1B7084486
:10A09000931759005287DA860146A2853E95829928
:10A0A0000509C9BF4844931759005287DA86054607
:10A0B000A2853E9582990509E9B71783FFFFE7025C
:10A0C000C3FE814517F5FFFF1305054897C7FF1F1E
:10A0D000239E07A297000000E780A0F61783FFFFEA
:10A0E0006700E3FE97C7FF1F938707A29C4395C3B2
:10A0F0001783FFFFE70263FB814517F5FFFF130599
:10A10000A54497000000E780C0F31783FFFF6700B6
:10A1100003FC82801783FFFFE70283F737E4040024
:10A120008327841241112315E100AE893289368AD2
:10A130003A8681460147ED45AA8482972AC621C9FD
:10A140000356A100D28597400100E780C0248327F1
:10A15000C413CE8526858297058905C98327440DBA
:10A160002314210101462C00268582972A8401C9E7
:10A17000B7E7040083A7C712ED4528008297228520
:10A1800041011783FFFF6700E3F34944D5B76554E6
:10A19000FDB75C41FD175CC182801783FFFFE702BA
:10A1A000C3F0B7E70400FC5F829795473305F502DB
:10A1B00081450D811783FFFF670063F11783FFFF60
:10A1C000E702A3EEB7E70400FC5F829795473305EB
:10A1D000F5020D811783FFFF670063EF1783FFFF11
:10A1E000E702A3ECB7E7040083A7870B035505003C
:10A1F00082971783FFFF670083ED1783FFFFE70256
:10A20000C3EA035505003287AE861796FF1F035633
:10A21000C62697C5FF1F9385E58F97000000E7804E
:10A22000A0EF1783FFFF670083EA1783FFFFE702B2
:10A23000C3E7B7E7040083A7C71782971783FFFF19
:10A240006700E3E81783FFFFE70223E6B7E70400B0
:10A2500083A7871397C5FF1F9385C58B82970145F9
:10A260001783FFFF6700A3E61783FFFFE702E3E31F
:10A27000B7E7040083A7C71F81451795FF1F035544
:10A28000C51B82971783FFFF670063E41783FFFFF7
:10A29000E702A3E1B7E7040083A7871397C5FF1F71
:10A2A00093854588829701451783FFFF670023E266
:10A2B0001783FFFFE70263DFB7E7040083A7C71F29
:10A2C00081451795FF1F0355451D82971783FFFF93
:10A2D0006700E3DF1783FFFFE70223DD2E8597800A
:10A2E0000000E780E0AF97800000E780E0EC178394
:10A2F000FFFF6700C3DD1783FFFFE70203DB9780E3
:10A300000000E780E0F61783FFFF670043DC5C494D
:10A31000E1175CC95CC583572501A1072319F50026
:10A3200083570501A1072318F5008280F147330503
:10A33000F50297C7FF1F9387E7809C433E95828075
:10A340008D476315F60803D74600854763F0E70895
:10A350001783FFFFE70263D5368536842E89971071
:10A360000000E780005929C9835744009314050170
:10A37000C18063E39704228597100000E78060574F
:10A38000FD14231294009307A0026300F5029307C3
:10A39000B0026307F50293079002631FF500228560
:10A3A00097000100E780C08501A80146CA85228583
:10A3B00097A00000E78060B01783FFFF670023D1FC
:10A3C000228597100000E780C003FDB7828097B612
:10A3D000FF1F938666779C42014599CF9843D442EC
:10A3E00017B6FF1F2322E6766396D70097B6FF1FA6
:10A3F00023AEE6741385C7FE82801783FFFFE70252
:10A40000C3CA97000000E780A04B71443305850262
:10A41000914597900000E78020E911E56555178385
:10A42000FFFF6700C3CA97B7FF1F23ABA770970052
:10A430000000E780E04833058502914597900000D1
:10A44000E78080E661DD97B7FF1F23ADA76E970019
:10A450000000E780E04697B7FF1F239DA76C970099
:10A460000000E780E04597B7FF1F2396A76C97771A
:10A4700001009387E7F017B7FF1F2321F76C9707B9
:10A480000000938707E917B7FF1F2327F76A0145E5
:10A4900079B71783FFFFE70243C1AA8517B5FF1FEE
:10A4A0001305456997100000E780C05B1783FFFF25
:10A4B0006700E3C11783FFFFE70223BF9700000097
:10A4C000E78060FD97100000E780405B97B7FF1FB3
:10A4D000938787679C4391CF1387C7FE19CB83D59A
:10A4E000C7FF17B5FF1F1305A56697200100E7807A
:10A4F00020191783FFFF670083BD1783FFFFE70263
:10A50000C3BA97000000E780C0EC09CD83478500FF
:10A510002A8493F7070499EB0355E50097000000A0
:10A52000E78080F91783FFFF670063BA8347C500A0
:10A530009304450117B9FF1F1309096185E38327B8
:10A5400009005CC997B7FF1F23A0976083274900C4
:10A55000F1FB97B7FF1F23AB975EE9B7FD17230603
:10A56000F500610597800000E780C0D6830784006E
:10A5700063CB07048347840093E707F82304F400C0
:10A58000B7E704009C5F82974205A9474181337574
:10A59000F5028347840093F707FCC98F2304F40076
:10A5A0008347D4003E951C402318A40089CF9843CC
:10A5B00019CB8347C4005040814585073305F50218
:10A5C000420541810297832709005CC897B7FF1FA6
:10A5D00023AC97568327490089E797B7FF1F23A726
:10A5E00097568347C4009DDF8355040117B5FF1FAD
:10A5F0001305055697200100E780800825B71783CB
:10A60000FFFFE70283AA97B7FF1F9387A7799C47AD
:10A6100001448583858B85E3AE84B2853A869710A5
:10A620000000E780804B2A8419C597100000E7805E
:10A63000C041829408CC22851783FFFF670023A9BD
:10A640001783FFFFE702C3A441112E8932C6AA89EE
:10A6500097000000E780C031324713060502CA8622
:10A66000970500009385C5CC17B5FF1F1305854CD2
:10A6700097000000E780E0F82A8425C99304C5000C
:10A6800097000000E780E0411946AA8526859710CB
:10A690000000E78080158545268597100000E7803B
:10A6A000601117750100130565CB4E9583450500B4
:10A6B000268597100000E78020165C4831468145CA
:10A6C000A1075CC85CC483572401E1172319F40077
:10A6D00083570401E1172318F4001C4C3E85978032
:10A6E000FFFFE780809FA304250122854101178396
:10A6F000FFFF6700239D1783FFFFE702039B4111C4
:10A70000AA842EC632C497100000E7806036004D40
:10A71000B2452246834784000CC050C093F7F7032C
:10A7200093E707042304F4002318040026859710F8
:10A730000000E780803183479400A9462317A400D6
:10A7400013D7370005073307D7029D8B85072306EC
:10A75000F400A306E40083C70401D8488507230F4B
:10A76000F7FE17B7FF1F1307273E5843232A04009D
:10A770009307440129E317B7FF1F2329F73C17B7B5
:10A78000FF1F2323F73C17B4FF1F1304643C2285EB
:10A7900097200100E78000E11C44858B5D8D19E561
:10A7A0008145228597200100E78080ED41011783D4
:10A7B000FFFF6700C3911CC317B7FF1F2328F7389B
:10A7C000D9B71783FFFFE702438E970500009385F3
:10A7D00065B7014597000000E78000B00145178389
:10A7E000FFFF6700C38E1783FFFFE702038C97000C
:10A7F0000000E78080B01783FFFF6700438D834729
:10A80000C500A5E31783FFFFE702238A2A840355C7
:10A81000E50097000000E78000C821C1834784005D
:10A8200093F7F7FB2304F4001C4091C7DC4381C776
:10A830004C400145829797000000E78080B917B52A
:10A84000FF1F1305E53097200100E780A0E50355C1
:10A85000E40097000000E78020C61783FFFF670031
:10A86000038782801783FFFFE702238497B7FF1FC8
:10A870009387872D97050000938565C817B5FF1F3F
:10A880001305052D23A0070023A207009720010030
:10A89000E780E0CE1783FFFF670063831C4D91CFF5
:10A8A000DC4381CF1783FFFFE70223808345070046
:10A8B00082971783FFFF67008381828097B7FF1F0E
:10A8C0009387472B9C4303C50700828097B7FF1FE0
:10A8D0009387472A9C4303C51700828097B7FF1FC1
:10A8E000938747299C4303C52700828097B7FF1FA2
:10A8F000938747289C4303C54700828097B7FF1F73
:10A90000938747279C4303C53700828097B7FF1F73
:10A91000938747269C4303C55700828097B7FF1F44
:10A92000938747259C4303C56700828097B7FF1F25
:10A93000938747249C4303C57700828097B7FF1F06
:10A94000938747239C4303C58700828097B7FF1FE7
:10A95000938747229C4303C59700828097B7FF1FC8
:10A96000938747219C4303C5A700828097B7FF1FA9
:10A97000938747209C4303C5B70011E11D458280A2
:10A9800097B7FF1F9387071F9C4303C5C7008280AB
:10A9900097B7FF1F9387071E9C4303C5D70082808C
:10A9A00097B7FF1F9387071D9C4303C5E70082806D
:10A9B00097B7FF1F9387071C9C4303D5070182802D
:10A9C00097B7FF1F9387071B9C4303C5270182800E
:10A9D00097B7FF1F9387071A9C4303D547018280CF
:10A9E00097B7FF1F938707199C4303D567018280A0
:10A9F00097B7FF1F938707189C4303D58701828071
:10AA000097B7FF1F938707179C4303C5A701828051
:10AA100097B7FF1F938707169C4303C5B701828032
:10AA200097B7FF1F938707159C4303C5C701828013
:10AA300097B7FF1F938707149C4303C5D7018280F4
:10AA400097B7FF1F938707139C438857828097B758
:10AA5000FF1F938727129C4303D5C702828097B7B5
:10AA6000FF1F938727119C4303D5E70219E11305C4
:10AA7000800C828097B7FF1F9387C70F9C4303C545
:10AA80000703828097B7FF1F9387C70E9C43C85B5D
:10AA9000828097B7FF1F9387670D8843828097B79F
:10AAA000FF1F9387E70C8843828019E17D558280E0
:10AAB000F5DE984265DFFDD917B7FF1F1307872E14
:10AAC0001847AA877155058B631D072403C5070026
:10AAD0001547E37DA7FC03C737001305F0057D1775
:10AAE0001377F70FE364E5FC03C35700E30003FCAF
:10AAF00083C86700E38C08FA03C7770049457917D4
:10AB00001377F70FE364E5FA03C7A70011481305AD
:10AB1000F7FF1375F50FE36BA8F803CE97000D4808
:10AB20001305FEFF1375F50FE362A8F803C8B7001D
:10AB30006309080065181378F80F1305600DE367C3
:10AB400005F703C5C700794879151375F50FE36F4D
:10AB5000A8F403C8D7000D457D181378F80FE367F4
:10AB600005F503D80701930E4017511842081358F2
:10AB70000801E3ED0EF303C8E7007D181378F80F22
:10AB8000E36605F303C827017D181378F80FE36F18
:10AB900005F103C88700C54E75181378F80FE3E771
:10ABA0000EF103D86701856E938EBEE06D184208E2
:10ABB00013580801E3EC0EEF03D847016D18420863
:10ABC00013580801E3E40EEF03D88701791842080F
:10ABD00013580801E36C05ED03C8A7017D1813782D
:10ABE000F80FE36505ED03C5B7011D487D15137525
:10ABF000F50FE36DA8EA03C5D70171487915137500
:10AC0000F50FE365A8EA03D5E7011308E00F7D150A
:10AC100042054181E36CA8E803C50702494879155C
:10AC20001375F50FE364A8E8C85301C937C83400A9
:10AC30005915130858BFE36BA8E603A8870237C568
:10AC40003400130555BF5918E36205E717B5FF1F18
:10AC50002320C5F203C6050117B5FF1F232CF5F00D
:10AC60000545E375C5E403D82501D04933760603CD
:10AC7000E31E06E203C61501E30A06E217B6FF1F4C
:10AC80002326B6EE83C5270001466387A50003C6C9
:10AC90001700F1453306B60283C707039305C002C8
:10ACA00072971A071307C70516031A97960846974F
:10ACB000B387B70241553E9732974207418363629B
:10ACC000E8061773FFFFE702433E368597800000D2
:10ACD000E780A06897000100E78020482A8497A0B9
:10ACE0000000E780805A2A9497F00000E7806026F1
:10ACF0002A9497900000E780A0812A9497F0FFFFA4
:10AD0000E780E06F2A9497400000E78060932A94E0
:10AD100097700000E780A09C22951773FFFF6700E3
:10AD2000033B82801773FFFFE70223384111A3071B
:10AD3000A10097A00000E780A0C59305F1001705CA
:10AD400000001305E5B597F0FFFFE780802F014570
:10AD500041011773FFFF670083371773FFFFE70297
:10AD6000433217B4FF1F1304E40303288400795906
:10AD70009368180097B4FF1F23AA140313781800D0
:10AD800063100802BA84BE89368B328A2E89AA8A59
:10AD900097F0FFFFE780E0A77D15269519E531596B
:10ADA0004A851773FFFF6700433197F0FFFFE78085
:10ADB00040A67D152695A167E353F5FE97B7FF1FC3
:10ADC0009387473598433E8C814B01CB014597F0E3
:10ADD0000000E7802044933B15004A85DA865686BA
:10ADE000D28597900000E780C04D2A8911CD1C4480
:10ADF000F99B17B7FF1F232BF7FA83270C00CDD33E
:10AE0000E3800BFA829769BF268597B7FF1F23ADB2
:10AE100007F897F0FFFFE780809C4146CE8517B585
:10AE2000FF1F1305A50197300100E780C05697D09A
:10AE30000000E78040990325040B97D00000E780CD
:10AE4000009D054597D00000E78000A405459700C8
:10AE50000000E78060EDA9B797B7FF1F938787F4DD
:10AE60009C47858BEDC71773FFFFE702032417B5D7
:10AE7000FF1F1305E5FA97B7FF1F23A507F297B742
:10AE8000FF1F23A307F297B7FF1F23A107F2972005
:10AE90000100E780208197500000E780E0F59710DF
:10AEA0000100E780A04C97100100E780A05297B7FF
:10AEB000FF1F9387A7ED9C4391C70545978000002E
:10AEC000E780402097B7FF1F938707D69C4399C719
:10AED00041657D1597700000E78040A297F0000063
:10AEE000E780E03D97D00000E780808F97B7FF1F95
:10AEF000938747009C43139717016356070097F009
:10AF00000000E78000AD97B7FF1F23A907F297B7AE
:10AF1000FF1F23A707F297B7FF1F23A507F297B7D5
:10AF2000FF1F23A307F297000000E780008C970023
:10AF30000000E780007297F0FFFFE780401897F06D
:10AF40000000E78040D61773FFFF67004318828038
:10AF500097B7FF1F938707E5884382801773FFFF2A
:10AF6000E702A31497800000E780607597800000D7
:10AF7000E780C0771773FFFF670063151773FFFF44
:10AF8000E70203112A849304140201112E85B28969
:10AF9000A685214636C63A8997300100E780403DB4
:10AFA0000DE9B24638082686CE85130594049750DD
:10AFB0000000E780604121462C084A859730010057
:10AFC000E780003B1335150005611773FFFF67002D
:10AFD000630F0145D5BF1773FFFFE702030D93050C
:10AFE000450617B5FF1F130525B997100100E78027
:10AFF00020691773FFFF6700830D1773FFFFE702D8
:10B00000C30A41112EC697F0FFFFE780601BB245CF
:10B0100088C141011773FFFF6700630B1773FFFFC0
:10B02000E7020307AA842E8497800000E780006C63
:10B03000AA898545228597000000E780E07D83C7C7
:10B04000E4011389940899E313890403CE852285CA
:10B0500097000000E780407C214693051902228575
:10B0600097000000E780607897B7FF1F938787D32A
:10B070008C43228597100000E780C082214693858B
:10B080008402228597000000E78020761773FFFF77
:10B09000670043031773FFFFE702A3FE397197F0C0
:10B0A0000000E780E0B49305400661E99780000066
:10B0B000E78000606302051497B7FF1F83C787AD61
:10B0C00013B7170097B6FF1F2386E6AC014499CF4C
:10B0D000C16417B9FF1F1309E9CC9309400EFD1491
:10B0E00097000000E780C0866342A40A97F0FFFF44
:10B0F000E780000D4169B7290900096AFD7A2A8BAA
:10B1000081447D199389F97B130A0A71938A8AC74E
:10B1100097000000E780C08363D7A4041304400EA7
:10B12000B387840217B7FF1F1307C7C70324070B92
:10B130003E948357C4016382270B18403307EB40CA
:10B1400063EAE900834744008507B3874703D6973E
:10B150006365F70801468145094597F0FFFFE780E1
:10B16000604EAA8B29E597400000E78080838547E1
:10B170006317F50689659385057117B5FF1F1305DC
:10B18000A59F97100100E780A04F95A0B307340357
:10B190000327090BBA9703D7C7016308970003C7B2
:10B1A0005700A38207002382E700050415BF93051B
:10B1B000C500228597000000E78080E65E85228634
:10B1C000976501009385C51A97F0FFFFE780E0526D
:10B1D0005E8597100000E780608A850415BF97B7E9
:10B1E000FF1F938727BC9C478D83858BC1F7216107
:10B1F0001773FFFF670063EC01468545094502D0E0
:10B2000002D202D402D697F0FFFFE780A043AA84BF
:10B2100079DD97F00000E780E09C1389C4002A8460
:10B2200081454A8597000000E780005F0C40414659
:10B230004A8597000000E780405B832944006385CE
:10B24000090C4E8502D802DA02DC02DE97300100DA
:10B25000E78060402ACE141005462C0808184ECC12
:10B2600097500000E780E00A1375F50F51ED835504
:10B27000840093E525004A8597000000E780E05EA2
:10B2800011460C104A8597000000E78000560146E1
:10B29000976501009385450E268597F0FFFFE780AF
:10B2A000C045268597000000E780407D5C40A1D323
:10B2B000014685450D4597F0FFFFE780A038AA8439
:10B2C0001DD548401389C40097300100E780A0389D
:10B2D0002AC64A8597000000E780404C3246636FDB
:10B2E000C5004C404A8597000000E78000500146A9
:10B2F0008145268597F0FFFFE7802040268597004F
:10B300000000E780A077E5B583558400ADB71773DB
:10B31000FFFFE70283D997B7FF1F9387A7A89C4732
:10B320001DC193E7870017B5FF1F1305E58417B705
:10B33000FF1F232DF7A697100100E78040321773F7
:10B34000FFFF6700C3D8DD9B17B7FF1F2320F7A6B9
:10B3500097300000E780E0647DF117B5FF1F13050B
:10B36000A58197100100E780E033D1BF1773FFFF7D
:10B37000E70223D14169AA892E8AB28A368BBA8B19
:10B38000814417BCFF1F130CECA1930C400E7D19D8
:10B3900097F0FFFFE780C05B63C4A40001443DA0B9
:10B3A0003384940383270C0B3E948357C401638634
:10B3B00027055A87D6865286CE8513050403970043
:10B3C0000000E780E0BB01C923800B0022851773D2
:10B3D000FFFF670083CE8347F40185C35A87D68673
:10B3E0005286CE851305940897000000E78040B987
:10B3F00009C585472380FB00D1BF850451BF835712
:10B4000045006380071E1773FFFFE70263C8011141
:10B410002A8497000000E780C04D09C98547630969
:10B42000F50605611773FFFF6700C3C997E00000C9
:10B43000E780007C7DF5835744004947ED9BE3920C
:10B44000E7FEC145228597000000E7804033AA84CB
:10B45000228597000000E780204F0357440002CE6A
:10B4600091472A89631AF700228597000000E78038
:10B47000A0513C082ACC3ECE97E00000E7808076C1
:10B480005C55C5D374084A86A6850545829751BF89
:10B4900003574400D147E3F6E7F8032A0400C169E3
:10B4A000014997BAFF1F938AEA8F130B400EFD19CB
:10B4B00097F0FFFFE780C049634FA90E2285032A5A
:10B4C000040097000000E780C042A1452A89228538
:10B4D00097000000E780A02AAA8422859700000038
:10B4E000E780804A14402A86AA8978082685CA857A
:10B4F00097000000E780C0E7AA8405D503C7F401E0
:10B5000089476315F7008347C10181DF5546D2851E
:10B510001385640097300100E780E0E701459780DC
:10B520000000E780C01901C583D7C401A5E797B71C
:10B53000FF1F938727879C4793551900858913D749
:10B540003700058B01CF8983858B6399B70001454F
:10B550002EC697000000E780C0DBB2454E8597807D
:10B560000000E780601F0346C1012A84937519001B
:10B57000268597900000E780E03935C126859780C1
:10B580000000E780E018268511C001459780000083
:10B59000E780004C97300000E780A0408547E31229
:10B5A000F5E883C754001307F00FE38CE7E685073F
:10B5B000A382F400BDB5B304690383A70A0BBE944C
:10B5C00083D7C401638B37015546D2851385640048
:10B5D00097300100E780C0D955DD0509D1BD5DD8A0
:10B5E0006DB782801773FFFFE70283AA9780000080
:10B5F000E780000C05C1C164014417A9FF1F1309AE
:10B60000697A9309400EFD1497F0FFFFE7804034FC
:10B61000634EA40017A5FF1F1305055697100100E0
:10B62000E780E0031773FFFF6700C3A93305340306
:10B630008327090B3E958357C50163889700231222
:10B64000050097800000E780A00C050475BF97A750
:10B65000FF1F938727759C478D83858B8DE3177319
:10B66000FFFFE70283A417A5FF1F1305E5509710FE
:10B670000100E78020031773FFFF670043A5828066
:10B680001773FFFFE70263A2970500009385C5A02B
:10B6900017A5FF1F1305454E97100100E78020EE08
:10B6A0001773FFFF6700A3A21773FFFFE702E39F73
:10B6B0008841B7E70400BC5B0505420541818297DC
:10B6C00009C585472300F50005051773FFFF6700CF
:10B6D00003A083C7F5FF2E858507A38FF5FE828023
:10B6E00083C7F5FFFD1793F7F70FA38FF5FE99EFCB
:10B6F0001773FFFFE702639BB7E70400BC5713858E
:10B70000F5FF82971773FFFF6700639C82801C41DF
:10B71000035745008D8FBA951CC12312B5003E8595
:10B72000828093D78500A2051441DD8D83574500A3
:10B730001387E6FF18C189072312F50013D6850089
:10B740004111238FB6FEA38FC6FE410182801841AE
:10B750009307F7FF1CC18357450085072312F500A7
:10B76000A30FB7FE8280835745008D8F2312F5000B
:10B770001C41BE950CC12E858280AA8703D7470045
:10B7800008410D8FAA952392E7008CC3828018414F
:10B7900008453305A740828083574500035765005D
:10B7A0001D8F1C4108453385A7403305A740828083
:10B7B0001773FFFFE702638F41112EC62A8497009B
:10B7C0000000E780A0FDB2456373B50001A0835778
:10B7D00044000840BE952312B4003E954101177302
:10B7E000FFFF6700C38E1773FFFFE702038C411151
:10B7F0002E84B28532C697000000E780A0FB324657
:10B80000A28597300100E78000B941011773FFFF5F
:10B810006700E38B1773FFFFE70223892E848545BA
:10B8200097000000E78000F9230085001773FFFFF1
:10B830006700E3891773FFFFE7022387411123178E
:10B84000B100894597000000E780C0F68347E1001A
:10B850002300F5008347F100A300F50041011773B1
:10B86000FFFF6700C3861773FFFFE702038493D7C8
:10B870008500A2054111DD8D2317B1008945970090
:10B880000000E78020F38347E1002300F5008347B1
:10B89000F100A300F50041011773FFFF6700238348
:10B8A0001773FFFFE70263801397850193D7850124
:10B8B000C166938606F0D98F13D78500758FD98F0F
:10B8C000A2053707FF00F98D4111DD8D2EC6914588
:10B8D00097000000E78000EE6C00114697300100F1
:10B8E000E78060AB41011763FFFF6700437E17638A
:10B8F000FFFFE702837B1C41854503C407009700D7
:10B900000000E78080E622851763FFFF6700237C45
:10B910001763FFFFE70263791C414111894503C7A3
:10B92000070083C717002307E100A307F100970072
:10B930000000E78080E30355E10041011763FFFF4A
:10B940006700E3781763FFFFE70223761C4141118C
:10B95000894503C7070083C717002307E100A30732
:10B96000F10097000000E78040E08357E1004101CB
:10B9700013D58700A2075D8D420541811763FFFF44
:10B980006700E3741763FFFFE70223720C41411164
:10B990002A841146680097300100E780C09F9145D6
:10B9A000228597000000E78040DCB247C16693869D
:10B9B00006F01397870113D58701598D13D7870098
:10B9C000758F598DA2073707FF00F98F5D8D4101F3
:10B9D0001763FFFF6700A36F1C45BE950CC18280F3
:10B9E000AE87944391E6584101EF0CC15CC182805F
:10B9F00003C7570013671700A382E700B687D5B7C0
:10BA00000CC3EDB7AA87084119CD1841D44398C398
:10BA10006313D500D8C32A870346570093761600D0
:10BA200081E6232007008280944381CA8C4203A8C8
:10BA300047008CC363930601CCC3799A14C3A30255
:10BA4000C7003687D1BF1C45DC471D8DB777DBB6F5
:10BA5000938777DB09853305F502420541818280B2
:10BA6000F147B385F50248452E958280834745000E
:10BA700085072302F50082801763FFFFE702E36278
:10BA80002A8409E41763FFFF670063648347440067
:10BA9000F5DBFD1793F7F70F2302F400E5F71C44DD
:10BAA00003D7270005072391E700DC4399C32285CC
:10BAB00082974C4889CD83475400898B99E71C4471
:10BAC00022859C479C439C478297232A0400004080
:10BAD000232004007DB71763FFFFE702035D835750
:10BAE000250041112EC681EB0144228541011763D7
:10BAF000FFFF6700C35D035705008147F146E3057B
:10BB0000F7FEB385D702404585072E948345440050
:10BB100008C4F5F5B247AA8481E7232A040009A8DE
:10BB20001C456C0022859C439C43829748C84DDD90
:10BB300085472312F400B247232004002318040091
:10BB40002319F4005C485CC483D72400FD172391BB
:10BB5000F40061BF1763FFFFE702235597A7FF1F9C
:10BB60009387870388432326050023240500410586
:10BB700097100100E78000B31763FFFF67002355AC
:10BB80001763FFFFE702635217A4FF1F1304C400EB
:10BB90001C40411199CF9C472300B5002AC65CC1C7
:10BBA00097000000E78040FB1C40DC4399C332450E
:10BBB000829741011763FFFF670063510347450008
:10BBC00029E3584DAA877D551DCF1763FFFFE70274
:10BBD000C34D1CC3DC4797A6FF1F23AFE6FAF156FF
:10BBE000130507012390D7009705000093850502F0
:10BBF00097100100E780A09801451763FFFF6700D9
:10BC0000034D7D55828082801763FFFFE702E34981
:10BC100001116146814528009760FFFFE780E04BF6
:10BC200097A7FF1F938747F79C4328009305F00FC2
:10BC3000DC473EC697000000E780C0F4056117634B
:10BC4000FFFF6700C34897A7FF1F9387E7F49C4354
:10BC5000D847A1679387C702631EF70A397106DECA
:10BC600022DC26DA80004AD84ED652D456D232850B
:10BC7000B28497000000E780C0C7AA892685970094
:10BC80000000E78020C92318A4FC26859700000047
:10BC9000E78040C82319A4FC268597000000E780B0
:10BCA00060C783D744000A8A231AA4FC858393F7CC
:10BCB000F70F230EF4FC8607BD0793F7073F330108
:10BCC000F1408A8A01498347C4FD6367F902CE8542
:10BCD000130584FC232C54FD97000000E78080EAC4
:10BCE0005281130104FCF2506254D2544259B259A9
:10BCF000225A925A21618280268597000000E780AF
:10BD000060C193171900D69705092390A7001379EE
:10BD1000F90F55BF828097A7FF1F9387E7E79C43E2
:10BD2000D847A1679387A702631AF70A397106DE1D
:10BD300022DC26DA80004AD84ED652D456D232853A
:10BD4000B28497000000E780C0BAAA8926859700D0
:10BD50000000E78020BCFD572318A4FC268523198A
:10BD6000F4FC97000000E780E0BA83D744000A8A19
:10BD7000231AA4FC858393F7F70F230EF4FC8607A0
:10BD8000BD0793F7073F3301F1408A8A0149834792
:10BD9000C4FD6367F902CE85130584FC232C54FD92
:10BDA00097000000E78000DE5281130104FCF2508E
:10BDB0006254D2544259B259225A925A2161828015
:10BDC000268597000000E780E0B493171900D69706
:10BDD00005092390A7001379F90F55BF828097A713
:10BDE000FF1F938767DB9C43D847A16789076310D0
:10BDF000F70A397106DE22DC26DA80004AD84ED6F0
:10BE000052D456D23285328997000000E78060AE66
:10BE1000AA894A8597000000E780C0AF8357490090
:10BE20000A8A2318A4FC858393F7F70F230CF4FCEC
:10BE30008607BD0793F7073F3301F1408A8A8144A3
:10BE4000834784FD63E7F402CE85130584FC232A2F
:10BE500054FD97000000E780E0D25281130104FCFA
:10BE6000F2506254D2544259B259225A925A216124
:10BE700082804A8597000000E780C0A9939714004C
:10BE8000D69785042390A70093F4F40F55BF8280C2
:10BE900097A7FF1F938747D09C43D847A1679387F5
:10BEA000E704631EF70A397106DE22DC26DA800019
:10BEB0004AD84ED652D456D23285B284970000006A
:10BEC000E78020A3AA89268597000000E78080A448
:10BED0002318A4FC268597000000E780A0A3231A5E
:10BEE000A4FC268597000000E780C0A283D7440009
:10BEF0000A8A2319A4FC858393F7F70F230EF4FC19
:10BF00008607BD0793F7073F3301F1408A8A01494D
:10BF10008347C4FD6367F902CE85130584FC232C97
:10BF200054FD97000000E780E0C55281130104FC36
:10BF3000F2506254D2544259B259225A925A216153
:10BF40008280268597000000E780C09C9317190027
:10BF5000D69705092390A7001379F90F55BF828062
:10BF600097A7FF1F938747C39C43D847A167938731
:10BF7000C704631AF70A397106DE22DC26DA80006C
:10BF80004AD84ED652D456D23285B2849700000099
:10BF9000E7802096AA89268597000000E780809791
:10BFA000FD572318A4FC2685231AF4FC97000000F3
:10BFB000E780409683D744000A8A2319A4FC85832E
:10BFC00093F7F70F230EF4FC8607BD0793F7073F9F
:10BFD0003301F1408A8A01498347C4FD6367F9024E
:10BFE000CE85130584FC232C54FD97000000E780C8
:10BFF00060B95281130104FCF2506254D254425988
:10C00000B259225A925A21618280268597000000F7
:10C01000E780409093171900D69705092390A70051
:10C020001379F90F55BF828097A7FF1F9387C7B673
:10C030009C43D847A167DD076317F7041763FFFF29
:10C04000E702A30679713285328497000000E78009
:10C05000408A2AC6228597000000E780A08B231122
:10C06000A102228597000000E780A088B245230046
:10C07000A102280897000000E780C0B0456117635F
:10C08000FFFF6700C304828097A7FF1F9387C7B095
:10C090009C43D847A167938787046317F704176306
:10C0A000FFFFE70283007971328532849700000038
:10C0B000E78020842AC6228597000000E7808085DB
:10C0C0002311A102228597000000E7808082B245FB
:10C0D0002300A102280897000000E780A0AA45617C
:10C0E0001763FFFF6700A3FE828097A7FF1F938758
:10C0F000A7AA9C43D847A1679387A7046312F702B6
:10C100001763FFFFE70263FA0111280081459700DA
:10C110000000E78020A705611763FFFF670023FB8E
:10C12000828097A7FF1F938727A79C43D847A167C3
:10C13000938757026319F7021763FFFFE702E3F6DD
:10C140000111328597F0FFFFE780A07A2308A10054
:10C150008145280097000000E780C0A205611763B1
:10C16000FFFF6700C3F6828097A7FF1F9387C7A2D0
:10C170009C43D847A1679387E702631BF7041763C3
:10C18000FFFFE70283F201113285328497F0FFFF4F
:10C19000E7804078AA84228597F0FFFFE7808077C8
:10C1A000854709E9228597F0FFFFE7808074420503
:10C1B000B337A00028008145231891003ECA97009C
:10C1C0000000E780209C05611763FFFF670023F0F4
:10C1D000828097A7FF1F9387279C9C43D847994746
:10C1E0006313F7081763FFFFE70223EC79713285C9
:10C1F000328497F0FFFFE780C06F2AC6228597F050
:10C20000FFFFE78020712310A102228597F0FFFF36
:10C21000E780206E2301A102228597F0FFFFE780CF
:10C22000406DA301A102228597F0FFFFE780606CBB
:10C230002302A102228597F0FFFFE780806B231382
:10C24000A102228597F0FFFFE780A06AB245231480
:10C25000A102280897000000E780C092456117639B
:10C26000FFFF6700C3E6828097A7FF1F9387C792EF
:10C270009C43D847A1679387C7036313F7081763E5
:10C28000FFFFE70283E279713285328497F0FFFF86
:10C29000E78020662AC6228597F0FFFFE780806747
:10C2A0002310A102228597F0FFFFE780A0662311EB
:10C2B000A102228597F0FFFFE780A0632302A1027D
:10C2C000228597F0FFFFE780C062A302A1022285CA
:10C2D00097F0FFFFE780E0612303A102228597F03A
:10C2E000FFFFE7800061B245A303A1022808970081
:10C2F0000000E780208945611763FFFF670023DDA9
:10C3000082801763FFFFE70243DA01112A8497F066
:10C31000FFFFE780005EAA84228597F0FFFFE78099
:10C32000605F228597F0FFFFE780C05E03574400FF
:10C330008D4763F7E700228597F0FFFFE780805D78
:10C34000228597F0FFFFE780E05C2800A685970034
:10C350000000E780208305611763FFFF670023D794
:10C3600097A7FF1F938747839C43D847A167FD0783
:10C37000631FF7001763FFFFE70223D3328597009F
:10C380000000E78040F81763FFFF670043D4828016
:10C3900097A7FF1F938747809C43D847A167E5076E
:10C3A0006315F7081763FFFFE70223D07971328521
:10C3B000328497F0FFFFE780C0532AC6228597F0AA
:10C3C000FFFFE7802055228597F0FFFFE78080542C
:10C3D0002310A102228597F0FFFFE780A0535205AA
:10C3E00051812311A10222852302010297F0FFFF50
:10C3F000E7802050A302A102228597F0FFFFE7808B
:10C40000404F2303A102228597F0FFFFE780604E93
:10C41000B245A303A102280897F0FFFFE7808076CA
:10C4200045611763FFFF670083CA82809797FF1FEC
:10C43000938787769C43D847A1679387E703631F59
:10C44000F7001763FFFFE70243C63285970000003D
:10C45000E78060EB1763FFFF670063C782809797F1
:10C46000FF1F938767739C43D847A167938747044F
:10C47000631EF7021763FFFFE70223C3797132855A
:10C48000328497F0FFFFE780C0462AC6228597F0E6
:10C49000FFFFE7802048B245280897F0FFFFE780BC
:10C4A000606E45611763FFFF670063C282809797E4
:10C4B000FF1F9387676E9C43D847A16793878702C6
:10C4C0006310F7041763FFFFE70223BE797132851B
:10C4D000328497F0FFFFE780C0412AC6228597F09B
:10C4E000FFFFE7800041B2452300A102280897F032
:10C4F000FFFFE780206945611763FFFF670023BDE9
:10C5000082801763FFFFE70243BA011197F0FFFF34
:10C51000E780203EAA85280097F0FFFFE78080662D
:10C5200005611763FFFF670083BA9797FF1F938723
:10C53000A7669C43D847A167D107631FF70017631D
:10C54000FFFFE70283B6328597000000E780A0FB7B
:10C550001763FFFF6700A3B782809797FF1F93873A
:10C56000A7639C43D847A167C507631FF7001763FC
:10C57000FFFFE70283B3328597000000E780A0F851
:10C580001763FFFF6700A3B482809797FF1F93870D
:10C59000A7609C43D847A167B907631FF7001763DB
:10C5A000FFFFE70283B0328597000000E780A0F527
:10C5B0001763FFFF6700A3B182809797FF1F9387E0
:10C5C000A75D9C43D847A167AD07631FF7001763BA
:10C5D000FFFFE70283AD328597000000E780A0F2FD
:10C5E0001763FFFF6700A3AE82809797FF1F9387B3
:10C5F000A75A9C43D84789476318F7021763FFFF80
:10C60000E702A3AA0111328532C897F0FFFFE78045
:10C61000402EAA85280097F0FFFFE780A05605610D
:10C620001763FFFF6700A3AA82809797FF1F938776
:10C63000A7569C43D847A1678D076311F70417637A
:10C64000FFFFE70283A601113285328497F0FFFFD6
:10C65000E780202A13066100AA844C0022859730C7
:10C660000000E780C0232800A68597F0FFFFE78041
:10C67000605105611763FFFF670063A5828097978C
:10C68000FF1F9387A7519C4381CFDC4391CB176356
:10C69000FFFFE70283A182971763FFFF670023A3D1
:10C6A00082801763FFFFE70243A079713C08AE84E4
:10C6B0003ED2A165B7070A002A843ED448103C0840
:10C6C000DD053ED636C432C63AC297D0FFFFE780BA
:10C6D000E02F12474810BA8597F0FFFFE780C0139C
:10C6E00032464810B28597F0FFFFE780E014A2467B
:10C6F0004810B68597F0FFFFE78000125010014701
:10C700008146A685228597D0FFFFE780805145614D
:10C710001763FFFF6700A39B1763FFFFE702E39820
:10C7200001117C000329C501AE843ECAA165B7078B
:10C7300007002A843ECC48087C00C5053ECE97D031
:10C74000FFFFE780A0288345D900480897F0FFFF46
:10C75000E780800C500801478146A685228597D046
:10C76000FFFFE780004C05611763FFFF670023961A
:10C770001763FFFFE702639383C7950093F7F707FB
:10C78000A384F50097000000E78040F91763FFFFDE
:10C790006700E3931763FFFFE702239179713C0879
:10C7A000AE843ED2A165B70709002A843ED4481062
:10C7B0003C08938545043ED632C636C497D0FFFF69
:10C7C000E780C020A2464810B68597F0FFFFE780BB
:10C7D000A00432464810B28597F0FFFFE780C005FD
:10C7E000501001478146A685228597D0FFFFE7803C
:10C7F000404345611763FFFF6700638D1763FFFFC9
:10C80000E702A38A83C7950041112A8493F7F707AB
:10C81000A384F50032852EC697F0FFFFE780800FD6
:10C8200085672AC46370F50297700000E78020E9ED
:10C830002246B24509ED1147814622859700000046
:10C84000E78060E641011763FFFF67004388014707
:10C850008346F501DDB71763FFFFE702638301112C
:10C860003C003ECAB7070A003ECC3C003ECE83C720
:10C870009500AA89328593F7F707A384F5002E84E3
:10C8800097F0FFFFE78000098567637DF504A165E8
:10C89000AA8493858504480897D0FFFFE78000139A
:10C8A000268597700000E78080E12A8929E191457B
:10C8B000480897F0FFFFE78020F6A685480897F024
:10C8C000FFFFE78060F7CA85480897F0FFFFE78021
:10C8D000A0F4014781465008A2854E8597D0FFFFFE
:10C8E000E780203405611753FFFF6700A37D814572
:10C8F000480897F0FFFFE78020F20349090275BF5F
:10C900001753FFFFE702C37879711C103ECAB707BF
:10C910000F003ECC404D1C10AA84AE8948089945B2
:10C9200032C636893ECE97D0FFFFE780200A3246D6
:10C930004808B28597F0FFFFE78000EE630C09021C
:10C94000A545480897F0FFFFE780C0E62546CA8561
:10C9500097200100E78020A4500801478146CE853A
:10C96000268597D0FFFFE780C02B45611753FFFF57
:10C97000670043758355C402480897F0FFFFE780BE
:10C98000A0EB0355E402814505C585478545630154
:10C99000F502C167FD179305F00F630BF5007D15D8
:10C9A00097700000E780208E9305150093F5F50F32
:10C9B000480897F0FFFFE78020E683450403480816
:10C9C00097F0FFFFE78040E583451403480897F0A0
:10C9D000FFFFE78060E483552403480897F0FFFFDA
:10C9E000E78080E583554403480897F0FFFFE78020
:10C9F000A0E49DB71753FFFFE702236B83C79500A1
:10CA00008146014693F7F707A384F50097000000DD
:10CA1000E78040EF1753FFFF6700636B1753FFFF7B
:10CA2000E702A36879713E841C103ECA2E89B707BD
:10CA30000F00A1653ECCFD051C10AA84480842C029
:10CA40003AC23ECE36C432C697D0FFFFE78000F828
:10CA500032464808B28597F0FFFFE780E0DBA24648
:10CA60004808B68597F0FFFFE78000DD12474808C9
:10CA7000BA8597F0FFFFE78020DC0248630C0802CC
:10CA80009145480897F0FFFFE780C0D21146A28584
:10CA900097200100E7802090500801478146CA8511
:10CAA000268597D0FFFFE780C01745611753FFFF2A
:10CAB0006700E3618945480897F0FFFFE78080CF72
:10CAC000834704002300F50083471400A300F5000A
:10CAD000E1B71753FFFFE702A35B83C7950001117E
:10CAE0002A8A93F7F707A384F5003285AE8432C60D
:10CAF00097F0FFFFE78000E232462A89328597F0FF
:10CB0000FFFFE78000DF85676373F902AA894A8522
:10CB100097700000E780A0BA2A8419ED114781467A
:10CB20004A86A685528597000000E780C0B7056158
:10CB30001753FFFF670003599387E9FF93F7F70F38
:10CB40000547E366F7FE8347F50195EB8947E380E8
:10CB5000F9FE8346F401528501474A86A68597006F
:10CB60000000E78040B4A167D90748083ECC230AFB
:10CB7000010002CE97000000E780A0B04DBF639E89
:10CB8000E7008947639EF90093071020231FF500F3
:10CB900097700000E780C0B76DBF0947E39BE7FAD5
:10CBA0008D47E398F9FA228597700000E78080DFCF
:10CBB0009797FF1F9387871D9C4399E79797FF1FC0
:10CBC000938787069C4399C703D50400978000008C
:10CBD000E780A0CE231F040022855DBF1753FFFF0F
:10CBE000E702A34C01113C003ECAB7070B003ECC44
:10CBF0003C003ECE83C795002A89328593F7F7071C
:10CC0000A384F500AE8497F0FFFFE780A0D09317D0
:10CC10000501C187635AF006A1652A849385E50260
:10CC2000480897D0FFFFE78060DAA285480897F0B0
:10CC3000FFFFE78060C09797FF1F9387E7FE9C4345
:10CC4000A9EB01449375F40F480897F0FFFFE780C4
:10CC5000A0BC9355844093F5F50F480897F0FFFF6B
:10CC6000E78080BB9355044193F5F50F480897F092
:10CC7000FFFFE78060BA014781465008A6854A85D4
:10CC800097D0FFFFE780E0F905611753FFFF6700CA
:10CC90000344416585460546A2857D1597500000F1
:10CCA000E78060BD59DD510597000100E780808F66
:10CCB000130440063344850271B71753FFFFE702A0
:10CCC000C33E0111B70706003EC683C79500216425
:10CCD0002A8993F7F707A384F500AE84280093050B
:10CCE000A4040AC40AC897D0FFFFE78020CE300012
:10CCF00001478146A6854A8597D0FFFFE78060F20D
:10CD000097E0FFFFE780801513049404480822CCC5
:10CD1000230A010002CE97000000E780809605619B
:10CD20001753FFFF6700A33A1753FFFFE70243368D
:10CD3000C1642A8901449799FF1F9389A906130AA0
:10CD40008002FD1497E0FFFFE78080C16347A400E5
:10CD500001451753FFFF6700E336B307440303A7FA
:10CD6000C90ABA9703D707006306970083D727003D
:10CD7000638427010504F9B70545E1BF1753FFFF99
:10CD8000E70203312A8A2E8999C123A0050081492F
:10CD90008144979AFF1F938AAAE0614B97E0FFFFB7
:10CDA000E78040C263C7A4004E851753FFFF6700AA
:10CDB00063313384640383A70A003E9483570400DD
:10CDC00099E763040900232089008504C1BF414617
:10CDD000D2851305440097100100E780605975F56E
:10CDE000A289E5B71753FFFFE702832A39717C0850
:10CDF0003ED4B7070A003ED67C083ED883C79500CC
:10CE00002A8A328593F7F707A384F5002E8932C664
:10CE100097F0FFFFE78000B085676373F50832463F
:10CE2000AA84328597F0FFFFE780A0AC8547AA89E6
:10CE300063E8A706A16593858504281097D0FFFFB6
:10CE4000E780C0B8268597700000E78040872A8475
:10CE500029ED9145281097F0FFFFE780E09BA6851C
:10CE6000281097F0FFFFE780209DCE85281097F0CF
:10CE7000FFFFE780609A014781463010CA855285DE
:10CE800097D0FFFFE780E0D9A16793877704481820
:10CE90003EDC230A010202DE97F0FFFFE780607E9E
:10CEA00021611753FFFF6700E3218145281097F0A8
:10CEB000FFFFE7806096A685281097F0FFFFE780C8
:10CEC000A0979797FF1F9387A7249C4381CB228528
:10CED0006389090097D00000E7804024834504025D
:10CEE00071B797D00000E780C022CDBF1753FFFF76
:10CEF000E702031A83C795004111AA8993F7F70740
:10CF0000A384F5003285AE84328A97F0FFFFE78074
:10CF100060A08567637FF5022A8997600000E7803B
:10CF2000007A2A84914631C58347F5010547638716
:10CF3000E70291C70D476366F704AD461DA8930548
:10CF4000050303250A00414697100100E78040428F
:10CF50000DE941011753FFFF6700C31693059508BC
:10CF600003250A00414697100100E7806040814692
:10CF700069F54A86A6854E8597000000E780C08146
:10CF8000C9BF83250A001305940897700000E78045
:10CF9000A02919C1C146F1BF9797FF1F938707DFEB
:10CFA0009C4399E79797FF1F938707C89C4399C7AE
:10CFB000228597800000E780208A69FD8547A30FBE
:10CFC000F400228597B00000E78060842285976096
:10CFD0000000E780E0734E8581464A86A68597F07B
:10CFE000FFFFE780607BA1679387570448003EC43A
:10CFF0002302010002C697F0FFFFE780806891BF1F
:10D000001753FFFFE702E30783C795004111AA8981
:10D0100093F7F707A384F50032852E89B28A97F03B
:10D02000FFFFE780208F85676374F50EAA84976001
:10D030000000E780C0682A840DED416B014A979B90
:10D04000FF1F938B2BD6130C400E7D1B19A83304A6
:10D050008A0383A70B0B3E948357C4016383670540
:10D06000050A97E0FFFFE780A08EE342AAFE9546FF
:10D070000DA08357C501639697029305050303A589
:10D080000A00414697100100E780802E994611E181
:10D0900081462686CA854E8597F0FFFFE780C06FE0
:10D0A00085A883A50A001305040397700000E78094
:10D0B000A017C14679FD2285231E940097A0000089
:10D0C000E780E074228597600000E78060649797AE
:10D0D000FF1F9387E7039C43A9C323000402228513
:10D0E00097D00000E78040F04E8581462686CA85AD
:10D0F00097F0FFFFE780406AA16793870704480025
:10D100003EC42302010002C697F0FFFFE78060578C
:10D1100041011753FFFF670043FA89472300F402D8
:10D12000E1B7397106DE22DC4AD8800052D456D2EB
:10D130005AD026DA4ED65ECE2E8A32892A8B97D0E6
:10D14000FFFFE780E07D0605710541998A8A33017A
:10D15000A140232224FC231404FC97D0FFFFE78086
:10D16000207C83479A000605350593F7F7072315BA
:10D17000A4FCA304FA004A85232624FC97E0FFFFC1
:10D18000E780407993170501C1876340F00256811B
:10D19000130104FCF2506254D2544259B259225A3B
:10D1A000925A025BF24B21618280AA844A8597E001
:10D1B000FFFFE7802076AA894A8597E0FFFFE78096
:10D1C0006075A1659385C5022A89130544FC97C043
:10D1D000FFFFE780A07F268597C0FFFFE780E07311
:10D1E000854511C94A86CE8597C0FFFFE780606DEF
:10D1F000AA8B21E98945130544FC97E0FFFFE780EE
:10D20000A061A685130544FC97E0FFFFE780C0629C
:10D21000CE85130544FC97E0FFFFE780E061CA85F7
:10D22000130544FC97E0FFFFE7800061014781465A
:10D23000130644FCD2855A8597D0FFFFE780609E95
:10D24000B9B78145130544FC97E0FFFFE780C05C58
:10D25000A685130544FC97E0FFFFE780E05DCE85DF
:10D26000130544FC97E0FFFFE780005DCA851305C6
:10D2700044FC97E0FFFFE780205C814497D0FFFFEC
:10D28000E780006AE3D4A4FA83A70B011397140084
:10D29000BA9783D5070099C5130544FC97E0FFFFB3
:10D2A000E78080598504D9BF797106D622D44AD047
:10D2B00000184ECE52CC56CA26D25AC8AE893289F0
:10D2C000AA8A97D0FFFFE780A06506056905419906
:10D2D0000A8A3301A140232A24FC231C04FC97D092
:10D2E000FFFFE780E06383C7990006052D0593F7EC
:10D2F000F707231DA4FCA384F9004A85232E24FCF0
:10D3000097E0FFFFE780006193170501C187634F36
:10D31000F0005281130104FDB2502254925402597C
:10D32000F249624AD24A424B45618280AA844A85C8
:10D3300097E0FFFFE780005EA1659385A5022A893B
:10D34000130544FD97C0FFFFE7804068268597C01E
:10D35000FFFFE780805C854509C9CA8597C0FFFF4C
:10D36000E78020592A8B29E18945130544FD97E080
:10D37000FFFFE780604AA685130544FD97E0FFFFA5
:10D38000E780804BCA85130544FD97E0FFFFE780E7
:10D39000A04A01478146130644FDCE85568597D0A5
:10D3A000FFFFE7800088B5B78145130544FD97E08E
:10D3B000FFFFE7806046A685130544FD97E0FFFF69
:10D3C000E7808047CA85130544FD97E0FFFFE780AB
:10D3D000A046814497D0FFFFE7808054E3DBA4FAA6
:10D3E00083270B0113971400BA9783D5070099C5BB
:10D3F000130544FD97E0FFFFE78000448504D9BF93
:10D400001753FFFFE70263CA83474500404DD5EF3E
:10D41000FD575DC48346940009476363D70A0346FA
:10D42000B400854663EEC6088306E40063CA0608B6
:10D430005C45F9562390D7009787FF1F83C78776EF
:10D4400099E3A304E4009787FF1F9387E77D9C433C
:10D4500081E78947A306F4009797FF1F938747CB7F
:10D460009C4381E789472306F400970500009385D4
:10D470004506AA841305040197F00000E7802010F8
:10D48000FD57231AF40281471CDC01489787FF1FD0
:10D4900023A687709787FF1F93878770232E040327
:10D4A00004C0804397D0FFFFE780C0516146330638
:10D4B000C502814522859750FFFFE78000C2814762
:10D4C0003E851753FFFF670083C0FD57D5BF175335
:10D4D000FFFFE70283BD2A840355450297600000E1
:10D4E000E780E01D19E5231E04001753FFFF6700C6
:10D4F00003BE8357E401F5DB930504FF17450100E4
:10D500001305452197E00000E780E014F9BF1753A9
:10D51000FFFFE70283B92E89A16541119385E503D9
:10D520002A8436C432C6BE843AC297C0FFFFE78061
:10D53000E04912472285BA8597E0FFFFE780C02DBA
:10D5400032462285B28597E0FFFFE780E02EA246B3
:10D550002285B68597E0FFFFE780002E630309026E
:10D560009145228597E0FFFFE780C0241146A685FC
:10D5700097100100E78020E241011753FFFF670089
:10D5800003B58945228597E0FFFFE780A02283C786
:10D5900004002300F50083C71400A300F500E9BFD1
:10D5A0001753FFFFE70263B083C79500444D05475B
:10D5B00093F7F707A384F5001C42411183C70700C6
:10D5C0006367F7062E842A89B1C003C7D400630FAE
:10D5D000F7021787FF1F13072765184305C3A386A4
:10D5E000F40097A00000E780404A83C7D40099E781
:10D5F00041657D1597400000E780403083D72403C4
:10D60000918B89C797E00000E780C0134A85A28507
:10D6100097F0FFFFE7808010A167C10748003EC474
:10D620002302010002C697F0FFFFE7808005410159
:10D630001753FFFF6700A3A91753FFFFE702E3A6F5
:10D6400003D745008D47AA8441112E8432892E8547
:10D6500063E3E70297E0FFFFE780C02BAA85230082
:10D660000900268597C0FFFFE780A02841011753D6
:10D67000FFFF6700C3A597E0FFFFE780A0292AC648
:10D68000228597E0FFFFE780E028B24585472A869C
:10D690002300F900268597C0FFFFE7808022F9B7B5
:10D6A000397106DE22DC26DA80004ED652D456D2FC
:10D6B0004AD85AD05ECEAE89B284AA8A97D0FFFFEC
:10D6C000E780002506051305250241990A8A3301E2
:10D6D000A140232224FC231404FC97D0FFFFE78001
:10D6E000202383C7990006054D0593F7F7072315F7
:10D6F000A4FCA384F9002685232624FC97E0FFFFE1
:10D70000E780402193170501C1876340F0025281F1
:10D71000130104FCF2506254D2544259B259225AB5
:10D72000925A025BF24B21618280AA8B03AB040008
:10D7300097C0FFFFE780601E51E583D74400014991
:10D740008544F11793B71700A301F4FC834734FC19
:10D75000A165C9C79385E504130544FC97C0FFFF85
:10D76000E780C026A685130544FC97E0FFFFE7800D
:10D77000A00ADE85130544FC97E0FFFFE780C00B9D
:10D78000834734FC114691E30946DA85130544FCCE
:10D7900097E0FFFFE78060058144630A0900416B61
:10D7A0007D1B97D0FFFFE780A01663CCA402014742
:10D7B0008146130644FCCE85568597C0FFFFE7805F
:10D7C0004046B1B7A685130634FC97000000E780F9
:10D7D000E0E6933415002A8986048DBF9385C5043D
:10D7E000A5BF8327C90013971400BA9783D50700F4
:10D7F00063886501130544FC97E0FFFFE780C003E1
:10D80000850445B71753FFFFE702A38779711C1002
:10D810003EC4B7070F003EC61C103EC883C7950024
:10D82000AA8A328593F7F707A384F500AE8932847C
:10D8300097E0FFFFE780000E93170501C187635A49
:10D84000F0062A8A228597E0FFFFE780A00C2A894C
:10D850005285032B040097C0FFFFE780000C39EDD1
:10D860008357440081440544F11793B71700A3037D
:10D87000F10083457100DA872287CA865286280024
:10D8800097000000E780E0C8014781463000CE8560
:10D89000568597C0FFFFE780C038A1679387D703FD
:10D8A00048083ECC230A810026CE97F0FFFFE78090
:10D8B00040DD45611753FFFF67002380A2851306F3
:10D8C000710097000000E78060D7AA84094455D111
:10D8D0003544E30055FB4A8597F0FFFFE78000459C
:10D8E0000D4441D9014497D0FFFFE7806002634DAA
:10D8F000A400C16B0144FD1B97D0FFFFE7804001EE
:10D90000634EA4001544B5B7DC4413171400BA974E
:10D9100083D70700638327030504F1B7D84493171F
:10D920001400BA9703D70700631B770123902701E0
:10D93000268597A00000E78080DB01441DBF050419
:10D9400065BF1743FFFFE702A37483C7950041112A
:10D950002A8A93F7F707A384F50032852E8932844B
:10D9600097E0FFFFE78000FB93170501C187635332
:10D97000F006AA89228597E0FFFFE780A0F923112E
:10D98000A1004E85832A040097C0FFFFE780E0F8DE
:10D9900039E58357440085440144F11793B71700D4
:10D9A000A300F1000348110003572100D6875285D8
:10D9B000CE862686CA8597F0FFFFE7806006A167BE
:10D9C000F10748003EC42302910022C697F0FFFFF2
:10D9D000E78020CB41011743FFFF6700A36EA285BC
:10D9E0001306110097000000E78040C52A8489448F
:10D9F00055D98357210011678544BA97C20711672B
:10DA0000C1831307F7EFE36FF7F89787FF1F93873B
:10DA1000E7379C4381CB85451305210097500000D3
:10DA2000E7802075835521002285814497C0FFFF40
:10DA3000E78040E525D923100500228597A0000046
:10DA4000E78040CD85B71743FFFFE702836383C7B5
:10DA5000950041112A8B93F7F707A384F5003285CF
:10DA60002E8A328497E0FFFFE780C0EA9317050112
:10DA7000C1876351F006AA8A228597E0FFFFE780FD
:10DA800060E92A895685832B040097C0FFFFE78051
:10DA9000C0E831E58357440081440544F11793B74A
:10DAA0001700A301F10003483100DE875A854A8739
:10DAB000D6862286D28597F0FFFFE78060F6A167C1
:10DAC000ED0748003EC42302810026C697F0FFFF01
:10DAD000E78020BB41011743FFFF6700035EA2857B
:10DAE0001306310097000000E78040B5AA8409447E
:10DAF0005DD99167CA97C2071167C1831307F7EF12
:10DB00000544E362F7FACA8597C0FFFFE78080D734
:10DB1000014451F9814997D0FFFFE78060E063DB62
:10DB2000A900984893971900BA9703D7070005EF03
:10DB30002390270197D0FFFFE78080DE1544E38420
:10DB4000A9F6268597A00000E780C0BC9787FF1F35
:10DB50009387C7239C430144B9D74A859750000057
:10DB6000E780C05889B785097DB71743FFFFE702F3
:10DB7000235279713E847C083EC82E8AB707140070
:10DB8000A1653ECAE5057C08AA89080836C4428911
:10DB900032C6BA8AC6843ECC97C0FFFFE78000E356
:10DBA000CA85080897E0FFFFE78000C732460808EB
:10DBB000B28597E0FFFFE78020C8A246630A090408
:10DBC0009D45080897E0FFFFE780C0BE1D468145E0
:10DBD0009740FFFFE780605063890A089145080875
:10DBE00097E0FFFFE78000BD1146A6859700010082
:10DBF000E780607A100801478146D2854E8597C03C
:10DC0000FFFFE780000245611743FFFF6700834B7A
:10DC1000B685080897E0FFFFE78000C21C400808AF
:10DC2000D8439355C701858912075183B205D98D11
:10DC300097E0FFFFE78040C01C40080883C58700CD
:10DC400097E0FFFFE78040BD1C40080883C5A700A0
:10DC500097E0FFFFE78040BC1C40080883C59700A1
:10DC600097E0FFFFE78040BB85BF8945080897E044
:10DC7000FFFFE78020B483C704002300F50083C7BB
:10DC80001400A300F500BDB71743FFFFE7024340B0
:10DC900083C795004111AA8993F7F707A384F5007C
:10DCA0003285AE84328497E0FFFFE780A0C69317E9
:10DCB0000501C187635DF0042A89032A040097C027
:10DCC000FFFFE78080C519E9835744000548F11735
:10DCD00093B71700A307F100814631A81306F1009E
:10DCE000A28597000000E78060951DC51C459DC773
:10DCF00083D6470001480347F10093078500D28887
:10DD00004A86A6854E8597000000E78040E64101DF
:10DD10001743FFFF6700033B09487DBF1D486DBFE8
:10DD20001743FFFFE702C33665715C083EC4B707BF
:10DD30007B013EC65C083EC883C795002A8A3285AF
:10DD400093F7F707A384F500AE8997E0FFFFE7801C
:10DD500040BA8357E100E1C78945280097C0FFFF1B
:10DD6000E780C0C68145280097E0FFFFE780C0AA92
:10DD700097C0FFFFE780A0CC9787FF1F93874739A5
:10DD80009C431784FF1F0344E4E1AA8433348000DA
:10DD900099C3136424009787FF1F9387E7E89C4388
:10DDA00099C3136444009787FF1F938727FE9C4302
:10DDB00099C31364840083D504002800014997E0C7
:10DDC000FFFFE78060A783D52400280097E0FFFFCE
:10DDD000E78080A683D54400280097E0FFFFE78016
:10DDE000A0A597D0FFFFE780A0AE93150501C181E4
:10DDF000280097E0FFFFE78020A4A285280097E095
:10DE0000FFFFE78060A39C446360F90201478146FD
:10DE10003000CE85528597C0FFFFE78080E05961D2
:10DE20001743FFFF6700032ADC441314490028004E
:10DE30003E9497E0FFFFE7806096834744000347E6
:10DE4000540089070607BA978607E36AF5FC8355ED
:10DE500024002800814A97E0FFFFE780E09D83458A
:10DE60004400280097E0FFFFE780009B83455400B3
:10DE7000280097E0FFFFE780209A8347440063C9AA
:10DE8000FA00814A8347540063C1FA020509A5BF1D
:10DE90001C4413975A002800BA9783D50700850AB7
:10DEA00097E0FFFFE7804099C9BF032BC400939719
:10DEB0005A0028003E9B83552B00850A97E0FFFF00
:10DEC000E780809783550B00280097E0FFFFE780ED
:10DED000A0964DBF1743FFFFE702231D5C4993E760
:10DEE00017005CC997A00000E78020B61743FFFF2A
:10DEF0006700E31D1743FFFFE702231B2E848145C4
:10DF000097F0FFFFE780C0E705C583570500FD17C1
:10DF10002310F50009C4835725002310F40097004F
:10DF20000000E78060FB01451743FFFF6700231AED
:10DF300031457DD823100400C5BF1743FFFFE7021A
:10DF4000231583C7950041112A8A93F7F707A38405
:10DF5000F50032852E89328497E0FFFFE780809BB1
:10DF600093170501C1876356F006AA89C14522852A
:10DF700097E0FFFFE780A0802A8B4E85832A04006C
:10DF800097C0FFFFE780609931E983574400231170
:10DF900001000544F11793B71700A300F100814475
:10DFA0000348110003572100D6875285CE8622866A
:10DFB000CA8597F0FFFFE780A0A6A16793871702A5
:10DFC00048003EC42302810026C697E0FFFFE78099
:10DFD000406B41011743FFFF6700C30E130611009A
:10DFE000A28597F0FFFFE7806065AA8409E5231109
:10DFF0000100094475B7930521005A859700000078
:10E00000E78080EF835721002A84D9DB9787FF1FA1
:10E010009387C7D79C4381CB854513052100975033
:10E020000000E7800015835521002685314497C004
:10E03000FFFFE78020852DD52310050026859790CA
:10E040000000E780206D0144A1BF1743FFFFE702F6
:10E05000C30541112E896C00AA8402C697F0FFFF08
:10E06000E78000D20DC10357050005072310E50026
:10E0700097000000E78040E681473E854101174355
:10E08000FFFF6700C3043247954765DBCA852685D5
:10E0900097300000E780400DC147E34005FE324461
:10E0A000854741462310F40083570900A6851305D0
:10E0B00044002311F40097000100E780C02D228561
:10E0C00045BF1743FFFFE702A3FC83C7950041113B
:10E0D000AA8A93F7F707A384F5003285AE893284C4
:10E0E00097E0FFFFE780008393170501C187635620
:10E0F000F0062A8AC145228597D0FFFFE780206875
:10E10000AA845285032B040097C0FFFFE780E080BC
:10E1100031E983574400231101008544F11793B777
:10E120001700A300F1000144034811000357210028
:10E13000DA875685D2862686CE8597F0FFFFE78060
:10E14000208EA1679387070248003EC423029100F6
:10E1500022C697E0FFFFE780C05241011743FFFF4F
:10E16000670043F6A2851306110097F0FFFFE780D2
:10E17000E04C2A8409E523110100894475B72685FE
:10E180009305210097000000E78060ECAA8449FD18
:10E1900083552100228597B0FFFFE780A06E49F5E7
:10E1A000014997C0FFFFE780A077635DA900184889
:10E1B00093171900BA9703D707000DEF03572100F3
:10E1C0002390E70097C0FFFFE78080756306250373
:10E1D0009787FF1F938787BB9C4399C703552100EF
:10E1E00097500000E78080F0228597900000E7803C
:10E1F00060521DBF050975B795443DB705C193072A
:10E20000F00F630FF500C547630CF5009307F5FFAA
:10E2100005453315F5004205418182800145828024
:10E2200041657D158280B9E91743FFFFE702E3E707
:10E2300003450603328497000000E78060FC9305E5
:10E24000803EB305B502C205C18181CD0357E4020A
:10E25000854763F8E7001305040197E00000E780B5
:10E2600020428357E40241677D176385E700FD176D
:10E270002317F4021743FFFF670063E5828017430B
:10E28000FFFFE70203E0004283C79500444D0349C6
:10E29000140093F7F707A384F500834704002209CD
:10E2A00011673369F900A167B347F90041112A8B5F
:10E2B000AE8A63ECE70E834724001307C00EB9173C
:10E2C00093F7F70F6373F71003473400C14763EE0A
:10E2D000E70E834744001307E00793C707086371FD
:10E2E000F70C8349840083477400A209B3E9F9005D
:10E2F000856763F7F90A034A6400834754004E8533
:10E30000220A336AFA0097500000E780403B61C15F
:10E3100023962403834B3400137AFA00239A3403A0
:10E32000238874032399440393890401631C09001F
:10E3300023A60402239804024E8597E00000E7809C
:10E3400060363DA0034924004A8597000000E7801D
:10E3500020EB2397A402834744004E85A388F40250
:10E36000E38D0BFCE30B09FC97E00000E780202F16
:10E3700097900000E780007381460146D6855A8554
:10E3800097E0FFFFE7800058A167938797033EC49B
:10E3900023020100480002C697E0FFFFE780602EDD
:10E3A00041011743FFFF670043D18544A2862686BB
:10E3B000D6855A8597E0FFFFE780C054A167938711
:10E3C00097033EC423029100F1B7BD44C5B7914401
:10E3D000F1BF1743FFFFE702A3CB01111C08404D1B
:10E3E0003EC2B7070F003EC41C083EC62A89AE894C
:10E3F00097C0FFFFE780A0DA585C1C5C6346B70E4D
:10E400006394E50063E2A70E3385A740B3B7A70086
:10E41000B305B7401306803E81469D8D97000100ED
:10E42000E78080B793140501C180A1659385C5037A
:10E43000480097B0FFFFE78060598145480097D0BA
:10E44000FFFFE780603D83550404480097D0FFFF3D
:10E45000E780803E83552404480097D0FFFFE78083
:10E46000A03D814589CCC167FD179305F00F6388F6
:10E47000F400268597500000E780E0E0AA85480078
:10E4800097D0FFFFE780403903554404814501CD13
:10E49000C167FD179305F00F6307F5009750000063
:10E4A000E78060DEAA85480097D0FFFFE780C0368E
:10E4B00083456404480097D0FFFFE780E03583453B
:10E4C0007404480097D0FFFFE780003550000147F3
:10E4D0008146CE854A8597B0FFFFE780807405614D
:10E4E0001743FFFF670003BE814481B71743FFFF57
:10E4F000E702A3BB83C7950093F7F707A384F50052
:10E5000097000000E78020ED1743FFFF670023BC62
:10E510001743FFFFE702C3B783C795004111404D82
:10E5200093F7F707A384F5002A8A3285B284AE896F
:10E5300097D0FFFFE780003E2A8B268597D0FFFF0C
:10E54000E780403D2A89268597D0FFFFE780603A23
:10E5500093170B0163CA0702E177CA97C207C18309
:10E56000116763E3E70293070910C207C18313072A
:10E57000B00F637BF70093170901C187AA8A634A2A
:10E58000F000C54763FE570141011743FFFF6700D5
:10E5900063B397B0FFFFE780C028E31725FFD5B727
:10E5A00063080B0263060902814463890A02B70704
:10E5B0007F0023106405231124057CC05685970035
:10E5C0000000E780E0C39304803EB304950239A0C5
:10E5D000B7077F00232004047CC081440355240432
:10E5E00097E00000E780A0A3A1C497C0FFFFE780E9
:10E5F00000BB269593D7F44133379500AE97BA9771
:10E6000008DC5CDCCE85528597000000E780A0DC4A
:10E6100099E023220404A1679387B70348003EC40E
:10E620002302010002C697E0FFFFE7808005A9BF33
:10E63000814701481CDC232E0403E9B71743FFFF81
:10E64000E702A3A697C0FFFFE780C037E147330585
:10E65000F502914597500000E78000C5E55711C5C8
:10E660009777FF1F23AEA75281473E851743FFFFD1
:10E670006700E3A585471777FF1F2305F7528280C0
:10E680001743FFFFE70263A29777FF1F93870751A6
:10E6900080433DC0835704046390A7068357240436
:10E6A000639CB7043689B28497C0FFFFE78020AF30
:10E6B0005C5C63C3B7046395B7001C5C63EEA702A0
:10E6C0008347640463F3F400A6872303F4048347B9
:10E6D000740463F39700A687A303F40483574404E8
:10E6E00041677D176385E70085072312F4043C44E6
:10E6F00081C7CA85268582971743FFFF6700239D40
:10E700009777FF1F938787499C43014599C303C5AA
:10E71000870082801743FFFFE70223990111B707A3
:10E7200007003EC683C79500584D0AC493F7F70704
:10E730000AC8A384F5002A89AE8411CB1C4283C782
:10E7400007002304F70097900000E780003421645D
:10E7500093055402280097B0FFFFE7802027970019
:10E760000000E78020FAAA85280097D0FFFFE78005
:10E77000A00A300001478146A6854A8597B0FFFF71
:10E78000E780204A13044402480822CC230A0100EF
:10E7900002CE97E0FFFFE780C0EE05611743FFFF61
:10E7A0006700E3921743FFFFE702239001117C000B
:10E7B0003ECAB70707003ECC7C003ECE83C795001B
:10E7C0002E84AA8493F7F707A384F500A1659385A7
:10E7D0005502480897B0FFFFE780401F97000000F0
:10E7E000E78040F2AA85480897D0FFFFE780C00283
:10E7F000500801478146A285268597B0FFFFE78034
:10E80000404205611743FFFF6700638C9777FF1F46
:10E810009387C7389C43094599C303C597008280F5
:10E820009777FF1F938787379C43094599C303C593
:10E83000D70082809777FF1F938747369C43014517
:10E8400099C303C5A70082801743FFFFE7024384F3
:10E850000111B70708003EC683C79500404D0AC4A2
:10E8600093F7F7070AC8A384F5002A89AE8429C460
:10E870001442854703C7060063E0E70A8347940014
:10E88000094681496380C702B307F740A304E40047
:10E89000B339F00083C716002305F40097900000F9
:10E8A000E780A01E03572403058B19C76386090060
:10E8B00097D00000E78000E92164930584022800D6
:10E8C00097B0FFFFE780801097000000E78040F4DA
:10E8D000AA85280097D0FFFFE78000F4970000008A
:10E8E000E78080F5AA85280097D0FFFFE780C0F277
:10E8F000014781463000A6854A8597B0FFFFE78033
:10E90000403213047402480822CC230A010002CECC
:10E9100097E0FFFFE780E0D605611733FFFF670050
:10E92000637A1733FFFFE702437801117C003ECA88
:10E93000B70708003ECC7C003ECE83C795002E84EE
:10E94000AA8493F7F707A384F500A1659385850250
:10E95000480897B0FFFFE780600797000000E78056
:10E9600020EBAA85480897D0FFFFE780E0EA9700F0
:10E970000000E78060ECAA85480897D0FFFFE78099
:10E98000A0E9500801478146A285268597B0FFFF80
:10E99000E780202905611733FFFF670043739777EE
:10E9A000FF1F9387A71F9C43014599C303C5B70069
:10E9B00082801733FFFFE702436F0111B70707009B
:10E9C0003EC683C79500404D0AC493F7F7070AC8AF
:10E9D000A384F5002A89AE8405C81C42054783C775
:10E9E00007006368F7060347B400630FF700A30549
:10E9F000F40097900000E78040098347B400B9CF46
:10EA000097D0FFFFE78040BE21649305B400280043
:10EA100097B0FFFFE78080FB97000000E78060F879
:10EA2000AA85280097D0FFFFE78000DF01478146D5
:10EA30003000A6854A8597B0FFFFE780801E290435
:10EA4000480822CC230A010002CE97E0FFFFE780AE
:10EA500040C305611733FFFF6700636797D0FFFF6F
:10EA6000E78020BF55B71733FFFFE70203640111AA
:10EA70007C003ECAB70707003ECC7C003ECE83C771
:10EA800095002E84AA8493F7F707A384F500A16567
:10EA9000AD05480897B0FFFFE78040F397000000FE
:10EAA000E78020F0AA85480897D0FFFFE780C0D60E
:10EAB000500801478146A285268597B0FFFFE78071
:10EAC000401605611733FFFF670063609777FF1FEC
:10EAD0009387C70C9C43094599C303C5C70082802F
:10EAE0001733FFFFE702635C01117C00AE843ECA6E
:10EAF000A165B70707002A843ECCD1057C004808F1
:10EB00003ECE97B0FFFFE78060EC97000000E78003
:10EB100020FCAA85480897D0FFFFE780E0CF500887
:10EB200001478146A685228597B0FFFFE780600FE9
:10EB300005611733FFFF670083591733FFFFE702B3
:10EB4000C35683C7950093F7F707A384F500970092
:10EB50000000E78020F91733FFFF670043571733A2
:10EB6000FFFFE702E35283C795000329C501411166
:10EB700093F7F707A384F5001C4283C90700854774
:10EB800063E637079777FF1F938787589C432E8448
:10EB9000AA8485CF97000000E78080F38947630649
:10EBA000F502630409028347C90063803703230623
:10EBB000390197900000E78040ED83572903898B46
:10EBC00089C797D00000E780E0B72685A285970027
:10EBD0000000E78020F1A167CD0748003EC4230272
:10EBE000010002C697E0FFFFE780A0A941011733AB
:10EBF000FFFF6700234D9777FF1F938727FA9C43FA
:10EC00001D4599C303C5E70082801733FFFFE70264
:10EC1000C3490111B70707003EC683C79500584D89
:10EC20000AC493F7F7070AC8A384F5002A89AE84BB
:10EC300015C71C4283C7070093968701E18663C40A
:10EC4000060685466381D7068346E7006388F6009B
:10EC50002307F70097900000E78020E321649305E5
:10EC6000E400280097B0FFFFE78040D6970000003F
:10EC7000E780A0F8AA85280097D0FFFFE780C0B9F9
:10EC8000014781463000A6854A8597B0FFFFE7809F
:10EC900040F93504480822CC230A010002CE97E04F
:10ECA000FFFFE780009E05611733FFFF67002342E7
:10ECB0001733FFFFE702633F01117C003ECAB7072D
:10ECC00007003ECC7C003ECE83C795002E84AA84EC
:10ECD00093F7F707A384F500A165B905480897B035
:10ECE000FFFFE780A0CE97000000E78000F1AA8533
:10ECF000480897D0FFFFE78020B2500801478146BF
:10ED0000A285268597B0FFFFE780A0F10561173344
:10ED1000FFFF6700C33B1733FFFFE7026337AA8497
:10ED200001441779FF1F1309A9E7E14997C0FFFFC5
:10ED3000E78040C96344A400014519A833053403A2
:10ED4000832709003E958357250063979700110597
:10ED50001733FFFF670003370504C9BF032E850083
:10ED6000630A0E121773FF1F1303430203230300EA
:10ED70006315030029436390061203234E016315B4
:10ED800003001D43639907101733FFFFE702632F4A
:10ED9000C689428A3E89BA8AB684328BAE8B2A846F
:10EDA000B5E103554E0019E501431A851733FFFFFE
:10EDB0006700A330A167A98F116763FBE700970085
:10EDC0000000E78080F5814597F0FFFFE780C012E3
:10EDD0000844B70700E05841F98F18455CC1B707F0
:10EDE000001FF98F1CC55C4991C7610597E00000C1
:10EDF000E780408BE38A09FA228597900000E7803C
:10EE000060C65DB7328597C00000E78040430D4380
:10EE100049DD1C44116703D54700A167A98F63FB37
:10EE2000E70097000000E78040EF814597F0FFFF83
:10EE3000E780800C0323840093164B01D182834723
:10EE4000B300035663008588FD8BA305F300FD77AF
:10EE50007D8E558EFD76FD16B204F18E832743011B
:10EE6000C58E231273012313D300230453012305FA
:10EE70002301A3044301BDDF228597B0FFFFE78094
:10EE800020CDAA850844B5D1610597D00000E78060
:10EE9000207F8DB71D431A8582801733FFFFE7025D
:10EEA000231F0569AA84AE89328A0144FD5A7D195F
:10EEB00097C0FFFFE780C0A56347A4000145173353
:10EEC000FFFF67002320D84493171400BA9703D795
:10EED0000700631F37032390570163070A00268545
:10EEE00097900000E780A0809C449DC383D7670073
:10EEF000B3F72701639E3701D28801488147014754
:10EF0000814601468145268597000000E78040E55F
:10EF1000050479BF1733FFFFE702831779711C10CF
:10EF20003EC4B7070F003EC61C103EC883C79500FD
:10EF3000AA8A328593F7F707A384F5002E893284D5
:10EF400097D0FFFFE780009D93170501C187635AA3
:10EF5000F006AA89228597D0FFFFE780A09B2A8A26
:10EF60004E85032B040097B0FFFFE780009B39ED2F
:10EF70008357440081440544F11793B71700A30356
:10EF8000F10083457100DA872287D2864E862800F9
:10EF900097E0FFFFE780E057014781463000CA85D0
:10EFA000568597B0FFFFE780C0C7A1679387F70337
:10EFB00048083ECC230A810026CE97D0FFFFE78089
:10EFC000406C45611733FFFF6700C30FA28513062E
:10EFD000710097E0FFFFE7806066AA84094455D17D
:10EFE000528597E0FFFFE78060D40D4459D905466C
:10EFF000D285268597000000E78060EA2A8451B711
:10F000001733FFFFE702630A835507000346270013
:10F0100041112A842E8532C62EC497E0FFFFE78077
:10F02000E0D001C93246A245228597000000E78062
:10F0300000E741011733FFFF670063091733FFFF44
:10F04000E702230483C795004111AA8A93F7F707C3
:10F05000A384F5003285AE89328497D0FFFFE78024
:10F06000608B93170501C1876357F00AC1452A8A4F
:10F07000228597C0FFFFE78080702A8D228597D078
:10F08000FFFFE78020892A89228597D0FFFFE7804C
:10F090004086930705F893F7F70F1307E007AA8B4D
:10F0A000637BF706228597D0FFFFE78080842A8C58
:10F0B000228597D0FFFFE780C083AA8C5285032B5F
:10F0C000040097B0FFFFE780408539E9835744008B
:10F0D000231101008144F11793B71700A300F10039
:10F0E0000544034711008356210093878400568509
:10F0F000DA8822885286CE8597F0FFFFE78020A726
:10F10000A167E90748003EC42302810026C697D0C4
:10F11000FFFFE780005741011733FFFF6700E3F966
:10F1200013061100A28597E0FFFFE7802051AA8413
:10F1300009E52311010009446DB7930521006A8593
:10F1400097F0FFFFE780A0F02A8441FD835521005E
:10F150009356C9001316490185486688E2875E8781
:10F16000858A5182268597000000E78060BF2A8447
:10F170008DBF1733FFFFE702C3F083C7950041112E
:10F180002A8B93F7F707A384F5003285AE89328482
:10F1900097C0FFFFE780007893170501C18763528E
:10F1A000F00A2A8A228597C0FFFFE780A076AA8A04
:10F1B000228597C0FFFFE780E0752A89228597C0E6
:10F1C000FFFFE7800073930705F893F7F70F130726
:10F1D000E0072A8C6377F706228597C0FFFFE78058
:10F1E0004071AA8C228597C0FFFFE78080702A8D2E
:10F1F0005285832B040097A0FFFFE780007239E55A
:10F200008357440085440144F11793B71700A301C5
:10F21000F10003473100930784005A85DE88268871
:10F22000D6865286CE8597F0FFFFE78040948D47C3
:10F2300048003EC42302910022C697D0FFFFE7801A
:10F24000404441011733FFFF670023E7A2851306FF
:10F25000310097E0FFFFE780603E2A84894455D95A
:10F260009356C9001316490185486A88E687628764
:10F27000858A5182D68597000000E78060AEAA8417
:10F2800049BF1733FFFFE702A3E02A898144014405
:10F29000617A916A177BFF1F130B4BAF97B0FFFF8B
:10F2A000E780006863C7A40022851733FFFF67006B
:10F2B00063E18327090093991400CE9703D50700D3
:10F2C00033074501420741836364570305C10327A0
:10F2D0000B0019C785453E8597400000E78060E92F
:10F2E000832709000504CE972390070085047DB786
:10F2F00097000000E78060A2832709000504CE97ED
:10F300002390070065D5814597F0FFFFE780C0BED9
:10F31000F1BF1733FFFFE702A3D783C79500411161
:10F320002A8A93F7F707A384F50032852E89328461
:10F3300097C0FFFFE780005E93170501C187635AFE
:10F34000F004AA89832A040097A0FFFFE780E05C0D
:10F3500031E58357440085440144F11793B7170002
:10F36000A301F10003483100D68752850147CE86BC
:10F370002686CA8597D0FFFFE780806AA167F507D8
:10F3800048003EC42302910022C697D0FFFFE780C9
:10F39000402F41011733FFFF6700C3D2A285130638
:10F3A000310097E0FFFFE78060292A8489445DD916
:10F3B0009777FF1F9387879D9C4381CF044997B020
:10F3C000FFFFE780E055AA85268597400000E7808B
:10F3D00040DA1305040197000000E780C0EA2285A7
:10F3E00097800000E78000338144ADBF1733FFFFF3
:10F3F000E70223C983C795004111AA8A93F7F7074B
:10F40000A384F5003285AE8932842311010097C0B0
:10F41000FFFFE780205093170501C1876354F00672
:10F420002A8AC145228597C0FFFFE7804035AA8B15
:10F430005285032B040097A0FFFFE780004E21E9CF
:10F440008357440085440144F11793B71700A30084
:10F45000F1000348110003572100DA875685D28650
:10F460002686CE8597D0FFFFE780805BA1679387D4
:10F47000270248003EC42302910022C697D0FFFF16
:10F48000E780202041011733FFFF670003C3A285F7
:10F490001306110097E0FFFFE780401A2A84894491
:10F4A0004DD99777FF1F9387678E98433E8901CF89
:10F4B000044997B0FFFFE780A046AA8526859740BC
:10F4C0000000E78000CB1305040197000000E780EF
:10F4D00080DB97B0FFFFE780A04495443DD99305BA
:10F4E00021005E8597F0FFFFE78060B6AA8435F1C2
:10F4F0001C480357210022852390E70097800000D5
:10F50000E780402183270900A9D7035521009740B0
:10F510000000E780A0BD35BF1733FFFFE70263B6E9
:10F5200083C795004111AA8A93F7F707A384F500D2
:10F530003285AE89328497C0FFFFE780A03D9317E4
:10F540000501C1876351F0062A8A228597C0FFFF13
:10F55000E780403C2A895285032B040097A0FFFFD7
:10F56000E780A03B31E58357440085440144F1170F
:10F5700093B71700A301F10003483100DA875685DD
:10F580004A87D2862686CE8597D0FFFFE7804049FE
:10F59000A167F90748003EC42302910022C697D014
:10F5A000FFFFE780000E41011733FFFF6700E3B064
:10F5B000A2851306310097E0FFFFE78020082A8428
:10F5C00089445DD99167CA97C2071167C183130740
:10F5D000F7EF8544E362F7FA9767FF1F9387077B8E
:10F5E0009843BE8B01CF044997B0FFFFE7804033BB
:10F5F000AA85268597400000E780A0B7130504017F
:10F6000097000000E78020C897B0FFFFE7804031F7
:10F6100095443DD11C482285814423902701978041
:10F620000000E780200F83A70B00B9D74A859740D9
:10F630000000E780A0AB89B71733FFFFE702E3A61E
:10F640002A844105B28497000000E780C0C311C539
:10F65000228597800000E780E00B81460146A68561
:10F66000228597800000E780C04E1C4C89C7DC478C
:10F6700099C3228582971733FFFF670043A59767D9
:10F68000FF1F9387A7519C43014599C31385070129
:10F6900082809767FF1F9387675088438280173364
:10F6A000FFFFE70283A09317C600DD8DC20541115D
:10F6B000C1812A8432C697C0FFFFE780E017324637
:10F6C000228511829375F60F97C0FFFFE780C01463
:10F6D00041011733FFFF6700839F1733FFFFE702E6
:10F6E000239B79713C083ED2B7070C003ED43C08FE
:10F6F0003ED683C79500AE842A8993F7F707A38483
:10F70000F500A16593853504481097A0FFFFE780B9
:10F71000E02BC165FD150144176AFF1F130A8A68B3
:10F72000930A400EAE892E8B2EC697B0FFFFE7805E
:10F7300020224205931704014181C183B24563E948
:10F74000A702C167FD176387F500481097C0FFFF48
:10F75000E780800E501001478146A6854A8597A014
:10F76000FFFFE780004C45611733FFFF670083957B
:10F770003307540383270A0BBA9703D6C701630ADA
:10F780003601638A3501481097000000E78060F178
:10F79000DA85050451BFB285EDBF1733FFFFE702DD
:10F7A000438E79717C083EC8B70711003ECA7C08B9
:10F7B0003ECC83C79500AA89328593F7F707A384C7
:10F7C000F5002E8997C0FFFFE780C0148567637836
:10F7D000F504A165AA848905080897A0FFFFE780C2
:10F7E000E01E268597400000E78060ED1334150089
:10F7F0000A04A285080897C0FFFFE780E001A685FC
:10F80000080897C0FFFFE780200325CC0147814609
:10F810001008CA854E8597A0FFFFE78080404561AC
:10F820001733FFFF67006389B30754030327CA0A2E
:10F83000BA9703D70700631C970003D6270063809D
:10F840006505080897000000E780A0E5DE8505044F
:10F850002EC697B0FFFFE780A01042059317040162
:10F860004181C183B245E3E1A7FCC167FD17E38F86
:10F87000F5F8080897C0FFFFE78000FC41BFB2859C
:10F88000F9B7C165FD150144176AFF1F130A8A51B4
:10F89000930A80022E8BAE8B65BF1733FFFFE70202
:10F8A000C38018418347170083460700A207D58FFE
:10F8B000D207D1832390F500834727000347170021
:10F8C0008D45A207D98F91832310F60097C0FFFFC3
:10F8D000E780A0E91723FFFF6700637F1723FFFF7F
:10F8E000E702037BC16401441769FF1F1309894BB9
:10F8F00093098002FD1497B0FFFFE780600663471D
:10F90000A40001451723FFFF6700C37B33053403C1
:10F910008327C90A3E9583570500E38597FE0504B2
:10F92000D9BF1723FFFFE702A3762A8AAE89B284E4
:10F93000B68A97400000E78080D819E591473E8558
:10F940001723FFFF670003782A894E8597C00000C0
:10F95000E780E08E2A84638E0A048D476DD10357B9
:10F960000500C547E31D47FD0347F9018546AD473F
:10F97000E317D7FC8347450081CF4146A6855D0547
:10F9800097F00000E780C09E814755D9AD4745BF3D
:10F99000130965012302E500CA852685971000003A
:10F9A000E780606231C1A547E38B0AF823020400B7
:10F9B00079B705C183570500E39247F94146A6850B
:10F9C000190597F00000E780A09A81472DD9994743
:10F9D000BDB74E8597000000E78080F02A849547E8
:10F9E00039DD130955004DBF4146A685231044015A
:10F9F000231134011305190097F00000E780A09946
:10FA0000228597800000E780A0EA81470DBF172379
:10FA1000FFFFE702836979717C003ECCB7070A00DB
:10FA20003ECE7C003ED083C79500B2842E8493F7EF
:10FA3000F707A384F5001306A1002A892C00268568
:10FA400097000000E780A0E5A16528088D0597A034
:10FA5000FFFFE780A0F790408355A1000355810088
:10FA6000854697000000E78000ECAA84AA85280854
:10FA700097C0FFFFE78040DA0356A100835581005D
:10FA8000280897000000E780C0C130080147814680
:10FA9000A2854A8597A0FFFFE780A01885474810F8
:10FAA0003ED42302910202D697D0FFFFE78060BDCB
:10FAB00045611723FFFF670083611723FFFFE702FC
:10FAC000C35E79717C003ECCB7070A003ECE7C0055
:10FAD0003ED083C79500B2842E8493F7F707A384A2
:10FAE000F5001306A1002A892C0026859700000046
:10FAF000E780E0DAA16528088D0597A0FFFFE78081
:10FB0000E0EC90408355A1000355810081469700A9
:10FB10000000E78040E1AA84AA85280897C0FFFF7B
:10FB2000E78080CF0356A100835581002808970005
:10FB30000000E78000B7300801478146A2854A856A
:10FB400097A0FFFFE780E00D48102302910202D446
:10FB500002D697D0FFFFE780C0B245611723FFFFB1
:10FB60006700E3561723FFFFE702235497000000C6
:10FB7000E78060DB1723FFFF670063559767FF1F70
:10FB800093870702884382801723FFFFE702E35130
:10FB9000835725004111AE842A842307B10017F54D
:10FBA000FFFF130525466C002316F10097A0FFFF09
:10FBB000E780204991C4228597800000E780E0D645
:10FBC000FD572310F400130620028145130554004D
:10FBD0009720FFFFE780605041011723FFFF670078
:10FBE000034F1723FFFFE702A34A79717C003ECC45
:10FBF000B7070A003ECE7C003ED083C79500AA8995
:10FC0000AE8493F7F7073285A384F5001306A100AD
:10FC10002C0097000000E78080C803558100114444
:10FC200097400000E780A0A915C50355A100014435
:10FC300097B00000E780A06011CD035705008357FF
:10FC4000810045446318F700854597000000E78070
:10FC5000E0F30144216993053900280897A0FFFFCC
:10FC6000E780C0D6A285280897C0FFFFE780C0BA0A
:10FC70000356A10083558100280897000000E78003
:10FC800040A2300801478146A6854E8597A0FFFF18
:10FC9000E78020F948104AD42302810202D697D087
:10FCA000FFFFE780009E45611723FFFF6700834148
:10FCB0001723FFFFE702C33D9767FF1F938707EEF8
:10FCC0002A8488432E8915C5035745038357C401E9
:10FCD0006311F7022326050223180502410597D078
:10FCE0000000E780209C6306090097800000E78001
:10FCF00060DB81449769FF1F9389C90A130A800258
:10FD000097B0FFFFE780C0C563C4A4049767FF1FD7
:10FD1000938787F19C4399C70355C401972000003E
:10FD2000E780C0BD63070900228597800000E78057
:10FD3000C0A01306400E814522859720FFFFE78073
:10FD4000C039FD57231EF4001723FFFF67008337D8
:10FD50003385440383A7C90A3E950357050083579B
:10FD6000C4016317F700CA8597000000E78000E22E
:10FD7000850479B71723FFFFE702833183C7950016
:10FD80004111AA8993F7F707A384F5003285AE8461
:10FD900097C0FFFFE78000B885676378F5042A897C
:10FDA00097400000E780A091014401CD83D7040073
:10FDB000314463882701854597000000E78080EF84
:10FDC00001444E85A2864A86A68597D0FFFFE7802C
:10FDD000A09CA1679387170448003EC423028100BA
:10FDE00002C697D0FFFFE780C08941011723FFFFBC
:10FDF0006700432D1723FFFFE70283299767FF1F43
:10FE00009387C7D9804329C4014597C00000E78084
:10FE1000002181470148C1641CDC232E04032320F8
:10FE200004041769FF1F1309E9F701449309400E01
:10FE3000FD1497B0FFFFE780A0B1634FA400814598
:10FE400017F5FFFF1305857F97A0FFFFE780601F71
:10FE50001723FFFF67000327330534038327090BAC
:10FE60003E958357C501638797008545970000003D
:10FE7000E78040E4050475BF9357050113D7870059
:10FE8000A380F50093170501C183A1832380E500BA
:10FE90002381F500A381A50082801723FFFFE702DD
:10FEA000C3202300050083C71500A300F50083C706
:10FEB00025002301F50083C73500A301F50083C7A2
:10FEC00045002302F50083C75500A302F50083C750
:10FED000650093059500A30305002303F5002304A3
:10FEE0000500328597000000E78040F91723FFFFE7
:10FEF0006700E31D1723FFFFE70283194111E9544F
:10FF00000DCD85CD93F9C5FF2E842A89AA84338A25
:10FF1000A900B7EA040063189A020D88854411CC41
:10FF2000B7E704009C5F82972AC622866C003305DF
:10FF3000390197E00000E78000462685410117233C
:10FF4000FFFF6700231883A78A0391048297931702
:10FF50000501C183A183A38EF4FE93570501238F6E
:10FF6000F4FEA183238EA4FEA38FF4FE6DB763E697
:10FF7000D5021723FFFFE7024313B28741113686EC
:10FF8000BE8536C697E00000E780E040B2464101FA
:10FF900036851723FFFF67008313814636858280ED
:10FFA000838705001387F5003D05FD8793F77708E4
:10FFB000834607007D158606B58FA300F50063070D
:10FFC000B7007D17834717009D83DDB78280172315
:10FFD000FFFFE702830DB7E7040083A70709328715
:10FFE0002A863A858297133515001723FFFF67008D
:10FFF000030E15C181478DC11723FFFFE702E30AF6
:020000040001F9
:10000000414697E00000E780003985473E85172389
:10001000FFFF6700C30B81473E8582801DCD1723FC
:10002000FFFFE7028308414681452A849720FFFFAE
:10003000E780A00A41468145130504039720FFFF8E
:10004000E780A0090147C1672322040438C87CC89F
:1000500005451723FFFF670083070145828081471D
:100060003DCDB5CD1723FFFFE7022304B2842E89CF
:100070001306800581452A849720FFFFE780E0056D
:10008000CA8524C4268597000000E780C0F6414653
:10009000814522859720FFFFE78020043044A28518
:1000A000228597000000E780C0F293040401A28536
:1000B000268597000000E780E0EEA6851305040280
:1000C00097000000E78000EE228597000000E7809F
:1000D00020F585473E851723FFFF670043FF3E85D8
:1000E00082801723FFFFE702A3FA4111E9540DCDE7
:1000F00085CD93F9C5FF2E842A89AA84338AA90065
:10010000B7EA0400639844030D88814411CCB7E733
:1001100004009C5F82972AC622866C003305390151
:1001200097E00000E7802027268541011723FFFF85
:10013000670043F983A78A03910482979317050107
:10014000C183A183A38EF4FE93570501238FF4FE90
:10015000A183238EA4FEA38FF4FE6DB765CD172374
:10016000FFFFE702E3F2B28411E605451723FFFF24
:10017000670043F52A842E890145EDD93C4878482B
:10018000B3E6E700E5D69386F7FFB3B7F6007D1731
:10019000032A4404BA9734C87CC863050A06C149D7
:1001A00013050A03B38949412295637D3601B2865E
:1001B0002E86A68597000000E780A0DB7C40BE94D9
:1001C00064C065B7CE862E86CE8597000000E78096
:1001D00040DAC114D2944E9923220404A2879306D4
:1001E000040103C7070003C607038507318FA38FE8
:1001F000E7FEE398F6FE3044A285228597000000D2
:10020000E78020DD2699C1493306994063EC9900C7
:10021000A9DCA686A6851305040397000000E780E5
:1002200040D579BF8147B306F4003307F600034792
:10023000070083C5060085072D8F2380E600E39421
:1002400037FF3044A285228597000000E78060D800
:10025000C1145DBF014582800DC11723FFFFE70276
:10026000C3E41306800581459720FFFFE780E0E6A1
:1002700005451723FFFF670083E50145828081471D
:1002800049C5C1C51723FFFFE70223E2FC414146F0
:100290002E84AA846399C70413860501A287814628
:1002A000C14503C7070003C507038507298F330529
:1002B000D600034505008506298FA38FE7FEE3924C
:1002C000B6FE3044A285268597000000E78060D006
:1002D000228597000000E78060F885473E85172358
:1002E000FFFF6700C3DE138507031D8E814522953E
:1002F0009720FFFFE78060DE7C40130700F81306BD
:100300000402A2972388E70251BF3E85828017230B
:10031000FFFFE70283D96D712E84B284AA85901005
:100320002800368997000000E780A0D309EDD55753
:1003300025A050400C40280097000000E78040E2D4
:100340007DD5FD142104F5F42C004A8597000000AA
:10035000E78020F3814761DD3E8551611723FFFF70
:100360006700E3D61723FFFFE70223D441112EC411
:1003700032C62C00054697000000E78080F9410155
:100380001723FFFF6700A3D41723FFFFE702E3D182
:1003900001112A842EC602C802CA02CC02CE97E0FE
:1003A0000000E780402BB2462A86A2850808970005
:1003B0000000E78060FB1375F50F05611723FFFF51
:1003C0006700E3D01723FFFFE70223CE7971B287DE
:1003D0002A8421462308B10013051101BE853AC4C1
:1003E00036C697E00000E78000FBB2469305910116
:1003F000368597000000E78060A8228514103546F6
:100400000C0897000000E78020F62A84224701E9C3
:1004100021460C103A8597E00000E780C0F722855E
:1004200045611723FFFF670083CA1723FFFFE70219
:10043000C3C77171AE84AA850A8532849700000013
:10044000E78060BB11C90A86A68522859700000057
:10045000E78020B8814711E1C5473E854D611723EC
:10046000FFFF6700C3C61723FFFFE70203C11D712B
:100470002A8AB289BE8435468547130511012E8C20
:10048000B68A3A8BC28C468D2308F10097E00000B3
:10049000E78060F010100C085285231F01009700C0
:1004A0000000E780C0F82A843DEDA1476313FD08F2
:1004B0009307900591E0E5473546E2851305110164
:1004C00013990A012308F1001359090197E000006C
:1004D000E78060EC1357890093978A00D98F9008C2
:1004E0000C085285231FF10097000000E78020F4DC
:1004F0002A8415E9A1E49387FA0091831379F9001E
:100500003EC6631309004149668B8144C14B854D4A
:10051000B247639F970C6A868C0033855C0197E035
:100520000000E78040E7228525611723FFFF670071
:1005300083B893079004C9F0A547BDBF8347010561
:100540000947C14B2308F10083471105A58FA30874
:10055000F10093872400814463E1FB040147140800
:100560003386E6008C08B386E400BA95DA9683C633
:10057000060083C505000507AD8E2300D600E39075
:10058000E7FE4147639CE70490080C0852859700FA
:100590000000E780C0E925D181A0B3069B00BA879F
:1005A0001008B305F60090083E9603C50600034602
:1005B000060085078506298E2380C500E39277FF14
:1005C000998F90080C085285BE9497000000E78030
:1005D00000E68947014749D12A84B1B790083E9681
:1005E000034606001408BE962380C600850759BF3F
:1005F000B24785046387971481471808B306F7004C
:1006000098083E973386F900034707000346060023
:100610008507318F2380E600E39177FF90080C086F
:10062000528597000000E78080E05DF53546E28561
:10063000130511012308B10197E00000E780A0D560
:10064000139704014183939784002183D98F101855
:100650000C085285231FF10097000000E78020DD81
:1006600025FD814710183387F9003E9603470700A0
:1006700003460600B306FB008507318F2380E600A2
:10068000E39277FF65A81808B306F70098083E972D
:100690003386F90003470700034606008507318FBC
:1006A0002380E600E3E127FFCA87639E770990086D
:1006B0000C08528597000000E78060D711FD814744
:1006C0009800B306F700900818103E973E9603472F
:1006D0000700034606008507318F2380E600E3917B
:1006E00077FF3546E285130511012308B10197E034
:1006F0000000E78040CA1397040141839397840068
:100700002183D98F10180C085285231FF100970000
:100710000000E780C0D1E31105EC81471018338752
:10072000F9003E960347070003460600B306FB00A8
:100730008507318F2380E600E3E227FFC109410BE3
:10074000C1BB814785B79408BE9683C606001808CA
:100750003E972300D700850789BF638006321723A1
:10076000FFFFE702839159712A84BE89B28B8547C6
:100770003546130511022E8B468C4289BA8A368A79
:100780002300F10297E00000E780E0C010180C1091
:1007900022852317010297000000E78040C96318F3
:1007A0000512A147631FFC06930790056393090098
:1007B000E5473546DA851305110293140A01230033
:1007C000F102C18097E00000E780E0BC93178A0047
:1007D00013D78400D98F90080C1022852317F102BB
:1007E00097000000E780A0C47DE1639209049307AD
:1007F000FA00BD88918391E0C144C207C183DE8CB9
:10080000814A3EC6414DB24763E2FA0E6286B38525
:100810004B01881097E00000E78080B54DC93D5539
:100820007DA093079004E39609F8A54759B783473D
:1008300001050947C14C2300F10283471105B3C7E5
:10084000F900A300F10293872900814963E1FC04C8
:10085000814618103306D7008C083387D900B69527
:1008600056970347070083C5050085062D8F230093
:10087000E600E390D7FE41476390E70690080C102E
:10088000228597000000E78080BA35D189A0B38621
:100890003A01BA871010B305F60090083E9603C5DA
:1008A00006000346060085078506298E2380C500BD
:1008B000E39297FF3387EC4090080C102285BA9999
:1008C00097000000E780A0B68947014741D16561E4
:1008D0001713FFFF6700237E90083E96034606002D
:1008E0001410BE962380C600850779B7B247850AE3
:1008F00093990A01939D8A0093D909016391570F37
:1009000085473546DA85130511022300F10293D994
:10091000890097E00000E78000A8B3ED3D0190005A
:100920000C1022852317B10397000000E78020B048
:1009300059FD8147A68963EA970626860C084A85F1
:1009400097E00000E78020A581471810B306F70064
:10095000100898083E973E96034707000346060096
:100960008507318F2380E600E3E197FE639FA905A9
:1009700090080C10228597000000E78040AB21F919
:1009800081479810B306F700900818183E973E96D6
:1009900003470700034606008507318F2380E600E2
:1009A000E391A7FF4109C10CB9BD18089000B30637
:1009B000F7003E963387FC00034707000346060016
:1009C0008507318F2380E600B5B798084E97034717
:1009D00007001C10CE972380E700850941BF85479B
:1009E0003546DA85130511022300F10293D98900F7
:1009F00097E00000E780209AB3ED3D0190000C10D5
:100A000022852317B10397000000E78040A2E3107E
:100A100005EC814718089000B306F7003E9633872F
:100A2000FC0003470700034606008507318F23803B
:100A3000E600E391A7FF41460C084A8597E00000D5
:100A4000E780609581471810B306F70010089808F2
:100A50003E973E9603470700034606008507318F01
:100A60002380E600E391A7FF90080C1022859700F1
:100A70000000E780C09B1DD599BD7D55828017136E
:100A8000FFFFE702836201112A842E85930551003E
:100A9000328902C002C202C402C69304740097F0F5
:100AA000FFFFE780A03D1D46A6851305910097E056
:100AB0000000E780408E10088A854A859700000074
:100AC000E780E09619ED93071400180883C6070025
:100AD0000346070085070507B18EA38FD7FEE3976E
:100AE000F4FE05611713FFFF6700635E1713FFFF36
:100AF000E702035A2E848C414111AA89838715008D
:100B00003289914463D30700A1449757FF1F93870D
:100B100027609C43A1C7C1CA8D472310F10083C73A
:100B200025004A852301F10083C73500A301F100A8
:100B300083C745002302F10083C75500A302F100DB
:100B400083C7650093059100A30301002303F1000F
:100B50002304010097F0FFFFE78040320C404A86F3
:100B60000A8597F0FFFFE78080330328040083564F
:100B70004400A6881D0881470147E51642868A85FC
:100B80004E8597000000E780408E2A8919E5A685EA
:100B9000228597B0FFFFE780E0C14A854101171326
:100BA000FFFF670023524A860A8597F0FFFFE78020
:100BB000002F6DB71713FFFFE702834D2E848C4182
:100BC0004111AA89838715003289914463D30700B4
:100BD000A1449757FF1F9387A7539C43A1C7C1C642
:100BE0008D472310F10083C725004A852301F100BA
:100BF00083C73500A301F10083C745002302F1003C
:100C000083C75500A302F10083C7650093059100D7
:100C1000A30301002303F1002304010097F0FFFF69
:100C2000E780C0250C404A860A8597F0FFFFE780E1
:100C3000002783564400032804008A85858EC20657
:100C40001D08C1822312D400A68881470147E516FA
:100C500042864E8597000000E78060B0410117137F
:100C6000FFFF670023464A860A8597F0FFFFE7806B
:100C700000234DBF1713FFFFE7022343B335B00036
:100C8000011185052A891315F6013365150123081D
:100C9000B1009305110136843AC632C03EC442C247
:100CA00097F0FFFFE780801DA2471248425593D678
:100CB0008700230BF1009305910193578800A30A45
:100CC000D100A30BF100230C010197F0FFFFE78097
:100CD000E01A3247024603280400B337E000835687
:100CE00044009207914411C2A1444A85A6884286D5
:100CF0000C0897F0FFFFE78040772A8919E5A68561
:100D0000228597B0FFFFE780E0AA4A8505611713A7
:100D1000FFFF6700C33B1713FFFFE70263370111B3
:100D20003EC68647B335B0008505AA891315F6017E
:100D30005D8D2308B1009305110136843A89B28490
:100D400042C446C297F0FFFFE78040132248924812
:100D5000164593578800A30AF1009305910193D794
:100D60008800230B0101A30BF100230C110197F064
:100D7000FFFFE780A0103247104083564400B3378E
:100D8000E000920703280900914891C0A1480C088F
:100D90004E8597000000E780809CAA8401E9835576
:100DA00044004A8597B0FFFFE780C0A02685056113
:100DB0001713FFFF67000331AA959307F00F17176A
:100DC00001001307A7986317B50013C5F7FF137544
:100DD000F50F828005058346F5FFB58FBA9783C767
:100DE0000700D5B70357450014419307F00F1716B6
:100DF00001001306A6953697420741831395060115
:100E00004181631BE500AD8FB29703C50700130551
:100E100015F3133515008280850603C5F6FFA98FEB
:100E2000B29783C70700D9BF1713FFFFE702E32775
:100E3000B28736842E86BA86AA853E85BA8497F014
:100E4000FFFFE7806052634F0500228597E00000B6
:100E5000E78060802A86A686A285268597F0FFFF18
:100E6000E78080501713FFFF670063261713FFFF0B
:100E7000E70203225D712A8BAE8A17150100130564
:100E8000658A2C00B284368ABA893E8997F0FFFFC2
:100E9000E780C04F2A845DE134104146DA8528009E
:100EA00097F0FFFFE780404C2A8449E98547A30378
:100EB000F100A6C2930771002408BEC4A686854728
:100EC0000D462C18281002DC02DED6C0BEC697F0F4
:100ED000FFFFE78000442A8435E183477102A6863C
:100EE0000D4693F7F7072300FA00C1473EDE2C18A2
:100EF0008947281026DCA303F10097F0FFFFE78065
:100F000040412A8405ED4146A6854E8597D00000D4
:100F1000E78060488D47A6860D462C182810A3034D
:100F2000F10097F0FFFFE780C03E2A8401E94146C7
:100F3000A6854A8597D00000E780E045228561615B
:100F40001713FFFF670003181713FFFFE702E315EE
:100F500097F70000938707EF984383C7470079719D
:100F60002A89AE84170501001305457C0C083AC494
:100F70002306F10097F0FFFFE78040412A8405ED4A
:100F800014104146CA85080897F0FFFFE780C03D6E
:100F90002A8415E1140815462C00081097F0FFFF6D
:100FA000E780803C2A8401E921462C08268597D0D9
:100FB0000000E780403E228545611713FFFF670070
:100FC00003111713FFFFE702430E97F70000938703
:100FD00067E79C477971AA842E84170501001305E1
:100FE00065750C083EC697F0FFFFE780203A0DE9D3
:100FF00014104146A685080897F0FFFFE780C03629
:1010000005E1140811466C00081097F0FFFFE78017
:10101000A03519E58347F10193F7F7032300F400A6
:1010200045611713FFFF6700830A1713FFFFE702ED
:10103000C3073688A14881470147E54697F0FFFF7F
:10104000E780A0421713FFFF670063081713FFFF35
:10105000E702A3053688A14881470147E54697F096
:10106000FFFFE780C06F1713FFFF670043061713EA
:10107000FFFFE702830301112A842E850C0832C684
:1010800097F0FFFFE780803009ED324797060100B7
:101090009386C6681008C145228597000000E78046
:1010A000E0D805611713FFFF670063021713FFFF06
:1010B000E702A3FF4111C1472EC032C48A85094609
:1010C0003EC23EC697F0FFFFE780A0244101171300
:1010D000FFFF6700C3FF1713FFFFE70203FD411186
:1010E000AE8613061009AA850A8502C002C202C490
:1010F00002C697F0FFFFE780202741011713FFFF8B
:101100006700E3FC1713FFFFE70223FA3287970615
:1011100001009386A6622E869305000297000000C8
:10112000E780C0D01713FFFF670063FA1713FFFFB4
:10113000E702A3F77971C1472ACC2ED032D42C080C
:101140000D4628003ECE3ED23ED602C402C602C89C
:1011500002CA97F0FFFFE780C01B45611713FFFF2E
:101160006700E3F61713FFFFE70223F40111AA84D7
:101170002E84170501001305E55C8A8597F0FFFFB3
:10118000E780C02015E514084146A6850A8597F03A
:10119000FFFFE780601D09ED8347E1010347F1018F
:1011A000A207D98FCA07C9836177D98F2310F400AA
:1011B00005611713FFFF670083F115CD1713FFFFBC
:1011C000E702A3EE9757FF1F938707A29043975517
:1011D000FF1F9385A5A11755FF1F1305E59C97D009
:1011E0000000E78000C51755FF1F1305E59B171387
:1011F000FFFF6700C3ED1755FF1F1305E59A8280B7
:101200008DCD1713FFFFE70243EA9757FF1F938720
:10121000A79D944301112E840A869755FF1F93853D
:10122000E59C97D00000E78040C60A8502940145FE
:1012300005611713FFFF670083E97D55828017134F
:10124000FFFFE70283E697D00000E78080D1975741
:10125000FF1F23ABA79817F5FFFF1305E5C997B04C
:101260000000E780C0741713FFFF670043E61757BD
:10127000FF1F1307A7999317150008433E95FD57C5
:101280002310F50082801713FFFFE70203E22A8490
:10129000084009E51713FFFF670063E31C4158404E
:1012A0001CC06313E5005CC0834755002320050084
:1012B000F99BA302F50097A0FFFFE780207CC9BF40
:1012C0001713FFFFE702C3DC9757FF1F93870796AB
:1012D00098432A8411CB8347350093F7070289C7C7
:1012E00003550500894502971305440197B0000096
:1012F000E780403B835504000355E400973000002D
:10130000E780A00C485819C597A0FFFFE780007739
:10131000232A04021305840397000000E780E0F607
:101320008144B1499790FFFFE780C06D63CBA40271
:10133000834734002320040493F727FCA301F4001F
:1013400000489790FFFFE780E06C13161500814579
:1013500022859710FFFFE78040D81713FFFF670033
:1013600063D6B38734030329040385043E994A8571
:1013700097000000E78060F12304090065B7834708
:10138000350093F7070299E3014582808357E50012
:10139000E39CB7FEC167FD176316F6000545828022
:1013A000054599A81713FFFFE70223D093170601FD
:1013B000C187B2842A8401496359F002835705002A
:1013C0009DCB01456367F600034584003E953325B8
:1013D000A6001375F50F0DA01C4813171900BA9736
:1013E00083D70700E38E97FA05099790FFFFE78000
:1013F0006062E343A9FE01451713FFFF670023CD99
:101400001713FFFFE702C3C8AE89AA849790FFFFB6
:10141000E78000562A8497D0FFFFE780A02EAA8697
:1014200001471306840197050000938585E417455D
:10143000FF1F1305E57D9790FFFFE780801C2A8939
:1014400025C98C441304C50022859E0593F5050823
:1014500097A0FFFFE780403CCC4083877400E18188
:1014600063DD070493E50508228597A0FFFFE78069
:10147000A03A0D4693854400228597A0FFFFE780A0
:10148000C03683D50400228597A0FFFFE780E03DAA
:1014900083D52400228597A0FFFFE780003D03D677
:1014A000490083A50900228597A0FFFFE780E0336C
:1014B0004A851713FFFF6700E3C093F5F5076DB783
:1014C0001713FFFFE70263BE01112A84328532C67B
:1014D00097A0FFFFE780E0279780FFFFE780603459
:1014E000835704001757FF1F1307C78B3246231B70
:1014F000F100930700F8A30DF1001C471843231ACD
:10150000A1008983858BB307F740B28548083ECE9A
:10151000231C0100230D010097000000E78080EEEE
:1015200005611713FFFF670083BA1713FFFFE70278
:1015300023B6004101453DC49304C4002685328989
:10154000AE8997A0FFFFE780C02495452A8A2685AB
:10155000035B040197A0FFFFE7802021268597A069
:10156000FFFFE780603E8D45AA8A268597A0FFFF92
:10157000E780A01F268597A0FFFFE780E03C5C483E
:10158000420A135A0A01D2975CC4231864018147A6
:1015900063983A0146054D8133062541933716007D
:1015A00013F5F70F1713FFFF6700C3B11713FFFF02
:1015B000E70223AD89692A8BAE8B328AB68A8144D1
:1015C0000144314CFD199790FFFFE780A04363CDA4
:1015D000A4009790FFFFE780E045018D33B5AA0096
:1015E0001713FFFF670063AD3389840383270B0064
:1015F0003E9963170A008347890085043E94E1B74A
:1016000003560A00DE854A8533F6C90097000000BC
:10161000E780E0F16DD10545E1B71713FFFFE70261
:10162000C3A801112A847C000355E5003ECAB70710
:1016300007003ECC7C003ECE97200000E7802008CB
:101640002A898545480897A0FFFFE78020399945FA
:10165000480897A0FFFFE780E015AA844A859720F5
:101660000000E780A0082380A4009747FF1F93870E
:1016700067739C434166130606F09396870113D760
:101680008701558F93D68700F18E558FA207B70635
:10169000FF00F58FD98F11462C00138514003EC42E
:1016A00097D00000E78020CF5008A382040089452E
:1016B000228597000000E780E0E019C9AA8513059C
:1016C000840397A0FFFFE780E0313C4085073CC0E2
:1016D00005611713FFFF6700839F1713FFFFE702E2
:1016E000C39C9790FFFFE780E0342A84050497901D
:1016F000FFFFE78020333305A402F147914533050E
:10170000F50297200000E78020BA11E56555171310
:10171000FFFF6700C39B9747FF1F23A1A750979028
:10172000FFFFE78020312A8405049790FFFFE780C0
:10173000602F3305A4028945060597200000E78045
:10174000A0B669D59747FF1F23A2A74C9790FFFF2C
:10175000E780402E2A8405049790FFFFE780802CC5
:101760003304A4029747FF1F2394874A9790FFFFF3
:10177000E780402C2A849790FFFFE780A02A9307F8
:1017800014003385A7029747FF1F2394A7489707A4
:1017900001009387E7BE1747FF1F232FF746014538
:1017A000BDB71713FFFFE702A38EAA842E89014459
:1017B0009749FF1F9389095F130A80069790FFFFDF
:1017C000E78040266347A40001451713FFFF670029
:1017D000638F3305440383A709024A86A6853E9595
:1017E00097000000E780E0B919E10504C1BF054595
:1017F000E9BF1713FFFFE702C388AA8A2E8BB28BBB
:10180000368C3A8A814401448149974CFF1F938C5E
:101810006C59130D80069790FFFFE780A02063C9E5
:10182000A40011E085494E851713FFFF6700E38888
:101830003389A40383A70C025E86D6853E994A8528
:1018400097000000E780E0B31DC19790FFFFE7809D
:10185000601E0544636D4501D2866286DA851305F4
:10186000090397000000E780A0D411C185498504D1
:101870005DB71713FFFFE702A381C16441112A89F5
:1018800001449749FF1F9389E951130A8006FD140B
:1018900036C632C42EC29790FFFFE780A01892454B
:1018A0002246B2466348A400014541011713FFFFD9
:1018B000670043813305440383A709023E9509C6A7
:1018C00083473500C18B9DC791C68347350093F789
:1018D00007028DC3630699008357E500639C2701C7
:1018E0000357050001CB63E7E50083478500BA97FE
:1018F000E3CDF5FA050469BF1703FFFFE70243795B
:10190000C1642A8901449749FF1F9389A949130A91
:101910008006FD149790FFFFE780C0106346A40087
:101920001703FFFF6700037A3305440383A7090207
:101930003E958357E500638A970063049900639698
:10194000270197000000E780E0970504E1B717033F
:10195000FFFFE702837289692A8AAE8A328BB68BCF
:101960008144174CFF1F130CEC43930C8006314D40
:10197000FD199790FFFFE780E00A63C6A4001703F4
:10198000FFFF670043733389940383270C02835559
:10199000CA015A863E994A8597000000E780609EFA
:1019A00031C1814D15A03384AD038327090303D6CC
:1019B0000B00D68533F6C9003E94228597000000BF
:1019C000E780E0B609E9850D9790FFFFE780800387
:1019D000E3CBADFC01A8228597000000E780E08AF8
:1019E00023040400850471B71703FFFFE70263694E
:1019F0004169AA8A014A174BFF1F130BAB3A7D19A5
:101A0000C14B054C9790FFFFE780C0016346AA00D9
:101A10001703FFFF6700636A93098006B3073A0361
:101A200083290B02BE9983D7E900638E2701638463
:101A30002A01639A570103A4890301E84E859700A0
:101A40000000E780C0BD050A75BF83570401639994
:101A500077099304C400268597A0FFFFE78060D331
:101A600085452A8D2685835C040197A0FFFFE780CA
:101A7000C0CF268597A0FFFFE780A0E762056185BC
:101A8000635905048D45268597A0FFFFE780E0CDCB
:101A90008945268597A0FFFFE78020CD89452685CB
:101AA00097A0FFFFE78060CC8545268597A0FFFFC4
:101AB000E780E0CC83470500094793F7F707639A6F
:101AC000E7009945268597A0FFFFE78040CBA3025A
:101AD00085014848337D2D01231894016A9548C437
:101AE0000040A1BF1703FFFFE702235C37E40400B7
:101AF0008327041D82979747FF1F83C7A7171725C2
:101B0000FF1F1305E59EA300F5008327441C829761
:101B10008327841C81461306F00F81450145829777
:101B20001703FFFF6700A35A1747FF1F1307870418
:101B300018439745FF1F83C5E5139747FF1F9387FA
:101B4000E71183468703034697036397D5009747BA
:101B5000FF1F2381C712828083C587010347A70324
:101B60006317B6009747FF1F2386E710828003C6DE
:101B700087016317C7009747FF1F238DD70E828009
:101B800083C68701130750026319D70093076002C9
:101B90001747FF1F2300F70E828083C687011306B5
:101BA00060026315D60093077002DDB783C7870113
:101BB00055BF9747FF1F9387670AD44B0947638D2B
:101BC000E6081703FFFFE702434E1749FF1F1309FB
:101BD00029063E8483470900918B9DCFB7E404001A
:101BE00083A7041D829783A7441C1745FF1F130575
:101BF000A504829783A7841C81461746FF1F0346CE
:101C0000A60581450145829721C583470900ED9BC3
:101C10001747FF1F230EF7008347040093F7F70FC2
:101C200085CB91471747FF1F2324F7049700000037
:101C3000E78080EB97000000E78040EFB7E7040003
:101C4000BC4F414691451745FF1F0345A5018297AB
:101C50001703FFFF6700A34782801703FFFFE70218
:101C6000C3448D4741116306F504C5476308F50277
:101C700085476310F5029747FF1F238FA7FEB7E73D
:101C80000400BC4B930500101745FF1F034585FD5D
:101C9000829741011703FFFF67006343854717479A
:101CA000FF1F230BF7FCB7E70400BC4B9305002094
:101CB000E1BF9747FF1F938767FAD44B1147638DA6
:101CC000E600B7E7040083A7071D8297B7E7040083
:101CD000BC4B930500044DBF05491747FF1F23293F
:101CE00027F983C7070032C62E8493F7F70FD5D3A1
:101CF000B7E4040083A7041D7D141374F40F8297C6
:101D0000E37689FCB245994703C61500E3F0C7FCAA
:101D1000FC4409061745FF1F130545F68297BC488A
:101D2000930500081745FF1F0345C5F3829779BF48
:101D30001703FFFFE70263371747FF1F130707F279
:101D40004047184B1C409746FF1F23AFF6F0631621
:101D5000E4001747FF1F232BF7F0130584FE97902D
:101D6000FFFFE78000AA035564FF9780FFFFE7802D
:101D7000807297A0FFFFE78060D01703FFFF670026
:101D800003351703FFFFE70243329747FF1F93878F
:101D9000E7ECD84BDC4789C797000000E78080F963
:101DA00085471747FF1F2325F7EC9747FF1F9387AA
:101DB00067DC9C43930500021745FF1F034585EA36
:101DC00083C787031747FF1F2306F7EAB7E7040017
:101DD000BC4B82971703FFFF6700632F9747FF1FD6
:101DE00023A0A7E882801703FFFFE702632A37E4F6
:101DF00004007C4CA1451745FF1F0345A5E68297CB
:101E00007C48A1451745FF1F0345C5E59744FF1FC3
:101E10009384C4E48297DC4489EB97000000E78058
:101E200080D91703FFFF6700E32903D567FF978079
:101E3000FFFFE7804066AA896DD1D84891476310BB
:101E4000F7027C4C91451745FF1F0345A5E182979A
:101E50007C4891451745FF1F0345C5E0829703A9BC
:101E6000490103D409018947B7E904001747FF1F57
:101E70002320F7E083A7091D21044204829783C72A
:101E800084011715FF1F1305A56661191717FF1F9A
:101E9000A300F76683A7491C418082979747FF1FDD
:101EA000238C07DC83A7C91C814609469375F40F70
:101EB0004A85829711E99747FF1F83C727EC89C797
:101EC0009710FF1FE780A0CFB7E70400BC4F214663
:101ED000A1451745FF1F0345E5D8829799B717031A
:101EE000FFFFE702831C93F7052001112E8481CFA9
:101EF00097000000E78020E91345042005611703DF
:101F0000FFFF6700C31C93F70510A9CF9744FF1F7D
:101F10009384C4D4DC4897000000E78020C11747B1
:101F2000FF1F130727C5184383C78401034787038F
:101F30006318F700DC4489C797000000E78080DF62
:101F400085471747FF1F2325F7D2B7E70400BC4B8F
:101F5000930500021745FF1F0345C5D0829713451F
:101F6000041069BF93F70508BDC79747FF1F83C7D4
:101F7000F7D0E91719469745FF1F938545D01305FC
:101F8000D10093F4F70F1749FF1F034929CF97C0DA
:101F90000000E780404093970401C1831747FF1F6B
:101FA000130747CE231DF100231CF1009747FF1FA5
:101FB0009387C7CA3ACE3ACAD8432306010009CB51
:101FC000DC439315890154080D46E185680082972A
:101FD0001345040825B793F72500A5C39747FF1FAE
:101FE0009387C7C7D84B89476306F7029747FF1FF8
:101FF00083C707C413F7270011EF918B99CFB7E779
:102000000400BC4F1306000A89451745FF1F03450E
:1020100065C5829713452400D5B59747FF1F938761
:1020200067B59C4383C787031747FF1F2304F7C483
:1020300097000000E78060DBF1BF93F7050281CBDA
:1020400097000000E78060DA1345040245BD93F76E
:10205000850081CB97000000E780E0D21345840023
:1020600071BD93F7150081CB97000000E780A0B405
:102070001345140061B593F7450081CB970000002C
:10208000E78060B31345440095BD93F7050495C3FD
:102090009747FF1F83C787BC91CB97000000E7805D
:1020A000A0A491471747FF1F2324F7BC134504043E
:1020B000B1B593F705010145E38207E49747FF1F98
:1020C0009387C7B9D84B91476310F7049747FF1F11
:1020D000938707B69C4313D727008583D98F858BB9
:1020E00091E7B7E7040083A7071D8297B7E70400CD
:1020F000FC4F91451745FF1F0345C5B6829785479D
:102100001747FF1F2326F7B613450401C5BB9747A2
:10211000FF1F2385A7C682801703FFFFE702E3F8AE
:102120009747FF1F23A207B49747FF1F23A007B4B9
:1021300085471744FF1F1304E4A31747FF1F2329F4
:10214000F7B21C4083C787031747FF1F2304F7B26A
:102150009790FFFFE780409329C59717FF1F23AD96
:10216000A7381C40170500001305A5D783C78703B0
:102170001747FF1F2300F7B01717FF1FA30AF736F3
:102180009747FF1FA38C07ACB7E7040083A7070896
:1021900082979747FF1F2387A7AC1703FFFF6700AE
:1021A00003F3B7C7898E938767ED1717FF1F2325A2
:1021B000F73445BF1747FF1F034747AA795555E72F
:1021C0009747FF1F938787A903C7170005079746FF
:1021D000FF1FA385E6A803C717008D463377D702F4
:1021E0009746FF1FA38CE6A683C617001747FF1F5D
:1021F00013074798184393F6F60FA9EE8347870312
:102200001747FF1F2308F7A685471747FF1F230718
:10221000F7A49747FF1F9387A7A19C430145998B7C
:10222000A9E71703FFFFE70243E837E404007C480F
:10223000C1451745FF1F0345E5A282973C488545E8
:102240001745FF1F034505A2829701451703FFFFAE
:102250006700E3E783C7170085466395F600834769
:10226000970379BF8347A70361BF82809747FF1F0A
:1022700083C7C79EA1CF1703FFFFE70203E337E43D
:1022800004009747FF1F238B079C7C488545174513
:10229000FF1F0345259D82977C4C91451745FF1FE5
:1022A0000345459C82977C4891451745FF1F034590
:1022B000659B82973C48C1451745FF1F0345859A9A
:1022C000829701451703FFFF670063E0795582801D
:1022D0001703FFFFE70263DD2A84035565FF97803C
:1022E000FFFFE780401B9747FF1F93872797D8473B
:1022F000BE841DEF9790FFFFE78080779C482320E6
:1023000004009DEB9747FF1F23A287969747FF1F67
:1023100023AC8794B7E70400BC4B89451745FF1FE2
:1023200003454594829701451703FFFF670023DAB1
:10233000630A8700184375BF80C39747FF1F23A711
:102340008792C9BF7955CDB71703FFFFE702E3D5E1
:102350009747FF1F9387C7A288432326050023249E
:102360000500510597A00000E780C0331703FFFF69
:102370006700E3D51703FFFFE70223D31744FF1FCE
:10238000130404A01C40411199CF9C472302B500BF
:102390002AC61CC197000000E78040FB1C409C4BF4
:1023A00099C33245829741011703FFFF670023D28B
:1023B0001703FFFFE70263CF4111444D328532849A
:1023C0002EC69790FFFFE780C0522AC422859790BF
:1023D000FFFFE780205403A84400630C0800B245C7
:1023E000835744001840224683D54500AA86268597
:1023F000029841011703FFFF670063CD1703FFFF3A
:10240000E702A3CA404D1DC808C097050000938588
:1024100065031305440197A00000E7804016974725
:10242000FF1F9387E7959C43014589E79747FF1F67
:1024300023A887941703FFFF670063C97D55DDBF9D
:102440001703FFFFE70263C6011168009305F00F51
:1024500002C602C802CA02CC02CE97000000E78082
:10246000A0F105611703FFFF670063C69747FF1FD1
:10247000938707919C43D847A1679D076319F7028B
:102480001703FFFFE70263C2011132859790FFFF38
:10249000E7802046230AA1008145680097000000DC
:1024A000E78080ED05611703FFFF670043C282806C
:1024B0009747FF1F9387C78C9C43D847A167938793
:1024C00077036319F7021703FFFFE70203BE011149
:1024D00032859790FFFFE780C041230AA100814524
:1024E000680097000000E78020E905611703FFFFFF
:1024F0006700E3BD82809747FF1F938767889C43EF
:10250000D84795476316F7041703FFFFE702E3B9BF
:102510000111328532849790FFFFE780803D230AC6
:10252000A10022859790FFFFE780C03E83574400BB
:10253000231BA10081453ECC1C4068003ECE970085
:102540000000E78060E305611703FFFF670023B821
:102550008280930785FF8DC38327C5FF91CFDC4B16
:1025600081CF1703FFFFE70243B4032585FF82975E
:102570001703FFFF6700A3B582801703FFFFE70281
:10258000C3B22A8432859790FFFFE7808036BD472B
:1025900063EBA70018449377F5000345B700419912
:1025A0005D8DA305A7001703FFFF670043B2170364
:1025B000FFFFE70283AF01117C003ECAB7070700A7
:1025C0003ECC7C003ECE5C4DA9C72A841385870093
:1025D000AE8497A00000E780E0FCA1652A899D05F4
:1025E00048089770FFFFE780603E9305803EB34543
:1025F000B902480893F5F50F9790FFFFE780C021D7
:10260000014781465008A68522859770FFFFE78025
:10261000406105611703FFFF670063AB1703FFFF0E
:10262000E702A3A897000000E780A0F81703FFFFC8
:102630006700E3A91703FFFFE70223A701117C004E
:10264000AE843ECAA165B70707002A843ECC48087D
:102650007C00938575033ECE9770FFFFE7800037BF
:102660001C44480883C5B700BD899790FFFFE780E9
:10267000A01A500801478146A68522859770FFFF62
:10268000E780205A05611703FFFF670043A4170383
:10269000FFFFE70283A12A84AE8497000000E78051
:1026A00000EEA685228597000000E780E0F817037A
:1026B000FFFF6700C3A11703FFFFE702039F970017
:1026C0000000E78060F71703FFFF670043A01703D0
:1026D000FFFFE702839D0329C50141116308090239
:1026E0002A843285B2849790FFFFE78080202AC633
:1026F00026859790FFFFE780E021832749002A86FF
:1027000091C7DC4781C7B2452285829741011703F3
:10271000FFFF6700C39B1703FFFFE7020399444DC8
:1027200091CC2A8432859790FFFFE780A01EDC4081
:10273000AA8589C79C4799C3228582971703FFFF03
:102740006700E3981703FFFFE7028394032AC5019C
:102750004111630D0A062E89AA849545328532847B
:102760009770FFFFE7808026854522859790FFFFC1
:10277000E7804004AA89CA8522859790FFFFE780F9
:10278000A00B83274A008DCBDC439DC72285979001
:10279000FFFFE780A00083274A00104083564400D3
:1027A000DC437115A307A100B2961307F1004E8612
:1027B000CA852685829701C52380090001A8834523
:1027C000F10022859790FFFFE780C0FE41011703CB
:1027D000FFFF6700238F1703FFFFE702038D65717B
:1027E0001C083EC2B70780013EC41C0832893EC6A1
:1027F0002A84AE8497000000E780A0ED4A85979078
:10280000FFFFE78020118357A1008DC3AA855000E8
:10281000228597000000E78020F3014781465000A1
:10282000A68522859770FFFFE780A03F59611703B7
:10283000FFFF6700C3891703FFFFE7026385657128
:102840001C088329C5013EC2B70780013EC41C088D
:102850002A84AE8432893EC697000000E780E0EB10
:10286000638A09024A859790FFFFE780A00A835791
:10287000A100AA8585C35000228597000000E7804B
:10288000A0EC014781465000A68522859770FFFF86
:10289000E780203959611703FFFF6700A382170300
:1028A000FFFFE702838065711C083EC2B707800105
:1028B0003EC42A841C0832853EC6AE849790FFFF32
:1028C000E78040058357A1008DC3AA85500022856B
:1028D00097000000E78040E7014781465000A68549
:1028E00022859770FFFFE780C033596117F3FEFF21
:1028F0006700E37D17F3FEFFE702237B444D81EC85
:102900008347450093B71700B307F0403E8517F3A0
:10291000FEFF6700C37B1845FD576DDB970700007E
:10292000938747032A845CCB970500009385A5C253
:102930001385840097A00000E78060C480C003472F
:102940004400814761F71737FF1F232D97427DBF52
:1029500017F3FEFFE702C3738329C5014111032961
:10296000850081476387090A0324090191452A8A62
:1029700022859770FFFFE780600585452285979047
:10298000FFFFE78020E38945AA8A22859790FFFF11
:10299000E78040E2AA849770FFFFE780400A83A7A0
:1029A00049002A8B8DCB9C439DC722859790FFFFC2
:1029B000E780C0DE83A74900A306A100104083562C
:1029C00044009C431307D100B296D6851306E1005C
:1029D0005285829709CD83570B002380F400A18391
:1029E000A380F40023800A00A306010039A88357BE
:1029F000E10022852380F4008345D100A183A380D8
:102A0000F4009790FFFFE780E0DA8347D100B33707
:102A1000F0000347B900920701453D9BD98FA305FC
:102A2000F900410117F3FEFF6700C36917F3FEFFCA
:102A3000E702A36741110DED9737FF1F9387873496
:102A4000804315C80440130984009DC95C4099C7A0
:102A50009C4B89C726852EC68297B2459307803E38
:102A6000B385F5024A8597A00000E78060C121A0E8
:102A7000404DAA8469F8410117F3FEFF6700236502
:102A80004A8597A00000E780E0C15C40EDD7DC4BB1
:102A9000FDD326858297C5B717F3FEFFE702E360F3
:102AA0002A8432859790FFFFE780A0E4AA852285DB
:102AB00097000000E780C0F717F3FEFF670023616F
:102AC00017F3FEFFE702635E2A84AE8497000000DE
:102AD000E780C0FCA685228597000000E78060ADF6
:102AE00017F3FEFF6700A35E08413355B500058963
:102AF000828017F3FEFFE702435B1734FF1F1304C6
:102B0000642A1C5C0111231701008D83858BA303AC
:102B1000F1008327040B231801002319010003D7B8
:102B2000C7013ECA3C002314E1007D572315E10094
:102B30000357C4023ECC02CE2316E1009770FFFF7C
:102B4000E78020CE8357E101231EA10093F707E021
:102B500093E71710231FF1009737FF1F83C727271D
:102B600095C305470145638AE7008347840393E7DC
:102B700027001737FF1F2303F726056117F3FEFF12
:102B80006700E354814717F70000130767DB8546AA
:102B9000130671008545480897900000E780408F34
:102BA00069FD83478403F59B1737FF1F2308F7222E
:102BB00085471737FF1F230CF720C1B717F3FEFF18
:102BC000E702A34B973DFF1F938DCD1D03A6CD06B6
:102BD00039712A8981478144930600023357F600F0
:102BE000058B01C7850493F4F40F8507E398D7FE9E
:102BF00083A70D0B231701022318010203D7C70176
